:020000040800F2
:10000000700B00209D0100082B370008BD2D000853
:1000100029370008E90300088D48000800000000A7
:100020000000000000000000000000006D3C00081F
:10003000EB030008000000004B370008953C000867
:10004000B7010008B7010008B7010008B7010008B0
:10005000B7010008B7010008B7010008B7010008A0
:10006000B7010008B7010008B7010008B701000890
:10007000B7010008B7010008B7010008B701000880
:10008000B7010008B7010008B7010008B701000870
:10009000B7010008B7010008B7010008ED03000828
:1000A000B7010008B7010008B7010008B701000850
:1000B000B7010008B7010008B7010008B701000840
:1000C000B7010008B7010008B7010008B701000830
:1000D000B701000881480008B7010008B70100080F
:1000E000B7010008B7010008B7010008B701000810
:1000F000B7010008B7010008B7010008B701000800
:10010000B7010008B7010008B7010008B7010008EF
:10011000B7010008B7010008B7010008193D000841
:10012000B7010008B7010008B7010008B7010008CF
:10013000B7010008B7010008B7010008B7010008BF
:10014000B7010008B7010008B7010008B7010008AF
:10015000B7010008B7010008B7010008B70100089F
:10016000B7010008B7010008B7010008B70100088F
:10017000B7010008B70100080000000000000000FF
:10018000B7010008B7010008DFF80CD000F08CF8C8
:100190000048004719490008700B002006488047B6
:1001A00006480047FEE7FEE7FEE7FEE7FEE7FEE75C
:1001B000FEE7FEE7FEE7FEE7093D000889010008CB
:1001C0002DE9F05F0546002092469B46884606468C
:1001D000814640241BE0284641464746224600F01F
:1001E00052F853465A46C01A914110D31146184648
:1001F000224600F039F82D1A67EB01084F462246D7
:100200000120002100F030F817EB00094E41201EBC
:10021000A4F10104DFDC484631462A46434600F09B
:1002200000B830BCBDE8C09FD2B201E000F8012B9D
:10023000491EFBD270470022F6E710B513460A4666
:1002400004461946FFF7F0FF204610BD10B5002206
:1002500000E0521C835C8C5CA34201D1002BF8D1DE
:10026000D8B2E1B2401A10BD202A04DB203A00FACD
:1002700002F1002070479140C2F1200320FA03F3FD
:10028000194390407047202A04DB203A21FA02F0FB
:100290000021704721FA02F3D040C2F120029140C0
:1002A0000843194670470000064C074D06E0E06819
:1002B00040F0010394E8070098471034AC42F6D3AD
:1002C000FFF766FF083001082830010870B50446C2
:1002D000006881688268C1F3400112F0010F28D0E4
:1002E00039BB816801F00D01012914D18168124ADE
:1002F0001140891C816021680320086000F09CFE89
:10030000054612E000F098FE401B02280DD9206837
:100310008068C00709D0606D40F010006065A06D76
:1003200040F00100A065012070BD20688068C00712
:10033000E8D1002070BD0000C0FFFF7FF8B5044683
:10034000002000902068816811F0010F41D1816880
:10035000214A11422ED18168D5432940491C816030
:100360001E48806800F0E07000020DD51C481D4951
:100370000068B0FBF1F0401C00EB4000800000E0A2
:10038000401E00900028FBD100F056FE06461BE000
:10039000816811F0010F03D181682940491C8160F7
:1003A00000F04AFE801B02280ED920680068C04376
:1003B000C00709D0606D40F010006065A06D40F08E
:1003C0000100A0650120F8BD20680168C943C90784
:1003D000DED10020F8BD00003F0000800003045083
:1003E0001C000020400D0300FEE7704710B54FF4DD
:1003F000807000F0F3FCBDE810404FF4007000F096
:10040000EDBC72B6FEE70000F8B500260446009683
:1004100090F850000D4601280BD0012084F85000C0
:100420002046FFF753FF0100606D04D040F010003C
:100430002BE00220F8BD20F4885040F002006065F7
:1004400020688268134B1A4005F080431A4342F03B
:10045000004282604FF4912320680EE0009A521C03
:1004600000929A4209D3606D20F0020040F0100023
:10047000606584F850600120F8BD8268D20FEDD12C
:10048000606D20F0020040F00100606584F850606B
:100490000846F8BDC0FFFF3F2DE9F047044690F83D
:1004A00050009AB00E464FF00009012816D00120E6
:1004B00084F85000002515951695324F2068B842F3
:1004C00010D1DFF8C480CDF80080404602F032FF42
:1004D0008246206802F02EFF60B10EE002201AB0C2
:1004E000BDE8F087606D40F02000606584F85050F2
:1004F0000120F4E7BAF1000F0AD0606D40F020004F
:1005000060654FF0010900BF84F850504846E6E7A7
:100510001E4831681E4A0029816840F61F7321F485
:1005200060411CD094F830C041EA4C31D6F804C088
:1005300041EA0C018160B968D8F8087001F0010146
:1005400007F001079268394302F001021143DBD141
:10055000B2683168114382689A4311430FE08160A9
:10056000B968D8F8086001F0010106F00106926848
:10057000314302F001021143C6D181689943816081
:10058000C2E70000000004500001045000030450C2
:10059000000204502DE9F84F00270446009790F818
:1005A0005000DFF8B8930D46B846012811D0012657
:1005B00084F85060206802F0B9FE60B1606D40F0D0
:1005C000200060655FF0010784F85080384600F035
:1005D000DDB90220FBE76868052808D8022825D085
:1005E000032825D0042825D0052825D006202168F9
:1005F0000C2303EA901319442A680B6B00F01F00C8
:100600004FF01F0C0CFA00FCC2F3846223EA0C03C7
:10061000824013430B63206802F088FE8246206804
:1006200002F080FE5AEA000009D09AE00C20DEE7D2
:100630001220DCE71820DAE74FF48070D7E7AA68C9
:100640002968206802F07AFE20686969C268C2F3EE
:10065000C102520091402A69042A0FD000EB8200A7
:100660002B68026EDFF8F8C203F0F84302EA0C02CE
:100670000B431A4342F00041016672E0002102F090
:100680004BFE400320684FF0000172D002F044FEA0
:1006900090FAA0F0B0FA80F1286842036ED090FA88
:1006A000A0F0B0FA80F0814204D100221146206807
:1006B00002F053FE0121206802F02EFE4003206864
:1006C0004FF001015DD002F027FE90FAA0F0B0FAE1
:1006D00080F12868420359D090FAA0F0B0FA80F077
:1006E000814204D100220121206802F036FE02215D
:1006F000206802F011FE400320684FF0020148D04C
:1007000002F00AFE90FAA0F0B0FA80F128684203E5
:1007100044D090FAA0F0B0FA80F0814204D10022D7
:100720000221206802F019FE0321206802F0F4FD86
:10073000400320684FF0030133D002F0EDFD90FA42
:10074000A0F0B0FA80F1286842032FD090FAA0F010
:10075000B0FA80F0814204D100220321206802F027
:10076000FCFD2068816811F0010F22D0ABE000E0B1
:1007700004E002F0D1FDC0F384618DE7C0F3846032
:1007800091E702F0C9FDC0F38461A2E7C0F3846081
:10079000A6E702F0C1FDC0F38461B7E7C0F384604F
:1007A000BBE702F0B9FDC0F38461CCE7C0F384601D
:1007B000D0E72A7B296850F8B03FC1F3120C23EA36
:1007C0000C0302F0180C674A22FA0CF20A40134399
:1007D0000360E968494576D1286841031BD090FA47
:1007E000A0F1B1FA81F1491C01F01F0109294FEA7A
:1007F000403131D8002911D090FAA0F1B1FA81F13D
:1008000001F1010101F01F0106FA01F609D100BF53
:10081000C0F3846109E0C0F38461E4E7C0F384615C
:10082000EEE790FAA0F1B1FA81F101F1010101F0D6
:100830001F0146EA816102D1C0F3846003E090FAAF
:10084000A0F0B0FA80F000F1010000F01F0000EB12
:10085000400041EA005132E000290ED090FAA0F1A8
:10086000B1FA81F101F1010101F01F0106FA01F66F
:1008700006D100BFC0F3846106E0C0F38461F1E7F4
:1008800090FAA0F1B1FA81F101F1010101F01F012B
:1008900046EA816102D1C0F3846003E090FAA0F0DF
:1008A000B0FA80F000F1010000F01F002E4A00EBCA
:1008B000400002EB005041EA000141F00071AA68DB
:1008C000206802F03BFD29482A6802423FF47CAED2
:1008D00027488168274E284B284D01F0E071B2422D
:1008E0001DD10E021BD422689A4202D0AA427FF484
:1008F0006BAE826841F4000122F0E0720A4382602C
:100900001F4820490068B0FBF1F0401C00EB40009C
:10091000800000E0401E00900028FBD154E61A4EF3
:10092000B24209D1CE0107D422689A4201D0AA422C
:10093000F4D141F080710AE06FF00045EA42EDD158
:100940004A02EBD422689A42E8D141F480018268DD
:1009500022F0E0720A43826036E6000000007F4029
:1009600000F0FF03FFFF0700000020FE00000880EA
:1009700000030450000052C700000450000204505D
:100980001C000020400D0300000084CB18BCBDE813
:10099000E08F0000F8B54FF0000504002E460095EA
:1009A00002D0606D10B107E00120F8BD204600F0D4
:1009B000D3F8A66584F8506020688168C1F340715F
:1009C00019B181685A4A1140816020688168C1F379
:1009D000007189B98168574A114041F080518160A6
:1009E000554856490068B0FBF1F04000801C00E01B
:1009F000401E00900028FBD120688168C1F300717F
:100A000041B9616D41F010016165A16D41F00101D5
:100A1000A165012502F08AFC616DC90600D430B1E0
:100A2000606D40F01000606501252846F8BD606DDE
:100A300020F4807040F0020060652068806810F04B
:100A4000010F15D13E4880683E4900F001008968D9
:100A500001F0010108433C49896801F001010843A4
:100A600006D13A4960688A6822F47C1202438A609F
:100A7000E168606B627E0843A16841EA4231084345
:100A800094F8201040EA0140012904D1A18C304A99
:100A900002EB41410843A16A29B101F47071E26A95
:100AA000014342EA01002268D1682A4B1940014300
:100AB000D160206802F036FCA8B9207E94F830108E
:100AC000800340EA41012068C26844F202039A436D
:100AD0000A43C26094F8380001280CD020680169EC
:100AE00021F001010161206901282068016B21F0DA
:100AF0000F0111D013E0D4E90F010843D4E911121A
:100B00001143084321680A6940F2FC739A43104379
:100B100040F001000861E6E7E269521E11430163FB
:100B2000606D20F0020040F0010060657DE700008C
:100B3000C0FFFF5FC0FFFF7F1C000020400D0300CF
:100B4000000004500001045000020450000304504F
:100B50000000FEFF07C0F0FF10B5A8B00446142146
:100B600022A8FFF768FB88216846FFF764FB1D4950
:100B70002068884233D14FF48040009080031E905B
:100B80000320019001200290092003900720049087
:100B9000022005900620069088010790684600F024
:100BA0001DFB08B1FFF72DFC0F48C16C41F400514B
:100BB000C164C16C01F400512791C16C41F0040182
:100BC000C164C06C22A900F0040027900420229088
:100BD0000B20239000202490044800F00BF928B04B
:100BE00010BD000000000450001002400008004842
:100BF0002DE9F04104463748806800F01F05206861
:100C000002F094FB18B102210846BDE8F08194F887
:100C1000500001280CD0012084F850002046FFF736
:100C20008DFB01004FF0000304D084F85030EBE757
:100C30000220EAE7606D40F60162904340F4807064
:100C40006065254A2068254E904201D1374600E074
:100C50000746874200D01DB9676D27F48017676586
:100C6000676DFF0404D5A76D27F00607A76500E0B0
:100C7000A3651C27076084F850302068904201D19A
:100C8000334600E00346834215D0A5B1052D12D0AE
:100C9000092D10D0636D43F480136365904200D139
:100CA0003046C0688001AFD5606D20F4005040F43C
:100CB00080506065A8E7C268920105D5626D22F494
:100CC000005242F4805262658268054B1A40121D40
:100CD000826099E7000304500001045000000450B2
:100CE000C0FFFF7F10B590F825100022022905D023
:100CF0000421C16380F82420012010BD01680B6825
:100D000023F00E030B6001680B6823F001030B60F6
:100D100090F84410046C01F01C03012101FA03F364
:100D2000636080F8251080F82420104610BD10B5AF
:100D300090F825100024022903D00421C163012466
:100D40001AE001680A6822F00E020A6001680A6867
:100D500022F001020A6090F84410036C01F01C02BA
:100D6000012101FA02F25A6080F82510002180F872
:100D70002410816B01B18847204610BD70B5044630
:100D800000F05AF90546601C02D00448007804447B
:100D900000F052F9401BA042FAD370BD10000020B1
:100DA0004FF4007110B50C4A4B10884207D1194618
:100DB000104600F02EF900280DD1012007E09842DE
:100DC00009D1104600F025F9002804D1401EBDE8E5
:100DD000104002F013BE10BD00040048044910B5D5
:100DE0000A68024202D00860FFF7DAFF10BD000077
:100DF000140401402DE9F04FDFF8EC9100220127A7
:100E0000A9F1040B85B003254FF00F0C09F1040A7A
:100E1000ABF1040EE0E000BF07FA02F416EA0403A7
:100E20007ED00E7906F00306012E01D0022E1FD1CE
:100E300086680096560005FA06F80496009E26EA93
:100E400008060096D1F80C80049E08FA06F8009E69
:100E500048EA0608C0F80880466891F80480A6436E
:100E6000C8F3001808FA02F848EA0608C0F8048037
:100E7000D1F804806FEA0806B6070AD1C66AA6430D
:100E8000C8F3C00494403443C4620C79E443A4071B
:100E90000AD0C4684FEA420805FA08F6B4438E68DF
:100EA00006FA08F62643C6600C7904F00304022C07
:100EB00011D1D40800EB84060296D6F8208054079E
:100EC000E60E0CFA06F428EA04080C69B440029E07
:100ED00044EA0804346204685600029605FA06F6ED
:100EE000B4430E7906F00308029E08FA06F848EAB1
:100EF0000408C0F800804C6814F4403F6BD03B4CB1
:100F0000266E46F001062666246E22F0030604F0E3
:100F100001040094364C34440294A468960700E01F
:100F200059E04FEA16780CFA08F6B443B0F1904F46
:100F300004D0304EB04203D101261BE0002619E058
:100F40002D4EB04201D1022614E02C4EB04201D108
:100F500003260FE02A4EB04201D104260AE0294EB2
:100F6000B04201D1052605E0274EB04201D1062648
:100F700000E0072606FA08F62643029CA660D9F888
:100F800000404E46D1F804809C435FEAC82800D553
:100F90001C433460DAF800405646D1F804809C4384
:100FA0005FEA882800D51C433460DBF800405E46C9
:100FB000D1F804809C435FEA883800D51C43346034
:100FC000DEF800407646D1F804809C435FEAC838DA
:100FD00000D51C433460521C0B681E46D3407FF47E
:100FE0001BAF05B000F012B8080401400010024029
:100FF000000001400004004800080048000C0048C0
:1010000000100048001400480018004830BCBDE83B
:10101000C08F0069084000D001207047426921EA72
:1010200002030A4043EA0241816170470AB18161CB
:101030007047816270470000014880687047000077
:1010400010000020024881680278114481607047D6
:101050001000002010B50024032000F071F80F20CC
:1010600000F008F808B1012401E000F025F820465E
:1010700010BD000070B50E4E05460024307898B1C2
:101080004FF47A71B1FBF0F00A490968B1FBF0F056
:1010900000F09AFF40B9102D06D200222946501EBA
:1010A00000F02EF8756000E00124204670BD0000BD
:1010B000100000201C000020094808B5016E41F016
:1010C00001010166016E01F001010091816D41F0A5
:1010D00080518165806D00F08050009008BD000057
:1010E00000100240002809DB00F01F02012191409E
:1010F0004009800000F1E020C0F8001170470000B6
:10110000F0B40E4B1B680C46C3F30223C3F1070572
:10111000042D00D90425191D072901D2002300E060
:10112000DB1E012606FA05F1491E214099409E402A
:10113000761E16403143F0BC03F0B2BB0CED00E06C
:10114000064900F0070208684FF6FF03184040EA1E
:101150000220034A10430860704700000CED00E0D5
:101160000000FA051649B0F5007F0868C0F3412079
:1011700009D0022805D0086820F4C06040F48060DF
:101180000860002070470128FBD0086820F4C06088
:1011900040F4007008600B483222006850430A4A4D
:1011A000B0FBF2F0401C00E0401E4A69520501D538
:1011B0000028F9D148694005E3D5032070470000B5
:1011C000007000401C00002040420F0002480068F0
:1011D00000F4C06070470000007000402DE9F84F37
:1011E000044600270088E54D3E46010504F1200B2A
:1011F0001DD5606E78B1B0F5800F11D0B0F5000F3D
:1012000004D0B0F5400F22D001270FE0E86840F489
:101210008030E8601BE00021201D02F097FA03E017
:101220000021584602F028FB070010D03E462088D7
:10123000C00426D5A06EC0B1B0F1807F1AD0B0F145
:10124000007F0DD0B0F1407F19D0012718E0D5F80C
:101250008800616E20F440000843C5F88800E6E786
:10126000E86840F48030E86009E00021201D02F0C9
:101270006DFA03E00021584602F0FEFA0746F7B186
:101280003E46206880033AD5A86D4FF00008C000A4
:1012900009D4A86D40F08050A865A86D4FF00108F2
:1012A00000F080500090DFF8D8A2DAF8001041F486
:1012B0008071CAF80010FFF7BFFE814610E0D5F834
:1012C0008800A16E20F040700843C5F88800D8E778
:1012D000FFF7B2FEA0EB0900022801D9032705E0C1
:1012E000DAF80000C005F3D5002F7CD04FEA0706DE
:1012F000B8F1000F03D0A86D20F08050A8652078C9
:10130000C00707D0D5F88800A16B20F00300084380
:10131000C5F888002078800707D5D5F88800E16BEC
:1013200020F00C000843C5F888002078400707D556
:10133000D5F88800216C20F030000843C5F88800FB
:101340002078000707D5D5F88800616C20F0C00030
:101350000843C5F888002078C00607D5D5F888006E
:10136000A16C20F440700843C5F8880020788006FE
:1013700007D5D5F88800E16C20F440600843C5F833
:1013800088002088800507D5D5F88800E16D20F415
:1013900040200843C5F888002088400507D5D5F8C7
:1013A0008800216E20F440100843C5F8880020789A
:1013B000400607D5D5F88800216D20F44050084339
:1013C000C5F888002078000607D5D5F88800616D3B
:1013D00020F440400843C5F888002088C00509D59E
:1013E000D5F8880000E01CE0A16D20F440300843EF
:1013F000C5F8880020884FF0006780044FF08068AF
:101400004FD5D5F88800E16E20F040600843C5F85C
:101410008800E06EB8423CD1E86840F48010E86093
:101420003FE0D5F8900010F4407015D0D4F8841047
:10143000814211D0D5F89000D5F8901020F440707A
:1014400041F48031C5F89010D5F8901021F4803126
:10145000C5F89010C5F89000C00710D0FFF7ECFD5C
:10146000074641F2883906E0FFF7E6FDC11B494512
:1014700001D903263CE7D5F890008007F4D5D5F8CC
:101480009000D4F8841020F440700843C5F8900010
:101490002EE7404505D10121201D02F057F900B18A
:1014A00006462068000317D5D5F88800216F20F084
:1014B00040600843C5F88800206FB84204D1E8684E
:1014C00040F48010E86007E0404505D10121201D6F
:1014D00002F03CF900B106462068400317D5D5F864
:1014E0008800616F20F040600843C5F88800606F95
:1014F000B84204D1E86840F48010E86007E0404555
:1015000005D10121201D02F021F900B106462088F5
:1015100040041AD5D5F88800A16F20F04050084348
:10152000C5F88800A06FB0F1805F03D0B0F1005F14
:1015300005D00AE00221201D02F008F903E0022193
:10154000584602F099F900B106462088000407D5F4
:10155000D5F88800E16F20F080400843C5F8880086
:101560002068C00307D555F8880FD4F8801020F004
:10157000004008432860304600F004B800100240E4
:101580000070004018BCBDE8E08F00002DE9F04776
:101590000F4605006BD0494E306800F00700B84296
:1015A00009D2306820F0070038433060306800F01E
:1015B0000700B8425BD12878414C80070AD5A8685B
:1015C000A16801F0F001884204D9A16821F0F0017E
:1015D0000143A1602878C0072CD06868032811D087
:1015E000022812D0216898B1490500293FDAA16884
:1015F00021F003010143A160FFF71EFD804641F287
:10160000883910E021688901EFE721688903ECE758
:101610008907EAE7FFF710FDA0EB0801494502D969
:101620000320BDE8F087A068696800F00C00B0EB0B
:10163000810FEFD1287880070AD5A868A16801F04A
:10164000F001884204D2A16821F0F0010143A160B9
:10165000306800F00700B8420BD9306820F007006E
:1016600038433060306800F00700B84201D00120F4
:10167000D7E72878400705D5A068E96820F4E0603E
:101680000843A0602878000706D5A068296920F4DF
:10169000605040EAC100A06000F03EF8A168094A2D
:1016A000C1F30311515C01F01F01C84006490860F5
:1016B00006480068BDE8F047FFF7DCBC00200240A8
:1016C00000100240C02F01081C0000201400002060
:1016D0000548064900688968054AC1F30221515C42
:1016E00001F01F01C84070471C000020001002409C
:1016F000003001080548064900688968054AC1F3B9
:10170000C221515C01F01F01C84070471C0000203D
:10171000001002400030010870B52549002318462A
:101720008A68CC6812F00C0204F00306214C4FEAE0
:10173000640509D00C2A05D0042A32D0082A00D129
:10174000284670BD012E10D10B681B0704D4D1F8B8
:101750009430C3F3032302E00B68C3F30313164E64
:1017600056F82330DAB10C2AEBD1C86800F0030038
:10177000022818D0032818D01846CA68CB68C2F3CC
:101780000212C3F306234343521CB3FBF2F2C868B0
:10179000C0F34160401C4000B2FBF0F070BD184641
:1017A00070BD204670BD2046E7E72846E5E700000B
:1017B000001002400024F400D02F01082DE9F84366
:1017C00004006FD0FD4DA86800F00C06E86800F03A
:1017D00003072078C00664D576B10C2E01D1012F05
:1017E0000AD0A069002828687AD040F0010028605B
:1017F000FFF722FC80465DE02868800702D5A069DB
:101800000028DED0216A2868000703D5286800F088
:10181000F00004E0D5F89400F02202EA10108142B2
:1018200016D9084602F0ACF800283BD1286840F0F1
:10183000080028602868216A20F0F000084328602A
:101840006868E16920F47F4040EA0120686016E0A2
:10185000286840F0080028602868216A20F0F0001D
:10186000084328606868E16920F47F4040EA01206D
:10187000686026B9206A02F083F80028D5D1FFF706
:101880004BFFA968CE4AC1F30311515C01F01F015F
:10189000C840CC490860CC480068FFF7EBFB002843
:1018A0007ED12EE0CAE000BFFFF7C6FBA0EB080028
:1018B000022876D828688007F6D5286840F0080006
:1018C00028602868216A20F0F000084328606868D2
:1018D000E16920F47F4040EA0120686011E0FFE701
:1018E00020F001002860FFF7A7FB804606E000BF5C
:1018F000FFF7A2FBA0EB08000228DAD828688007CF
:10190000F6D42078C00740D0082E18D00C2E01D174
:10191000032F14D06068B0F5803F17D0B0F5A02F2A
:10192000286817D020F480302860286820F48020B0
:1019300028606068E0B1FFF77FFB804614E028680C
:10194000800322D56068002878D01EE0286840F423
:101950008030EDE740F480202860F7E7FFF76CFB6C
:10196000A0EB08006428A4D828688003F6D50CE012
:10197000FFF762FB804605E0FFF75EFBA0EB080087
:10198000642896D828688003F6D4207880073BD551
:10199000042E11D00C2E01D1022F0DD0E06801E0F1
:1019A00086E1D6E0002828681ED040F480702860C8
:1019B000FFF742FB07460CE0286840050CD5E068BD
:1019C0000028C1D008E000BFFFF736FBC01B02288B
:1019D00093D828684005F7D56868217C20F0F85036
:1019E00040EA016068600FE020F480702860FFF733
:1019F00023FB074605E000BFFFF71EFBC01B0228C4
:101A0000B1D828684005F7D42078000729D5606947
:101A10000028D5F8940012D040F00100C5F89400D9
:101A2000FFF70AFB074604E0FFF706FBC01B02288E
:101A300099D8D5F894008007F6D512E000E120F09F
:101A40000100C5F89400FFF7F7FA074605E000BF6C
:101A5000FFF7F2FAC01B02287BD8D5F89400800764
:101A6000F6D42078400766D5A86D0027C00008D4BA
:101A7000A86D40F08050A865A86D012700F0805047
:101A8000009052480168C90512D40168814641F4AA
:101A900080710160FFF7D0FA804605E0FFF7CCFACD
:101AA000A0EB0800022854D8D9F80000C005F5D5ED
:101AB000A068012816D00528D5F8900017D020F08E
:101AC0000100C5F89000D5F8900020F0040000BF98
:101AD000C5F89000A06841F28839C0B1FFF7ACFAB0
:101AE00080460FE0D5F8900040F00100F0E740F0AC
:101AF0000400C5F89000F5E7FFF79EFAA0EB080197
:101B0000494526D8D5F890008007F5D50EE0FFF7B7
:101B100093FA804606E000BFFFF78EFAA0EB0801BB
:101B2000494516D8D5F890008007F5D41FB1A86DA7
:101B300020F08050A865A06AF0B302280AD00C2ECD
:101B40007ED0286820F080702860FFF775FA044680
:101B5000B0E0ACE0E868E26A00F00301914229D10C
:101B6000216B00F0700209011039914222D1626BA1
:101B700000F4FE41B1EB022F1CD1A26B00F4003146
:101B8000072A01D0012200E00022914212D1A18F48
:101B900000F4C00249084905A1F50011914209D19C
:101BA00094F8401000F0C06049084906A1F10071A6
:101BB00081425ED00C2E0BE072E00000001002406B
:101BC000C02F01081C0000201400002000700040FD
:101BD00079D02868400176D42868C00073D428687A
:101BE00020F080702860FFF727FA064605E000BF66
:101BF000FFF722FA801B022859D828688001F7D401
:101C0000D4E90B016FF00F0202EB01110843A18F21
:101C10005204490802EB4151626B41EA0221084338
:101C200094F840104FF07E42490802EB41610843AE
:101C3000A16B090940EA4140E968244A114000E0EB
:101C400041E00843E860286840F080702860E86858
:101C500040F08070E860FFF7EFF9044605E000BF50
:101C6000FFF7EAF9001B022821D828688001F7D580
:101C700027E02868800124D4286840F0807028601C
:101C8000E86840F08070E860FFF7D6F9044604E0A9
:101C9000FFF7D2F9001B022809D828688001F7D580
:101CA0000FE000BFFFF7C8F9001B022802D903208C
:101CB000BDE8F88328688001F4D4E8680449084046
:101CC000E8600020F4E70120F2E700008C809DF935
:101CD000FCFFEEFE70B5040009D0606A002540B13B
:101CE00025616561A56294F85D0040B10CE00120BA
:101CF00070BD6068B0F5827FF4D0E561F2E784F8EA
:101D00005C50204600F056F8022084F85D00206800
:101D1000016821F040010160E1684FF4E062914206
:101D200001D9002001E04FF48050B1F5706F02D06E
:101D3000914200D0A562A188228901F4827102F447
:101D400004421143227C02F002021143227D02F080
:101D500001021143228B02F400721143227F02F030
:101D60003802114394F8202002F080021143228DA2
:101D700002F40052114322681160A169042202EAB0
:101D8000114194F8242000F4805002F01002114315
:101D900094F8342002F008021143A28902F4706220
:101DA00011430143206841602566012084F85D00ED
:101DB000002070BD70B586B0044614216846FEF759
:101DC0003AFA1849206888422AD11748816D41F4AF
:101DD00000418165816D01F400410591C16C41F0C4
:101DE0000401C164C06C022400F0040005904FF4AB
:101DF000E050CDE9000402AA00200325062682E86F
:101E0000610069460948FEF7F5FF2820CDE9000486
:101E100002AA012082E8610069460548FEF7EAFF50
:101E200006B070BD003C00400010024000080048B1
:101E3000000400482DE9F84F984616468A460446A5
:101E4000FFF7FAF8814694F85D00012820D1BAF135
:101E5000000F6FD0002E6DD094F85C00012817D0D1
:101E6000012784F85C70032084F85D000025256656
:101E7000C4F838A0A687E6872564A4F84450A4F8DF
:101E800046502565E564A068B0F5004F03D00CE02E
:101E9000022000F096B82068016821F0400101603E
:101EA0002068016841F480410160206801684906AA
:101EB00003D4016841F040010160E068B0F5E06FD3
:101EC000606826D908B1012E1FD1A06B2168008857
:101ED000C86006E020688168890709D5A16B098878
:101EE000C160A06B801CA063E08F401EE0870CE007
:101EF000FFF7A2F8A0EB0901414503D3B8F1FF3F7A
:101F000003D04BE0B8F1000F48D0E08F0028E1D1BA
:101F100039E008B1012E33D1E08F0128A06B03D93D
:101F200021680088C86010E021680078087314E018
:101F3000E08725E043E020688168890713D5E18FB9
:101F40000129A16B07D90988C160A06B801CA0631F
:101F5000E08F801EECE709780173A06B401CA06342
:101F6000E08F401EE4E7FFF767F8A0EB0901414569
:101F700003D3B8F1FF3F03D010E0B8F1000F0DD04C
:101F8000E08F0028D7D14A464146204601F07AFD2D
:101F900008B120202066A06830B109E084F85D70A7
:101FA00084F85C50032074E72068C1688068009062
:101FB00084F85D7004F85C5F60680028F3D001204D
:101FC00067E718BCBDE8E08F10B5401EB0F1807F18
:101FD00001D3012010BD4FF0E02460610F21601794
:101FE00002F05EFC0020A06107202061002010BDEF
:101FF000704770477047000030B590F83C20012AC8
:102000003AD0012280F83C20CA688B6822F44072E2
:102010001A434B6822F480621A430B6822F4006270
:102020001A430B6922F480521A434B6922F400527E
:102030001A438B6A22F480421A430B8B22F47022DB
:1020400042EA03420D4D03680024AB4202D00C4D1E
:10205000AB420CD18D8C22F4700242EA0552CD695C
:1020600022F080722A43096A22F000720A435A64FD
:1020700080F83C40002030BD022030BD002C0140E3
:1020800000340140F0B590F83C20012A39D00124F9
:1020900080F83C40022280F83D2002685368956831
:1020A000194E1A4FB24201D0BA4204D123F4700C37
:1020B0004B6843EA0C0323F0700C0B6843EA0C03F3
:1020C00053600268B24210D0B2F1804F0DD0104B75
:1020D0009A420AD00F4B9A4207D00F4B9A4204D033
:1020E000BA4202D00D4B9A4204D1896825F0800390
:1020F0001943916080F83D40002180F83C1008466B
:10210000F0BD0220F0BD0000002C01400034014071
:102110000004004000080040000C00400040014066
:1021200010B5040003D094F83D0010B107E0012081
:1021300010BD002084F83C00204600F023F8022067
:1021400084F83D00211D206801F0ECFD012084F899
:10215000480084F83E0084F83F0084F8400084F88A
:10216000410084F8420084F8430084F8440084F875
:10217000450084F8460084F8470084F83D000020BC
:1021800010BD000008B5114A01681148914211D1F3
:10219000816D41F020018165806D002200F02000FA
:1021A000009011463720FEF7ABFFBDE8084037200E
:1021B000FEF798BF074A914207D1016E41F4803182
:1021C0000166006E00F48030009008BD00140040ED
:1021D000001002400040014090F83D10012901D05C
:1021E00001207047022180F83D100168CA6842F062
:1021F0000102CA6000681149884211D0B0F1804FD5
:102200000ED00F4988420BD00E49884208D00E49A3
:10221000884205D00D49884202D00D49884207D135
:1022200081680C4A1140062906D0B1F5803F03D0E1
:10223000016841F00101016000207047002C01405D
:102240000004004000080040000C00400034014041
:10225000004001400700010070B5044690F83C00C2
:102260000025012817D0012684F83C60022084F85C
:102270003D00226890682F4B184020F47F4090600A
:102280000868502838D00DDC20284FD005DC90B3EA
:10229000102811D14AE0022070BD302846D04028D5
:1022A0000AD13BE060282FD070280DD0B0F5805FB8
:1022B00003D0B0F5005F12D0012584F83D60002006
:1022C00084F83C00284670BDCB68D1E90121206824
:1022D00001F09DFD2068816841F0770109E0CB683D
:1022E000D1E90121206801F092FD2068816841F464
:1022F00080418160E1E719E0CA684968206801F01F
:1023000021FF5021206806E0CA684968206801F072
:102310002AFF6021206801F084FDCEE7CA68496881
:10232000206801F00FFF40212068F4E72268014691
:102330001046F0E788FFFEFF70472DE9F0410446A4
:102340000068C66805694FF00007A90713D5B107F3
:1023500011D5F91E0161012020772068806980076E
:10236000204602D0FFF7E8FF04E000F0CFF8204657
:1023700000F0A4F92777680716D5700714D52168EF
:102380006FF004000861022020772068806910F453
:10239000407F204602D0FFF7CFFF04E000F0B6F800
:1023A000204600F08BF92777280715D5300713D57D
:1023B00021686FF008000861042020772068C06958
:1023C0008007204602D0FFF7B7FF04E000F09EF838
:1023D000204600F073F92777E80616D5F00614D5E5
:1023E00021686FF010000861082020772068C0691C
:1023F00010F4407F204602D0FFF79EFF04E000F07B
:1024000085F8204600F05AF92777E80708D0F0074A
:1024100006D021686FF001000861204600F0D2F973
:10242000280601D4A80408D5300606D521686FF423
:10243000025008612046FFF7DCFDE80508D53006AC
:1024400006D521686FF4807008612046FFF7D0FD43
:10245000680608D5700606D521686FF0400008614F
:10246000204600F0D9F9A8060AD5B00608D521689B
:102470006FF0200008612046BDE8F041FFF7BABDCB
:10248000BDE8F08110B586B0044614216846FDF71A
:10249000D2FE2368184C002118480222A34211D111
:1024A000C36C43F01003C364C06C00F010000590CF
:1024B00010020090CDE901210120CDE90310694609
:1024C0000F4814E00F4CA34213D1C36C43F0020336
:1024D000C364C06C00F0020005904FF4004000900F
:1024E000CDE901210E20CDE9031069460648FEF72B
:1024F00081FC06B010BD0000002C0140001002401D
:10250000001000480040014000040048704770B5CA
:10251000044690F83C0000260D4601280BD001200F
:1025200084F83C000C2A4AD007DC82B1042A20D06F
:10253000082A06D131E0022070BD102A53D0142A97
:1025400063D00126002084F83C00304670BD20682E
:1025500001F070FC2068816941F008018161206808
:10256000816921F004018161206881692A69114330
:1025700011E0206801F0ACFC2068816941F4006141
:1025800081612068816921F48061816120688169AD
:102590002A6941EA02218161D4E7206801F0E0FC68
:1025A0002068C16941F00801C1612068C16921F05A
:1025B0000401C1612068C1692A69114311E02068E2
:1025C00001F016FD2068C16941F40061C161206815
:1025D000C16921F48061C1612068C1692A6941EA49
:1025E0000221C161AEE7206801F03CFD2068416D29
:1025F00041F0080141652068416D21F00401416509
:102600002068416D2A69114311E0206801F062FDE4
:102610002068416D41F4006141652068416D21F4FD
:10262000806141652068416D2A6941EA0221416566
:1026300088E710B5040003D094F83D0010B107E01E
:10264000012010BD002084F83C00204600F022F854
:10265000022084F83D00211D206801F063FB012069
:1026600084F8480084F83E0084F83F0084F8400075
:1026700084F8410084F8420084F8430084F8440060
:1026800084F8450084F8460084F8470084F83D004B
:10269000002010BD08B500680649884208D10648E8
:1026A000016E41F400610166006E00F4006000906C
:1026B00008BD0000002C01400010024070470000DF
:1026C00030B50446022269B1042912D0082917D076
:1026D0000C291CD0102921D094F84300012824D0C3
:1026E000012030BD94F83E000128F9D184F83E2045
:1026F0001DE094F83F000128F2D184F83F2016E055
:1027000094F840000128EBD184F840200FE094F8C1
:1027100041000128E4D184F8412008E094F8420007
:102720000128DDD184F8422001E084F84320012211
:10273000206801F05FFB1A4A20681A4B1A49904240
:1027400009D0984207D0884205D0184DA84202D03F
:10275000174DA84203D1456C45F4004545642068F7
:1027600090420FD0B0F1804F0CD0124A904209D065
:10277000114A904206D0114A904203D0984201D0AB
:10278000884207D181680E4A1140062906D0B1F56A
:10279000803F03D0016841F001010160002030BD9D
:1027A000002C014000340140004001400044014041
:1027B000004801400004004000080040000C0040B8
:1027C000070001001249884220D1124881784278DE
:1027D00091421BD00378012B04D0022B04D0032B91
:1027E0000AD010E082700EE08A4201D9012200E096
:1027F000002202EBC20204E08A4201D9012200E079
:10280000002211448170807801F032BA70470000D4
:10281000500600200C000020704770B50446D0F828
:1028200080000025202801D0022070BD69B162B16E
:102830000120206600206066204601F07BFF206EAC
:10284000012804D00125284670BD012070BD2168F3
:1028500010200862216851E8000F40F0100041E8A4
:102860000002002AF6D1EEE72DE9F04104460E46BB
:102870002AA002F00DF82B4884424CD12A4F0025A3
:102880002AA1BD553846FDF7E1FCDFF8A8802A4CA7
:1028900060B12AA13846FDF7D9FC78B129A13846A4
:1028A000FDF7D4FCB0B10020656028E0607818B175
:1028B00000206070802107E00120FAE7A07838B19D
:1028C0000020A0704FF480714046FEF7A7FB1BE08C
:1028D0000120F6E7207830B100202070E07820B1A8
:1028E0000020E07010E00120F7E70120F9E700BFC9
:1028F00005EB850149003A5C30395518401CB0425F
:10290000F6DB124865600570BDE8F04134220649E7
:102910000448FFF782BFBDE8F081000072780D0A1D
:1029200000000000E8060020080500204C45443166
:102930000000000000100048040000204C45443214
:10294000000000004C454433000000000D00002052
:10295000704770472DE9F04102680446D06911685C
:10296000936840F60F0528424FF000054FF002062D
:1029700005D187067ED58F067CD5A16E33E1DFF8C1
:1029800094C203F0010701EA0C0C57EA0C0C71D059
:102990005FEAC07C0CD05FEAC15C09D54FF0010C46
:1029A000C2F820C0D4F8842042F00102C4F8842088
:1029B000820709D5DA0707D022681662D4F8842086
:1029C00042F00402C4F8842042070AD5DA0708D08E
:1029D000236804221A62D4F8842042F00202C4F868
:1029E000842002070CD501F020023A4308D0236866
:1029F00008221A62D4F8842042F00802C4F8842025
:102A000002050BD54A0109D523684FF400621A620A
:102A1000D4F8842042F02002C4F88420D4F8842022
:102A2000002A36D0800605D5880603D5A16E09B1E7
:102A300020468847D4F8840021688968490602D472
:102A400010F0280F27D0204601F061FC2068806834
:102A500040061BD52068083050E8001F21F04001D7
:102A600040E80012002AF5D1606F78B16A498163AD
:102A7000606F00E015E0FEF75AF9002809D0606F9A
:102A8000816B00E02046BDE8F04108472046FFF793
:102A900060FFBDE8F0812046FFF75BFFC4F884507B
:102AA000F7E7D4F860C02027BCF1010F7ED15FEAC0
:102AB000C06C7BD55FEAC16C78D5102010622068AD
:102AC000806840064FD5616F0A6850680004000CAA
:102AD0003DD0B4F85830834239D9A4F85A00086878
:102AE000006880062BD4206850E8001F21F4807114
:102AF00040E80012002AF6D12068083050E8001F94
:102B000021F0010140E80012002AF5D120680830C8
:102B100050E8001F21F0400140E80012002AF5D1E2
:102B2000C4F880702566206850E8001F21F010016D
:102B300040E80012002AF6D1606FFEF7D3F866660F
:102B4000B4F85800B4F85A10401A81B207E0B4F84B
:102B5000581081429DD1106880069AD5666620463D
:102B6000FFF782FE95E7B4F85800B4F85A10401AFF
:102B700081B2B4F85A0000288BD0002989D022688D
:102B800052E8000F20F4907042E80003002BF6D1C9
:102B90002068083050E8002F22F0010240E80023AE
:102BA000002BF5D1C4F88070256600E00AE0A56628
:102BB000226852E8000F20F0100042E80003002BCA
:102BC000F6D1CBE7C60209D55B0207D54FF48010DA
:102BD00010622046BDE8F041FFF7BABE020606D5F6
:102BE0000A0604D5E16E00297FF44CAF51E7400698
:102BF000B8D54806B6D52046026852E8001F21F035
:102C0000400142E80013002BF6D1C767C56600F00B
:102C1000D4F83EE720010004FB42000810B5040090
:102C200002D0E06F10B107E0012010BD002084F851
:102C30007800204600F026F82420E067206801682C
:102C400021F001010160606A10B1204601F09DFA97
:102C5000204601F04BFC0128E7D02068416821F4B0
:102C6000904141602068816821F02A0181602068DC
:102C7000016841F0010101602046BDE8104001F00B
:102C8000E8BA000010B5A8B00446142122A8FDF748
:102C9000D2FA88216846FDF7CEFA1C49206888429E
:102CA00031D10120002400900E946846FEF796FA78
:102CB00008B1FDF7A6FB1648016E41F4804101669C
:102CC000016E01F480412791C16C41F00101C164A2
:102CD000C06C22A900F0010027904FF4C060229040
:102CE0000220CDE9230403202590072026904FF0F1
:102CF0009040FEF77FF8002211462520FEF700FAEB
:102D00002520FEF7EFF928B010BD00000038014083
:102D10000010024070472DE9F8430446C06F984602
:102D200016460D46202802D00220BDE8F88395B152
:102D30008EB10020C4F884002120E067FEF77CF902
:102D4000A4F850608146A4F85260A0682027B0F52E
:102D5000805F02D003E00120E7E7206910B12E4632
:102D6000002510E000260EE08021204601F03EFD07
:102D7000C0B9D6B116F8010B21680885B4F8520025
:102D8000401EA4F85200B4F852004B464FF0000227
:102D9000CDF800800028E7D14FF04001204601F037
:102DA00025FD38B1E7670320BFE735F8020BC0F314
:102DB0000800E1E7E7670020B7E77047FEE72DE985
:102DC000F04107461C4615460E462A2000F074FACC
:102DD000380A00F07FFAF8B200F07CFA280A00F016
:102DE00079FAE8B200F076FA2B2000F065FA300AA2
:102DF00000F070FAF0B200F06DFA200A00F06AFA02
:102E0000E0B200F067FABDE8F0412C2000F054BABF
:102E100070B5040AC5B2EF2300211A460846FFF731
:102E2000CEFF0F4900204FF4107200BF01F8104090
:102E300001EB4003401C80B25D709042F6D301224A
:102E400010210848FEF7F2F800244FF49065294657
:102E5000034800F033F9641CA4B2642CF7D370BDAE
:102E6000240000200004004830B5254887B0C16C1C
:102E700041F00201C164C16C01F002010591C16C15
:102E800041F00801C164C06C1E4C00F008000590C0
:102E9000D02000900120019002900220039069460A
:102EA0002046FDF7A7FF0022D0212046FEF7BEF8FE
:102EB0008020154D009069462846FDF79BFF0022B3
:102EC00080212846FEF7B2F8002280212846FEF72E
:102ED000ADF8002280212046FEF7A8F8002240210C
:102EE0002046FEF7A3F87820FDF748FF0122402195
:102EF0002046FEF79BF800F095FD07B030BD0000BE
:102F00000010024000040048000C004810B5FFF714
:102F1000ABFF7820FDF732FF112000F0CDF97820CB
:102F2000FDF72CFF362000F0C7F9002000F0D2F9A1
:102F30003A2000F0C1F9652000F0CCF9B22000F091
:102F4000BBF90C2000F0C6F90C2000F0C3F90020FA
:102F500000F0C0F9332000F0BDF9332000F0BAF9D9
:102F6000B72000F0A9F9722000F0B4F9BB2000F0FE
:102F7000A3F93D2000F0AEF9C02000F09DF92C200F
:102F800000F0A8F9C22000F097F9012000F0A2F9A2
:102F9000C32000F091F9192000F09CF9C42000F042
:102FA0008BF9202000F096F9C62000F085F90F205B
:102FB00000F090F9D02000F07FF9A42000F08AF909
:102FC000A12000F087F9E02000F076F9D02000F091
:102FD00081F9042000F07EF90D2000F07BF911202A
:102FE00000F078F9132000F075F92B2000F072F949
:102FF0003F2000F06FF9542000F06CF94C2000F0F5
:1030000069F9182000F066F90D2000F063F90B2033
:1030100000F060F91F2000F05DF9232000F05AF95C
:10302000E12000F049F9D02000F054F9042000F02C
:1030300051F90C2000F04EF9112000F04BF913204B
:1030400000F048F92C2000F045F93F2000F042F94B
:10305000442000F03FF9512000F03CF92F2000F00F
:1030600039F91F2000F036F91F2000F033F9202035
:1030700000F030F9232000F02DF9212000F01CF998
:10308000292000F019F9EF2300211A460846FFF71E
:1030900096FE4FF6FF70FFF7BBFE0122BDE8104021
:1030A00080210148FDF7C2BF00040048024601200C
:1030B00000E05043491EC9B2FBD270472DE9F041F0
:1030C0004FF6FF75B1FBF5F70E468046002411E080
:1030D00008D1B6FBF5F005FB1061C4EB044202EB2E
:1030E000080004E0C4EB044101EB0800294600F0AD
:1030F000BFFC641CBC42EBD9BDE8F0812DE9F05F58
:10310000203AD7B21C46F022A2EB540282425BD393
:10311000C4F1F0028A4257DB0A19521E93B200EB47
:103120005402521E92B2FFF74AFE3F4E102C1AD0A4
:10313000202C18D00C2C49D0182C45D13B4907EB3A
:1031400047004FF0300A002401EB00194FEA06084F
:1031500019F80460E00756D004270025300654D53E
:10316000B8F8000053E0600700D0012000EBD40065
:10317000610810FB01F000F0FF082D48002500EB6E
:10318000071A00F5BE5000EBC71BB1461AE0102C21
:1031900009D0202C18D11BF805600027300605D572
:1031A000B9F8000004E01AF80560F6E7B9F8020083
:1031B00000F09EF870067F1C060EFFB2082FEDD3BC
:1031C0006D1CEDB24545E2D300F036B8194807EB67
:1031D00047014FF00C09002400EB8108002518F886
:1031E0000470380601D5308800E0708800F080F85F
:1031F00078066D1C070EEDB2062DF2D3641CE4B206
:103200004C45EBD3E0E70827A7E7B8F8020000F049
:103210006FF870066D1C060EEDB2BD429ED3641CA5
:10322000E4B2544594D3CFE700000020B054000826
:10323000C04E00084C4A000830BCBDE8C09F2DE9D4
:10324000FF5F0027DDE90E9B1D46924680463C4607
:103250004FEA590626E0281B401EC1B20A20FFF79C
:1032600025FFBAFBF0F00A21B0FBF1F201FB1200DE
:1032700027B9691E8C4201DA38B101273030C2B259
:1032800006FB048080B24B4607E006FB0480BBF1DE
:10329000000F80B24B4609D030220199FFF72EFF74
:1032A000641CE4B2AC42D6D300F002B82022F4E7AA
:1032B0003FBCBDE8C09F000001B5002210210448BA
:1032C000FDF7B4FE01216846FFF7F8FE08BD0000D7
:1032D0000004004801B5012210210448FDF7A6FEB4
:1032E00001216846FFF7EAFE08BD0000000400481F
:1032F00008B500210091010A8DF800108DF8010039
:10330000012210210348FDF791FE02216846FFF7D4
:10331000D5FE08BD0004004800EB8100006E00F0FF
:10332000F84070478068C0F3C00070478068C0F301
:10333000800070478068C0F380007047042303EA70
:10334000D15310B518444369C1F3045107248C408C
:10335000A3438A401343436110BD00EB8100016E1B
:1033600021F00041114301667047000030B589B07B
:10337000002406940794182168460894FCF75BFF24
:103380001C481B49042501604FF48021C0E9011449
:10339000C460C0E90445047644760121C16180F827
:1033A00020408462C46280F83040446380F8384032
:1033B000FDF7F0FA08B1FDF724F806A90D480694C8
:1033C000FDF76AF808B1FDF71CF80B4800900620DD
:1033D000CDE901047F200594CDE903056946054840
:1033E000FDF7D8F8002801D0FDF70BF809B030BD83
:1033F000000004503C0500200800900C2DE9F0412D
:1034000086B014216846FCF716FF3048C16C41F0C5
:103410008001C164C16C01F080010591C16C41F073
:103420000401C164C16C01F004010591C16C41F05B
:103430000201C164C16C01F002010591C16C41F04F
:103440001001C164C16C01F010010591C16C41F023
:103450000101C164C06CDFF8788000F001000590C4
:10346000002204214046FDF7E1FD1A4F4FF4C076DB
:10347000002231463846FDF7D9FD01240420CDE96C
:103480000004002569464046CDE90245FDF7B2FC3F
:10349000CDE9006469463846CDE90245FDF7AAFC4E
:1034A000700000904FF40410CDE9010569464046D4
:1034B000FDF7A0FC002211461720FDF721FE172082
:1034C000FDF710FE06B0BDE8F081000000100240DC
:1034D0000004004800100048124810B5104901606F
:1034E0004FF48271416000214FF44072C0E9021232
:1034F0004FF400720161C0E90512C1610162072247
:103500004162C0E90A12016308214163FEF7E2FB50
:10351000002803D0BDE81040FCF773BF10BD0000C9
:10352000003C0040A005002010B59AB00024129481
:10353000139414941594169417941C210BA81894A2
:10354000FCF779FE2C216846FCF775FE29482849CE
:1035500001604721C0E9011444F61F61C0E903146A
:1035600044618461FEF7DCFD08B1FCF74AFF4FF4CB
:103570008050129012A91F48FEF76EFE08B1FCF7AA
:1035800040FF1C48FFF755F808B1FCF73AFF1694C6
:1035900016A918481894FEF775FD08B1FCF731FF1D
:1035A00060200B904FF4FA70CDE90C040E940F9448
:1035B000109404220BA90F481194FEF7A8FF08B13C
:1035C000FCF71FFF00944FF40050CDE90440019434
:1035D00002940394694607480A94FEF70DFD08B16A
:1035E000FCF70FFF0348FEF74DFF1AB010BD0000B7
:1035F000004001409C06002010B596B000241294B3
:1036000013941C210BA81494FCF715FE2C2168467A
:10361000FCF711FE23482249016040F2CF21C0E9A6
:1036200001146321C0E9031444618461FFF701F8C8
:1036300008B1FCF7E6FE1294139412A919481494E9
:10364000FEF720FD08B1FCF7DCFE60200B90642043
:10365000CDE90C040E940F94109400220BA911488C
:103660001194FEF754FF08B1FCF7CBFE00944FF421
:103670000050CDE9044001940294039400030694A1
:10368000CDE907400994694606480A94FEF7B4FC60
:1036900008B1FCF7B6FE0348FEF7F4FE16B010BD05
:1036A000002C0140040600203EB500240E48009482
:1036B00001940C490294C0E900144FF6FF71C0E96F
:1036C00002418461FEF72CFD08B1FCF79AFE0094DC
:1036D000694605480294FEF7D5FC002801D0FCF7A6
:1036E00090FE3EBD00140040500600200D4810B56D
:1036F0000B4901604FF4E1314160002181600C22EF
:10370000C160C0E904128161C16101624162FFF7D9
:1037100085FA002803D0BDE81040FCF772BE10BD4A
:1037200000380140E8060020FEE7FEE7642801D0EB
:1037300020B107E0002905DD64207047002901DA87
:10374000002070470844C0B2704770472DE9F0412F
:10375000444C05468846E0680026810728680DD05D
:10376000E16801F00301814216D1A8B1E0686968FF
:10377000C0F30210401C88420ED120E0012804D082
:10378000022805D0032807D108E02168890701E055
:1037900021684905002907DB01265FE021688903CC
:1037A00002D421684903F5E7E1686A686FF00F0306
:1037B00021F0730103EB021211430143E160206821
:1037C00020F080602060FDF737FC074605E000BF71
:1037D000FDF732FCC01B022837D820680001F7D45F
:1037E000B8F1000F18D0B8F1010F1ED0287D4FF0AE
:1037F0007E41400801EB4060A96840EA0120216950
:10380000194A114008432061206840F08060206020
:10381000FDF712FC07461AE0A868E96800020909EA
:1038200040EA41402169114AEBE7288A10494008E3
:1038300001EB4050A96840EA012021690D4AE0E708
:10384000FDF7FAFBC01B022801D9032606E0206819
:103850000001F5D52069A969084320613046BDE81B
:10386000F081000000100240FF80FFF9FF80FDFFA3
:103870000000E0FFFF809FFF2DE9F0413D4C064630
:103880008846E0680025810730680DD0E16801F0C6
:103890000301814216D1A8B1E0687168C0F302103B
:1038A000401C88420ED120E0012804D0022805D017
:1038B000032807D108E02168890701E0216849054C
:1038C000002907DB012551E02168890302D4216822
:1038D0004903F5E7E16872686FF00F0321F07301A7
:1038E00003EB021211430143E160206820F0805095
:1038F0002060FDF7A1FB074605E000BFFDF79CFB3C
:10390000C01B022829D820688000F7D4B8F1000F26
:1039100015D0307C4FF07E41400801EB4060B1682B
:1039200040EA01206169144A11400843606120683F
:1039300040F080502060FDF77FFB07460FE0B06845
:10394000F1680002090940EA414061690B4AEBE76E
:10395000FDF772FBC01B022801D9032506E0206891
:103960008000F5D560697169084360612846BDE84B
:10397000F081000000100240FF80FFF9FF80FDFF92
:10398000F8B51C4D06460024A86DC00002D5FDF711
:103990001DFC0DE0A86D40F08050A865A86D00F0FA
:1039A00080500090FDF712FCA96D21F08051A965AF
:1039B000B0F5007F04D0802E07D94FF003040AE051
:1039C000802E08D9A02E01D804E001D1022402E003
:1039D000702E00D101240848016821F0070121431D
:1039E0000160006800F00700A04201D00120F8BD8E
:1039F0000020F8BD001002400020024001460748A8
:103A000000B50078002807D0054A1068406BC0B2A6
:103A1000FFF78CFE1168486300BD0000070000201E
:103A20000406002010B5114C0F484FF4E0612060EF
:103A30004FF4827060600020C4E90201022121611C
:103A4000012161614902C4E9061020626062A0623E
:103A50000720E0622046FEF73DF92068016841F04A
:103A60004001016010BD0000003C0040A4040020A3
:103A70000A4601464FF47A730148FEF7DBB90000AD
:103A8000A4040020F8B515460E460B4600920446E5
:103A900000224FF4C05100F019F888B933460022D3
:103AA00080212046009500F085F848B93346002271
:103AB0004FF4C0612046009500F008F8002804D0BB
:103AC000206E40F0200020660320F8BD2DE9FE4F57
:103AD0004FF0000A984617460E4604460C9D8DF896
:103AE00004A0FDF7A9FA411BA8EB0105FDF7A4FA14
:103AF000814620684FF4C06B0C3002902A48006861
:103B0000C0EBC00000EB8000000D6843009043E074
:103B10005E4506D12FB9029800788DF804009DF813
:103B20000400B8F1FF3F37D0FDF786FAA0EB09009B
:103B3000A84203D215B1009858B32BE02068416821
:103B400021F0E00141606068B0F5827F0BD1A06890
:103B5000B0F5004F02D0B0F5806F04D12068016845
:103B600021F040010160A06AB0F5005F09D1206832
:103B7000016821F4005101602068016841F400519E
:103B80000160012084F85D0084F85CA0032000F04F
:103B90000DB80025401E0090206880683040B84273
:103BA000B6D10020F3E700001C0000201EBCBDE8D9
:103BB000E08F00002DE9F8431E46914688460446F2
:103BC000089DFDF739FA401B351AFDF735FA07460F
:103BD00025480068C0F3CB30684338E0701C37D00C
:103BE000FDF72AFAC01BA84203D215B1009860B3B2
:103BF0002CE02068416821F0E00141606068B0F588
:103C0000827F0BD1A068B0F5004F02D0B0F5806F75
:103C100004D12068016821F040010160A06AB0F57C
:103C2000005F09D12068016821F40051016020681B
:103C3000016841F400510160012084F85D0000201A
:103C400084F85C000320BDE8F8830025401E009046
:103C50002068816838EA010004D000214945BDD1BF
:103C60000020F0E70121F9E71C0000207047000068
:103C7000064988704FF4FA614843B42190FBF1F093
:103C8000034900F5FA700968886370470C0000204A
:103C90009C060020FDF7D6B910B596B044216846C1
:103CA000FCF7C9FA142111A8FCF7C5FA4FF400700B
:103CB000FDF758FA08B172B6FEE701210804CDE914
:103CC0000010022003240A90CDE90B4112210D912E
:103CD0000721CDE90E1010906846FDF76FFD08B181
:103CE00072B6FEE70F20CDE9110400201390149066
:103CF0001590042111A8FDF749FC002801D072B6E7
:103D0000FEE716B010BD00000248016841F47001E2
:103D10000160704788ED00E00148FEF70EBB00002F
:103D2000500600202DE9F04702682A4B2A4D2B4E01
:103D30002B4F2C4C4FF0804A984209D0504507D069
:103D4000A84205D0B04203D0B84201D0A04204D16D
:103D500022F0700C4A6842EA0C02DFF88CC0DFF8EF
:103D60008C80DFF88C9098420FD050450DD0A8423F
:103D70000BD0B04209D0B84207D0A04205D0604570
:103D800003D0404501D0484503D122F44075CA68AC
:103D90002A434D6922F080022A4302608A68C26287
:103DA0000A688262984207D0A04205D0604503D0DD
:103DB000404501D0484501D10969016301214161B4
:103DC0000169C90703D0016921F001010161BDE862
:103DD000F0870000002C0140000400400008004073
:103DE000000C00400034014000400140004401400C
:103DF0000048014010B501F01F030121046A9940F9
:103E00008C430462016A9A401143016210BD10B5EF
:103E1000846842EA032224F47F440A4322438260F6
:103E200010BD826822F070020A4342F007018160EF
:103E3000704700002DE9F043056A026A22F0010292
:103E40000262436882691C4C25F0020522400C681E
:103E500022F0030214438A68194E2A43174D194F62
:103E6000DFF864C0DFF86490A84207D0B04205D004
:103E7000B84203D0604501D0484506D122F0080879
:103E8000CA6842EA080222F00402A84207D0B042FF
:103E900005D0B84203D0604501D0484505D14D69F1
:103EA00023F440731D438B692B434360846149684D
:103EB00041630262BDE8F0838FFFFEFF002C0140EA
:103EC00000340140004001400044014000480140EE
:103ED000F0B5056A026A22F0100202624268836944
:103EE000194C1B4E23400C6823F4407343EA04240E
:103EF00025F020038D6843EA0513144DA84201D034
:103F0000B04206D1CF6823F0800343EA071323F0C1
:103F10004003A8420AD0B04208D00E4DA84205D0B6
:103F20000D4DA84202D00D4DA84207D14D6922F493
:103F3000406242EA85028D6942EA850242608461FC
:103F4000496881630362F0BDFF8FFFFE002C0140D2
:103F5000003401400040014000440140004801405D
:103F6000F0B5056A026A22F4807202624368C2698F
:103F7000194C1B4E22400C6822F00302144325F416
:103F800000728D6842EA0522144DA84201D0B04269
:103F900006D1CF6822F4006242EA072222F480624E
:103FA000A8420AD0B04208D00E4DA84205D00E4D0E
:103FB000A84202D00D4DA84207D14D6923F44053C9
:103FC00043EA05138D6943EA05134360C4614968F8
:103FD000C1630262F0BD00008FFFFEFF002C0140B4
:103FE00000340140004001400044014000480140CD
:103FF00030B5046A026A22F4805202624268C369E0
:10400000124D24F400542B400D6823F4407343EA0E
:1040100005238D6844EA05340D4DA8420BD00D4DA3
:10402000A84208D00C4DA84205D00C4DA84202D0A1
:104030000B4DA84204D14D6922F4804242EA851218
:104040004260C36149680164046230BDFF8FFFFEB6
:10405000002C014000340140004001400044014078
:104060000048014030B5056A026A22F480320262DB
:104070004268436D114C23400C681C4325F4003307
:104080000D8943EA05430E4DA8420BD00D4DA842C1
:1040900008D00D4DA84205D00C4DA84202D00C4DC1
:1040A000A84204D14D6922F4803242EA05224260DE
:1040B000446549688165036230BD00008FFFFEFFE3
:1040C000002C014000340140004001400044014008
:1040D0000048014030B5046A026A22F4801202628C
:1040E0004268436D114D24F400142B400D6843EADF
:1040F00005230D8944EA05540D4DA8420BD00D4D02
:10410000A84208D00C4DA84205D00C4DA84202D0C0
:104110000B4DA84204D14D6922F4802242EA852247
:10412000426043654968C165046230BDFF8FFFFE90
:10413000002C014000340140004001400044014097
:104140000048014010B5036A046A24F001040462C7
:10415000846924F0F00444EA021423F00A020A43BA
:104160008461026210BD10B5036A046A24F0100471
:104170000462846923F0A00324F4704444EA023208
:1041800043EA01118261016210BD90F82410090711
:1041900006D501684A68436B22F400421A434A601C
:1041A00090F82410C90706D001684A68836A22F48F
:1041B00000321A434A6090F82410890706D5016836
:1041C0004A68C36A22F480321A434A6090F8241085
:1041D000490706D501684A68036B22F480221A4316
:1041E0004A6090F82410C90606D501688A68836B76
:1041F00022F480521A438A6090F82410890606D56A
:1042000001688A68C36B22F400521A438A6090F8EE
:104210002410490611D501684A68036C22F4801203
:104220001A434A60016CB1F5801F06D101684A68E3
:10423000436C22F4C0021A434A6090F82410090625
:1042400006D501684A68806C22F4002202434A6065
:1042500070472DE9F84300260446C0F88460FCF757
:10426000EBFE8046206800684FF0200500076FF0E5
:104270007E4712D54346002229042046009700F0CD
:10428000B5FA50B1216851E8000F20F0800041E8F4
:104290000002002AF6D1E56721E0206800684007A7
:1042A00022D5434600224FF480012046009700F0BB
:1042B0009DFAC8B1216851E8000F20F4907041E8E0
:1042C0000002002AF6D12068083050E8001F21F0D3
:1042D000010140E80012002AF5D1C4F8805084F8AA
:1042E00078600320BDE8F883E567C4F8805044F89F
:1042F000606F666026760020F4E710B5806A0021C2
:10430000A0F85A10A0F85210FEF723FB10BD016868
:1043100051E8002F22F4907241E80023002BF6D1DF
:104320000168083151E8002F22F0010241E8002322
:10433000002BF5D1016E012908D1026852E8001F57
:1043400021F0100142E80013002BF6D12021C0F823
:1043500080100021016681667047000010B5B0F83A
:104360005C20D0F880300168222B04D0088B40F00C
:104370000800088310BD898C436D11401980416D80
:10438000891C4165B0F85A10491EA0F85A10B0F8BF
:104390005A100029EED1016851E8002F22F49072E2
:1043A00041E80023002BF6D10168083151E8002FC5
:1043B00022F0010241E80023002BF5D12021C0F8B2
:1043C0008010002181664166154B02689A420BD02D
:1043D0005268120208D5036853E8002F22F0806269
:1043E00043E80024002CF6D1026E012A02D0FEF729
:1043F00091FC10BD0166026852E8001F21F0100117
:1044000042E80013002BF6D10168CA69D243D206F4
:1044100001D410220A62B0F85810FEF725FA10BD38
:104420000080004010B5B0F85C20D0F88030016802
:10443000222B04D0088B40F00800088310BD898C23
:104440001140426D1170416D491C4165B0F85A1020
:10445000491EA0F85A10B0F85A100029EED102688F
:1044600052E8001F21F4907142E80013002BF6D1AE
:104470000168083151E8002F22F0010241E80023D1
:10448000002BF5D12021C0F8801000218166416603
:10449000154B02689A420BD05268120208D5036885
:1044A00053E8002F22F0806243E80024002CF6D16C
:1044B000026E012A02D0FEF72DFC10BD01660268D3
:1044C00052E8001F21F0100142E80013002BF6D142
:1044D0000168CA69D243D20601D410220A62B0F838
:1044E0005810FEF7C1F910BD008000402DE9F041E1
:1044F0000446016880682269E36910436269002507
:104500001A431043814F0A68814B1A4002430A60E4
:1045100020684168E26821F44051114341602168FC
:10452000A069B94201D0226A10438A6822F430623D
:1045300002438A607749226877488A420DD1D0F8D1
:10454000880010F0030006D0012866D0022854D05D
:10455000032851D163E001204FE070498A420BD11A
:10456000D0F8880010F00C0047D0042845D0082867
:1045700051D00C2840D152E069498A420BD1D0F881
:10458000880010F0300038D0102846D0202842D0C3
:10459000302831D143E063498A420BD1D0F88800FA
:1045A00010F0C00029D0402837D0802833D0C02850
:1045B00022D134E05C498A420ED1D0F8880010F450
:1045C00040701AD0B0F5807F27D0B0F5007F22D0A0
:1045D000B0F5407F10D122E0BA420DD1D0F888006A
:1045E00010F4406009D0B0F5806F16D0B0F5006FC0
:1045F00011D0B0F5406F12D010204C4900264FF476
:104600000043BA422ED160B102280DD004280DD04B
:1046100008286FD10EE00220EFE70420EDE7082024
:10462000EBE7FDF755F803E00B4603E0FDF774F800
:10463000030060D0626802EB420098425AD8B3EBA4
:10464000023F57D8190E1B02500818187141002359
:10465000FBF7B6FD364AA0F5407191424AD8216871
:10466000C86048E0E2694FF6EF779A4227D10928FF
:1046700040D2DFE800F005080D3F213F3F3F0E002C
:10468000FDF726F801E0FDF735F8030001D132E02F
:104690000B466068590001EB5001B1FBF0F0A0F14E
:1046A0001001B94226D84FF6F0710140C0F3420024
:1046B00001432068C1601EE0FDF72EF8E5E70928F8
:1046C00018D2DFE800F005080D171D1717170E00A8
:1046D000FCF7FEFF01E0FDF70DF8030001D10AE051
:1046E0000B46606803EB5001B1FBF0F0A0F1100144
:1046F000B94208D90125A6662846E666BDE8F081DC
:10470000FDF70AF8E9E780B2A9E700000080004061
:10471000F369FFEF00380140001002400044004000
:1047200000480040004C0040005000400024F400CD
:10473000FFFC0F0030B54165A0F85820A0F85A20C2
:104740000022826681684FF48055FF23A94204D17C
:10475000016969BB40F2FF1130E07F2431B3B1F150
:10476000805F28D0A0F85C20C0F884202221C0F807
:1047700080100168083151E8002F42F0010241E841
:104780000023002BF5D18168A94201D10169D9B17B
:10479000144981660169C9B1016851E8002F42F4EA
:1047A000907241E80023002BF6D118E0016941B96D
:1047B000A0F85C30D8E7016919B13F21A0F85C107E
:1047C000D2E7A0F85C40CFE707498166026852E86B
:1047D000001F41F0200142E80013002BF6D1002019
:1047E00030BD0000254400085D4300082DE9F04776
:1047F000994617460D4604464FF00008089E33E0E0
:10480000701C31D0FCF718FCA0EB0900B04218D89E
:10481000BEB120680168490726D5802D24D0402DDF
:1048200022D0C169C94309070DD408250562204675
:10483000FFF76DFDC4F8845084F878800120BDE84E
:10484000F0870320FBE7C069C04300050CD4216852
:104850004FF4006008622046FFF759FD2020C4F89D
:10486000840084F87880ECE72068C06935EA0000AD
:1048700004D00020B842C3D00020E0E70120F9E7CF
:104880000148FEF767B80000E8060020FEE70000D8
:10489000014A024900F023B8014900082000002025
:1048A0000907090E002804DB00F1E02080F800145D
:1048B000704700F00F0000F1E02080F8141D7047F1
:1048C00002E008C8121F08C1002AFAD170477047D9
:1048D000002001E001C1121F002AFBD170472DE921
:1048E000F04116460F460446002503E03946B0471E
:1048F000641C6D1C20780028F8D12846BDE8F081A2
:1049000013B54FF6FF73012269460248FEF703FA1A
:1049100000981CBDE80600201CB5FCF79BFBFFF7C8
:10492000BBF9FEF76BFDFEF721FDFEF7DFFEFEF79C
:10493000D3FDFEF761FEFEF7F7FDFEF7B5FEFEF7CD
:10494000E5FA7F213648FBF75FFD342235493648CA
:10495000FDF763FF3248FCF74BF934491F2008800C
:1049600000213348FDF7ACFE04213248FDF7A8FED4
:10497000314C012280212046FCF758FB0122110214
:104980002046FCF753FB012251022046FCF74EFB68
:104990002AA0FFF77DFF2B48FDF71EFCA2462A4EFA
:1049A000234C00274FF010084FF0B4094FF47A7BE6
:1049B000CDE9008745460423C82132207268FEF7FE
:1049C0003EFC70684FF4FA61484390FBF9F2CDE980
:1049D000005704239621322002F5FA72FEF72FFCCD
:1049E00080215046FCF71AFB5846FCF7C7F930788F
:1049F0000028DDD05FF000052168C5F16400486340
:104A00000A20FCF7BBF96D1C642DF5DD002520683C
:104A100045630A20FCF7B2F96D1C642DF7DDC7E78A
:104A20003C05002008050020E806002000000020CA
:104A3000040600209C0600200010004848656C6CAD
:104A40006F2100005006002004000020000000003C
:104A500000000000000000000000202020202000B6
:104A60000020000028285000000000000000000086
:104A700000005050F85050F850500000002070A82E
:104A8000A0603028A8702000000048A8B0A87434A6
:104A90005448000000002050506CA8A89468000002
:104AA00040408000000000000000000008101020BE
:104AB000202020201010080040202010101010107E
:104AC0002020400000000020A87070A820000000F6
:104AD00000000010107C101000000000000000001A
:104AE00000000000404080000000000000FC0000CA
:104AF0000000000000000000000000000040000076
:104B00000004080810102020404080000000708839
:104B1000888888888870000000002060202020207D
:104B200020700000000070888810204080F800008D
:104B300000007088083008088870000000001030FD
:104B4000305090F8103800000000F88080F088089D
:104B5000887000000000304880B0C888887000006D
:104B6000000078081010202020200000000070882D
:104B700088708888887000000000708888986808AD
:104B800090600000000000002000000000200000F5
:104B9000000000000020000000202000000008109D
:104BA000204040201008000000000000FC00FC0035
:104BB0000000000000004020100808102040000005
:104BC0000000708888102020002000000000384479
:104BD00094B4B4B84438000000002020305050781D
:104BE00048CC00000000F0484870484848F00000F9
:104BF0000000788880808080887000000000F04885
:104C00004848484848F000000000F84850705040BC
:104C100048F800000000F8485070504040E00000A4
:104C20000000384880809C88483000000000CC4854
:104C30004878484848CC00000000F8202020202078
:104C400020F8000000007C1010101010101090E0F0
:104C50000000EC485060504848EC00000000E04084
:104C60004040404044FC00000000DCD8D8D8A8A850
:104C7000A8AC00000000DC486868585848E800000C
:104C80000000708888888888887000000000F048DC
:104C90004870404040E0000000007088888888E844
:104CA000987018000000F0484870504848EC000028
:104CB000000078888060100888F000000000F8A8E4
:104CC00020202020207000000000CC4848484848A0
:104CD000483000000000CC484850503020200000F0
:104CE0000000A8A8A8A87050505000000000D8509C
:104CF0005020205050D800000000D85050502020A4
:104D0000207000000000F8901020204048F80000BB
:104D10003820202020202020202038000040402063
:104D20002020101010080800701010101010101023
:104D30001010700020500000000000000000000073
:104D40000000000000000000000000FC4020000007
:104D500000000000000000000000000000304838A3
:104D6000483C000000C04040407048484870000087
:104D700000000000003848404830000000180808D3
:104D800008384848483C00000000000000304878DF
:104D900040380000001824202078202020780000CF
:104DA00000000000003C48304038443800C040401B
:104DB0004070484848EC000000202000006020209F
:104DC000207000000010100000301010101010E0D3
:104DD00000C040404058506050C8000000E0202013
:104DE0002020202020F800000000000000F0A8A8EB
:104DF000A8A800000000000000F0484848EC0000AF
:104E0000000000000030484848300000000000006A
:104E100000F04848487040E0000000000038484872
:104E20004838081C0000000000D8604040E0000046
:104E300000000000007840300878000000000020EA
:104E400020782020203800000000000000D84848CA
:104E5000483C00000000000000D850502020000016
:104E60000000000000A8A8705050000000000000E2
:104E700000D8502050D800000000000000CC484866
:104E8000301020C0000000000078102020780000C2
:104E900018101010103010101010180010101010F2
:104EA0001010101010101010602020202010202052
:104EB000202060006890000000000000000000005A
:104EC00000000000000000000000000000000000E2
:104ED0000000001010101010101000001010000042
:104EE0000012242448000000000000000000000020
:104EF0000000001212127E2424247E2424240000A8
:104F00000000083C4A4A48380C0A0A4A4A3C080849
:104F100000000044A4A8A8B0541A2A2A4A44000059
:104F200000000030484848506EA4949889760000EC
:104F30000060202040000000000000000000000091
:104F400000020408081010101010100808040200D5
:104F50000040201010080808080808101020400021
:104F6000000000001010D63838D6101000000000E5
:104F700000000000000808087F0808080000000082
:104F80000000000000000000000000006020204041
:104F900000000000000000007E0000000000000093
:104FA0000000000000000000000000006060000041
:104FB00000000204040408081010102020404000E3
:104FC000000000182442424242424242241800009B
:104FD000000000083808080808080808083E000013
:104FE0000000003C4242420204081020427E0000C1
:104FF0000000003C4242020418040242423C00000D
:10500000000000040C0C142424447F04041F00003E
:105010000000007E404040784402024244380000D4
:10502000000000182440405C62424242221C000002
:105030000000007E42040408081010101010000048
:105040000000003C4242422418244242423C0000FC
:105050000000003844424242463A0202241800004E
:1050600000000000000018180000000018180000E0
:1050700000000000000000100000000000101010F0
:105080000000000204081020402010080402000064
:105090000000000000007E00007E00000000000014
:1050A0000000004020100804020408102040000006
:1050B0000000003C42426204080808001818000082
:1050C00000000038445AAAAAAAAAAA5C423C0000DE
:1050D0000000001010182828243C444242E7000039
:1050E000000000F8444444784442424244F800003E
:1050F0000000003E424280808080804244380000B0
:10510000000000F8444242424242424244F8000059
:10511000000000FC424848784848404242FC0000F9
:10512000000000FC424848784848404040E0000009
:105130000000003C44448080808E84444438000059
:10514000000000E7424242427E42424242E7000003
:105150000000007C1010101010101010107C0000C7
:105160000000003E0808080808080808080888F039
:10517000000000EE444850705048484444EE00009F
:10518000000000E0404040404040404042FE0000FF
:10519000000000EE6C6C6C6C6C54545454D60000DF
:1051A000000000C7626252524A4A4A4646E2000084
:1051B0000000003844828282828282824438000069
:1051C000000000FC424242427C40404040E000007F
:1051D0000000003844828282828282B24C3806000B
:1051E000000000FC4242427C4848444442E3000044
:1051F0000000003E4242402018040242427C00006F
:10520000000000FE92101010101010101038000056
:10521000000000E74242424242424242423C000019
:10522000000000E7424244242428281810100000FF
:10523000000000D654545454546C282828280000E8
:10524000000000E7422424181818242442E7000034
:10525000000000EE44442828101010101038000000
:105260000000007E840408081020204242FC000058
:10527000001E1010101010101010101010101E0032
:10528000000040202020101010080804040402022E
:1052900000780808080808080808080808087800BE
:1052A00000182400000000000000000000000000C2
:1052B000000000000000000000000000000000FFEF
:1052C000006010000000000000000000000000006E
:1052D0000000000000000038440C34444C3600004C
:1052E00000000000C0404058644242426458000040
:1052F000000000000000001C22404040221C000072
:10530000000000000602023E42424242463B0000CC
:10531000000000000000003C42427E40423C000091
:10532000000000000C12107C10101010107C000007
:10533000000000000000003E444438403C42423C33
:1053400000000000C040405C6242424242E7000070
:10535000000000303000007010101010107C0000B1
:105360000000000C0C00001C040404040404447835
:1053700000000000C040404E4850704844EE00001D
:10538000000000107010101010101010107C0000A1
:1053900000000000000000FE4949494949ED0000B5
:1053A00000000000000000DC6242424242E70000D0
:1053B000000000000000003C42424242423C00002B
:1053C00000000000000000D864424242645840E0FF
:1053D000000000000000001A26424242261A02077E
:1053E00000000000000000EE3220202020F8000025
:1053F000000000000000003E42403C02427C0000F1
:10540000000000000010107C10101010120C0000A2
:1054100000000000000000C642424242463B00003D
:1054200000000000000000EE444428281010000096
:1054300000000000000000DB894A5A5424240000C8
:10544000000000000000007624181818246E0000E8
:1054500000000000000000E742242418181010602B
:10546000000000000000007E44081010227E0000B2
:1054700000030404040404040804040404040300F2
:10548000080808080808080808080808080808089C
:1054900000C0202020202020102020202020C0001C
:1054A000205A04000000000000000000000000007E
:1054B00000000000000000000000000000000000EC
:1054C00000000000000000000000000000000000DC
:1054D00000000000000000000000000000000000CC
:1054E00000000000000000000600060006000600A4
:1054F000060006000600020004000400040000008C
:105500000000000006000600060000000000000089
:1055100000000000066006600CC019801100220027
:10552000000000000000000000000000000000007B
:10553000000000000000000000000000000000006B
:10554000000000000000000008400840084008403B
:105550007FE07FE0104010801080108010807FE09E
:105560007FE020802080208020800000000000005C
:10557000000000000000020002000F801AC032C0CC
:1055800033C032001A000E0007000380038002C0FF
:1055900032C03AC032C012800F0002000200000088
:1055A0000000000000000000708050808900890029
:1055B00089008A008A005C0075C005400A200A2024
:1055C000122012201220214021C000000000000003
:1055D00000000000000000001C003600360036000D
:1055E00036003600340019E038805880CC80CC80FA
:1055F000C680C700C31063903CE0000000000000BC
:1056000000000000300038000800080010002000F2
:10561000000000000000000000000000000000008A
:10562000000000000000000000000000000000007A
:105630000000000000200040008001000100020086
:10564000020004000400040004000400040004003C
:105650000200020001000100008000400020000064
:1056600000000000400020001000080008000400B6
:105670000400020002000200020002000200020018
:105680000400040008000800100020004000000092
:105690000000000000000000000000000200030005
:1056A0000200623072F00B800F807AF062300200EC
:1056B00002000200000000000000000000000000E6
:1056C00000000000000000000000000000000200D8
:1056D00002000200020002007FF00200020002004D
:1056E00002000200000000000000000000000000B6
:1056F00000000000000000000000000000000000AA
:105700000000000000000000000000000000000099
:1057100000000000300038000800080010002000E1
:105720000000000000000000000000000000000079
:1057300000000000000000007FE00000000000000A
:105740000000000000000000000000000000000059
:105750000000000000000000000000000000000049
:105760000000000000000000000000000000000039
:105770000000000038003800380000000000000081
:105780000000000000200060004000C00080008099
:1057900001000100020002000600040004000800ED
:1057A00008001000100030002000600040000000E1
:1057B000000000000000000000000F00198030C051
:1057C00030C06060606060606060606060606060A9
:1057D000606030C030C019800F0000000000000081
:1057E0000000000000000000000002003E00060073
:1057F0000600060006000600060006000600060079
:1058000006000600060006003FC000000000000081
:10581000000000000000000000001F00218040C0C8
:1058200060C060C000C0008001800300060004006A
:1058300008001040204060407FC0000000000000D1
:10584000000000000000000000001E0063006180F6
:1058500061800180018003000E000180008000C093
:1058600000C060C060C061801F0000000000000038
:1058700000000000000000000000018001800380A3
:1058800005800580098011801180218041807FF092
:10589000018001800180018007E00000000000001D
:1058A000000000000000000000003FC020002000B9
:1058B0002000200020002F00318020C000C000C048
:1058C00060C060C0418021801F0000000000000017
:1058D00000000000000000000000078018C030C079
:1058E000300020006000678068C0706060606060A9
:1058F00060602060304018C00F0000000000000011
:10590000000000000000000000001FE030602040A8
:1059100020800080008001000100020002000200DF
:105920000600060006000600060000000000000059
:10593000000000000000000000001F8030C0606018
:1059400060606060304038C00F00138030C060601D
:1059500060606060606030C00F8000000000000088
:10596000000000000000000000000F00308030C088
:10597000604060606060606060E031601E60006098
:1059800000C000C0308031801E0000000000000018
:105990000000000000000000000000000000000007
:1059A00000000000070007000700000000000000E2
:1059B00000000000070007000700000000000000D2
:1059C00000000000000000000000000000000000D7
:1059D00000000000060006000000000000000000BB
:1059E00000000000000006000600020004000400A1
:1059F00000000000000000000020004000800100C6
:105A0000020004000800100020001000080004003C
:105A100002000100008000400020000000000000A3
:105A20000000000000000000000000000000000076
:105A3000000000007FE00000000000007FE00000A8
:105A40000000000000000000000000000000000056
:105A5000000000000000000020001000080004000A
:105A60000200010000800040002000400080010092
:105A700002000400080010002000000000000000E8
:105A80000000000000000000000007C01860203087
:105A900020303030303000E001800200020002008F
:105AA00000000000070007000700000000000000E1
:105AB0000000000000000000070018C0304033A0C4
:105AC00026A066A065A06D206D206D206D206D4024
:105AD00027803020304018C00F0000000000000078
:105AE00000000000000000000000060006000A00A0
:105AF0000B00090009001100118010801F8020C0D8
:105B000020C0204040404060F0F000000000000055
:105B1000000000000000000000007F0031C030C025
:105B200030C030C030C031803F0030C030403060C5
:105B300030603060306030C07F80000000000000C6
:105B40000000000000000000000007C018C0306026
:105B50003020202060006000600060006000600075
:105B600060203020304018C00F000000000000000E
:105B700000000000000000000000FE00318030C086
:105B800030C0306030603060306030603060306035
:105B9000306030C030C03180FE00000000000000E6
:105BA00000000000000000000000FFC060C0602096
:105BB00060206000610061007F00610061006100A1
:105BC0006000602060206040FFC000000000000016
:105BD00000000000000000000000FFC060C0602066
:105BE00060206000610061007F0061006100610071
:105BF0006000600060006000F8000000000000002D
:105C0000000000000000000000000F00188030407D
:105C100030402040600060006000600063F060C0C1
:105C200060C030C030C018C00F000000000000008D
:105C300000000000000000000000F0F06060606004
:105C400060606060606060607FE0606060606060B5
:105C50006060606060606060F0F000000000000064
:105C6000000000000000000000003FC00600060029
:105C700006000600060006000600060006000600F4
:105C800006000600060006003FC0000000000000FD
:105C9000000000000000000000001FE003000300FF
:105CA00003000300030003000300030003000300DC
:105CB00003000300030003000300630066003C00D0
:105CC00000000000000000000000F3C061806300DD
:105CD0006200640068006C0074007600620063007B
:105CE00061006180608060C0F1E0000000000000A1
:105CF00000000000000000000000F80060006000EC
:105D00006000600060006000600060006000600093
:105D10006000602060206040FFC0000000000000C4
:105D200000000000000000000000E0E061C061C071
:105D300071C071C072C072C052C05AC05AC05CC03B
:105D40004CC04CC04CC048C0E1E000000000000066
:105D50000000000000000000000071F030403840FA
:105D600038402C402C4026402640224023402140F1
:105D700021C021C020C020C0F84000000000000069
:105D8000000000000000000000000F00198030C07B
:105D90003040606060606060606060606060606053
:105DA0006060304030C019800F000000000000002B
:105DB00000000000000000000000FF0060C0606004
:105DC000606060606060606061C07F006000600073
:105DD0006000600060006000F8000000000000004B
:105DE000000000000000000000000F00198030C01B
:105DF00030406060606060606060606060606060F3
:105E00006E60324033C019800F0001E000C0000016
:105E100000000000000000000000FF8060C0606023
:105E200060606060606060C07F006200630061006D
:105E3000618060C060C06060F07000000000000021
:105E4000000000000000000000001F4030C0604063
:105E50006040600070003C001F0007C001C000E00F
:105E600040604060606030C00F80000000000000B3
:105E7000000000000000000000007FE046208610C7
:105E80008610060006000600060006000600060052
:105E900006000600060006001F800000000000004B
:105EA0000000000000000000000078E030403040BA
:105EB0003040304030403040304030403040304062
:105EC00030403040304018800F00000000000000DB
:105ED00000000000000000000000F0E060402080B2
:105EE00020803080308011001100190019000A0054
:105EF0000A000E000C000400040000000000000076
:105F000000000000000000000000EF70462042206A
:105F100062206220264026402740274039403980B1
:105F2000198019801180110011000000000000008C
:105F30000000000000000000000079E030801080C8
:105F4000188009000D0006000400060006000B0082
:105F500009001180108020C071E0000000000000E6
:105F600000000000000000000000F0F06020204071
:105F70003040108018801D000D000E000600060045
:105F800006000600060006001F800000000000005A
:105F9000000000000000000000003FE0304060C052
:105FA000408001800100020002000400040008009B
:105FB00018001020302020407FC0000000000000AA
:105FC0000000000007C004000400040004000400F6
:105FD00004000400040004000400040004000400A1
:105FE00004000400040004000400040007C00000D2
:105FF0000000000000000000200020001000100041
:106000000800080008000400040002000200030069
:10601000010001000080008000400040004000209E
:10602000000000003E000200020002000200020028
:106030000200020002000200020002000200020050
:106040000200020002000200020002003E00000006
:1060500000000600090010800000000000000000A1
:106060000000000000000000000000000000000030
:106070000000000000000000000000000000000020
:106080000000000000000000000000000000000010
:106090000000000000000000000000000000000000
:1060A0000000000000000000000000000000FFF001
:1060B00000000000180006000000000000000000C2
:1060C00000000000000000000000000000000000D0
:1060D00000000000000000000000000000000000C0
:1060E00000000000000000000000000000000000B0
:1060F000000000000F8030C030C000C007C038C0B2
:1061000070C060C060C071D03E7000000000000030
:10611000000000000000000010007000300030009F
:106120003000300033803CC0386030603060306018
:1061300030603060304038C0278000000000000030
:10614000000000000000000000000000000000004F
:10615000000000000F00318031806180600060002D
:1061600060006040304030800F0000000000000000
:106170000000000000000000004003C000C000C09C
:1061800000C000C01EC031C030C060C060C060C070
:1061900060C060C020C031E01E8000000000000030
:1061A00000000000000000000000000000000000EF
:1061B00000000000078018C01040306030603FE0F1
:1061C0003000300018201840078000000000000058
:1061D0000000000000000000000003C006600C602A
:1061E0000C000C007F800C000C000C000C000C005C
:1061F0000C000C000C000C003F80000000000000B0
:10620000000000000000000000000000000000008E
:10621000000000000FE01B60318031803180198068
:106220001F0030003F0033C060C060C071C01F005D
:10623000000000000000000010007000300030007E
:1062400030003000378038C030C030C030C030C07F
:1062500030C030C030C030C079E000000000000025
:106260000000000000000000000006000600000022
:10627000000002003E0006000600060006000600C0
:1062800006000600060006003FC0000000000000F7
:1062900000000000000000000000038003800000F8
:1062A000000000800F80018001800180018001805A
:1062B00001800180018001800180018033003E0067
:1062C00000000000000000001000700030003000EE
:1062D0003000300031C031003100320036003A0069
:1062E00031003180308030C079E0000000000000D3
:1062F000000000000000000002003E000600060052
:10630000060006000600060006000600060006005D
:1063100006000600060006003FC000000000000066
:10632000000000000000000000000000000000006D
:1063300000000000ECE077606660666066606660A2
:106340006660666066606660FFF000000000000046
:10635000000000000000000000000000000000003D
:1063600000000000778038C030C030C030C030C07E
:1063700030C030C030C030C079E000000000000004
:10638000000000000000000000000000000000000D
:10639000000000000F00198030C060606060606025
:1063A0006060606030C030C00F000000000000007E
:1063B00000000000000000000000000000000000DD
:1063C00000000000778038C030603060306030609E
:1063D0003060306030C038C03780300030007C0022
:1063E00000000000000000000000000000000000AD
:1063F000000000001E4031C030C060C060C060C0FE
:1064000060C060C020C031C01EC000C000C003E03A
:10641000000000000000000000000000000000007C
:1064200000000000F9C01A601C6018001800180075
:106430001800180018001800FF00000000000000FD
:10644000000000000000000000000000000000004C
:10645000000000000FC038C0304030401C000F006A
:1064600003C020C020C031C03F80000000000000F9
:106470000000000000000000000000000400040014
:106480000C000C007F800C000C000C000C000C00B9
:106490000C000C000C400C400780000000000000C5
:1064A00000000000000000000000000000000000EC
:1064B0000000104071C030C030C030C030C030C0AB
:1064C00030C030C030C039E01E8000000000000045
:1064D00000000000000000000000000000000000BC
:1064E0000000000078E03040108010801880090023
:1064F0000D000D0006000600040000000000000072
:10650000000000000000000000000000000000008B
:1065100000000000EF7046206220264026403740F1
:1065200039801980198019801000000000000000D7
:10653000000000000000000000000000000000005B
:10654000000000003DE0188008800D0006000600F5
:1065500007000900108010C079E000000000000072
:10656000000000000000000000000000000000002B
:106570000000000079E01080108010800900090000
:106580000D00060006000600040004002400380088
:1065900000000000000000000000000000000000FB
:1065A000000000003F80218023002200060004003C
:1065B0000C001840104030C03F8000000000000078
:1065C0000000000000C00100010001000100010006
:1065D00001000100010002000400020001000100AE
:1065E00001000100010001000100010000C00000E5
:1065F000020002000200020002000200020002008B
:10660000020002000200020002000200020002007A
:10661000020002000200020002000200020002006A
:106620000000000030000800080008000800080012
:106630000800080008000400020004000800080028
:1066400008000800080008000800080030000000EA
:10665000000038004420432001C00000000000007A
:10666000000000000000000000000000000000002A
:10667000000000000000000000000000000000001A
:10668000000000000000000000000000000000000A
:1066900000000000000000000000000000000000FA
:1066A00000000000000000000000000000000000EA
:1066B00000000000000000000000000000000000DA
:1066C00000000000000000000000000000000000CA
:1066D00000000000000000000000000000000000BA
:1066E00000000000000000000000000000000000AA
:1066F000000000000000000000000000000000009A
:1067000000000000000000000000000003C003C003
:1067100003C003C003C003C001C001800180018029
:1067200001800180018001800180000000000000E4
:10673000018003C003C001800000000000000000D1
:106740000000000000000000000000000000000049
:106750000000000000000000000000000000000039
:106760000000000000000000000000000000000029
:106770000000000000000000000000000000000019
:10678000000000000318073807380E700C6018C0AE
:106790003180210000000000000000000000000027
:1067A00000000000000000000000000000000000E9
:1067B00000000000000000000000000000000000D9
:1067C00000000000000000000000000000000000C9
:1067D00000000000000000000000000000000000B9
:1067E00000000000000000000000000000000000A9
:1067F0000000000000000000000000000000000099
:106800000000000000000000000000000408040870
:106810000408040804087FFE7FFE7FFE08100810AD
:1068200008100810081008107FFE7FFE7FFE183049
:106830001020102010201020000000000000000098
:106840000000000000000000000000000000000048
:106850000000000000000000000000000000000038
:106860000000000000000000000000000000000028
:106870000000000000000000000000000000000018
:1068800000000000000000000100010003C00D3006
:1068900009181918193819381D000D000F000700C4
:1068A00003C001E001F0013001380118391839182E
:1068B00031183130196007C00100010001000000EB
:1068C00000000000000000000000000000000000C8
:1068D00000000000000000000000000000000000B8
:1068E00000000000000000000000000000000000A8
:1068F0000000000000000000000000000000000098
:1069000000000000000000000000000038106C10C3
:106910004420C620C640C640C640C680C6804480CB
:106920006D38396C024402C602C604C604C608C6E5
:1069300008C60844106C1038000000000000000079
:106940000000000000000000000000000000000047
:106950000000000000000000000000000000000037
:106960000000000000000000000000000000000027
:106970000000000000000000000000000000000017
:106980000000000000000000000000000F001900DF
:106990003180318031803180310033003A001C0079
:1069A000387C3C104C10CE10C620C720C320C1C07C
:1069B000C1C260E6317C1E3800000000000000000B
:1069C00000000000000000000000000000000000C7
:1069D00000000000000000000000000000000000B7
:1069E00000000000000000000000000000000000A7
:1069F0000000000000000000000000000000000097
:106A00000000000038003C003C000C000C000800B6
:106A100030006000000000000000000000000000E6
:106A20000000000000000000000000000000000066
:106A30000000000000000000000000000000000056
:106A40000000000000000000000000000000000046
:106A50000000000000000000000000000000000036
:106A60000000000000000000000000000000000026
:106A70000000000000000000000000000000000016
:106A80000000000000020004000800180030002090
:106A90000060004000C000C00180018001800180D2
:106AA0000180018001800180018000C000C00040A1
:106AB0000060002000300018000800040002000000
:106AC00000000000000000000000000000000000C6
:106AD00000000000000000000000000000000000B6
:106AE00000000000000000000000000000000000A6
:106AF0000000000000000000000000000000000096
:106B00000000000040002000100018000C000400ED
:106B10000600020003000300018001800180018063
:106B200001800180018001800180030003000300D7
:106B3000060004000C0018001000200040000000B7
:106B40000000000000000000000000000000000045
:106B50000000000000000000000000000000000035
:106B60000000000000000000000000000000000025
:106B70000000000000000000000000000000000015
:106B80000000000000000000000000000000000005
:106B900000C001C001C030C6388E1C9C06B001C0C8
:106BA00001C006B01C9C388E318601C001C001C0F6
:106BB00000000000000000000000000000000000D5
:106BC00000000000000000000000000000000000C5
:106BD00000000000000000000000000000000000B5
:106BE00000000000000000000000000000000000A5
:106BF0000000000000000000000000000000000095
:106C00000000000000000000000000000000000084
:106C100000000080008000800080008000800080F4
:106C20003FFE0080008000800080008000800080A7
:106C30000000000000000000000000000000000054
:106C40000000000000000000000000000000000044
:106C50000000000000000000000000000000000034
:106C60000000000000000000000000000000000024
:106C70000000000000000000000000000000000014
:106C80000000000000000000000000000000000004
:106C900000000000000000000000000000000000F4
:106CA00000000000000000000000000000000000E4
:106CB00038003C003C000C000C0008003000600074
:106CC00000000000000000000000000000000000C4
:106CD00000000000000000000000000000000000B4
:106CE00000000000000000000000000000000000A4
:106CF0000000000000000000000000000000000094
:106D00000000000000000000000000000000000083
:106D10000000000000000000000000000000000073
:106D20007FFE0000000000000000000000000000E6
:106D30000000000000000000000000000000000053
:106D40000000000000000000000000000000000043
:106D50000000000000000000000000000000000033
:106D60000000000000000000000000000000000023
:106D70000000000000000000000000000000000013
:106D80000000000000000000000000000000000003
:106D900000000000000000000000000000000000F3
:106DA00000000000000000000000000000000000E3
:106DB00018003C003C00180000000000000000002B
:106DC00000000000000000000000000000000000C3
:106DD00000000000000000000000000000000000B3
:106DE00000000000000000000000000000000000A3
:106DF0000000000000000000000000000000000093
:106E0000000000000000000200060004000C000862
:106E100000180010003000200060004000C000801A
:106E20000180010003000200060004000C000800BD
:106E3000180010003000200060004000000000003A
:106E40000000000000000000000000000000000042
:106E50000000000000000000000000000000000032
:106E60000000000000000000000000000000000022
:106E70000000000000000000000000000000000012
:106E800000000000000000000000000003C0062019
:106E90000C30181818181808300C300C300C300C46
:106EA000300C300C300C300C300C300C180818182A
:106EB00018180C30062003C000000000000000007D
:106EC00000000000000000000000000000000000C2
:106ED00000000000000000000000000000000000B2
:106EE00000000000000000000000000000000000A2
:106EF0000000000000000000000000000000000092
:106F00000000000000000000000000000080018080
:106F10001F8001800180018001800180018001804B
:106F20000180018001800180018001800180018059
:106F30000180018003C01FF8000000000000000075
:106F40000000000000000000000000000000000041
:106F50000000000000000000000000000000000031
:106F60000000000000000000000000000000000021
:106F70000000000000000000000000000000000011
:106F800000000000000000000000000007E00838DA
:106F90001018200C200C300C300C000C00180018BD
:106FA0000030006000C001800300020004040804F7
:106FB0001004200C3FF83FF8000000000000000023
:106FC00000000000000000000000000000000000C1
:106FD00000000000000000000000000000000000B1
:106FE00000000000000000000000000000000000A1
:106FF0000000000000000000000000000000000091
:1070000000000000000000000000000007C0186041
:107010003030301830183018001800180030006078
:1070200003C0007000180008000C000C300C300C7D
:1070300030083018183007C00000000000000000C1
:107040000000000000000000000000000000000040
:107050000000000000000000000000000000000030
:107060000000000000000000000000000000000020
:107070000000000000000000000000000000000010
:107080000000000000000000000000000060006040
:1070900000E000E0016001600260046004600860DC
:1070A000086010603060206040607FFC006000601D
:1070B00000600060006003FC0000000000000000B1
:1070C00000000000000000000000000000000000C0
:1070D00000000000000000000000000000000000B0
:1070E00000000000000000000000000000000000A0
:1070F0000000000000000000000000000000000090
:107100000000000000000000000000000FFC0FFC69
:1071100010001000100010001000100013E01430D8
:1071200018181008000C000C000C000C300C300C6F
:1071300020182018183007C00000000000000000D0
:10714000000000000000000000000000000000003F
:10715000000000000000000000000000000000002F
:10716000000000000000000000000000000000001F
:10717000000000000000000000000000000000000F
:1071800000000000000000000000000001E0061800
:107190000C180818180010001000300033E03630CA
:1071A00038183808300C300C300C300C300C180CFF
:1071B00018080C180E3003E000000000000000006A
:1071C00000000000000000000000000000000000BF
:1071D00000000000000000000000000000000000AF
:1071E000000000000000000000000000000000009F
:1071F000000000000000000000000000000000008F
:107200000000000000000000000000001FFC1FFC48
:1072100010083010201020200020004000400040C6
:107220000080008001000100010001000300030054
:107230000300030003000300000000000000000042
:10724000000000000000000000000000000000003E
:10725000000000000000000000000000000000002E
:10726000000000000000000000000000000000001E
:10727000000000000000000000000000000000000E
:1072800000000000000000000000000007E00C30DB
:107290001818300C300C300C380C38081E180F2021
:1072A00007C018F030783038601C600C600C600C3F
:1072B000600C3018183007C000000000000000000B
:1072C00000000000000000000000000000000000BE
:1072D00000000000000000000000000000000000AE
:1072E000000000000000000000000000000000009E
:1072F000000000000000000000000000000000008E
:1073000000000000000000000000000007C018207E
:10731000301030186008600C600C600C600C600C61
:10732000701C302C186C0F8C000C0018001800100A
:107330003030306030C00F800000000000000000DE
:10734000000000000000000000000000000000003D
:10735000000000000000000000000000000000002D
:10736000000000000000000000000000000000001D
:10737000000000000000000000000000000000000D
:1073800000000000000000000000000000000000FD
:1073900000000000000000000000018003C003C0E6
:1073A000018000000000000000000000000000005C
:1073B000018003C003C00180000000000000000045
:1073C00000000000000000000000000000000000BD
:1073D00000000000000000000000000000000000AD
:1073E000000000000000000000000000000000009D
:1073F000000000000000000000000000000000008D
:10740000000000000000000000000000000000007C
:107410000000000000000000000000000380038066
:1074200003800000000000000000000000000000D9
:10743000000003800380038001800300030000003C
:10744000000000000000000000000000000000003C
:10745000000000000000000000000000000000002C
:10746000000000000000000000000000000000001C
:10747000000000000000000000000000000000000C
:1074800000000000000000000000000000040008F0
:1074900000100020004000800100020004000800ED
:1074A00010001000080004000200010000800040ED
:1074B0000020001000080004000000000000000090
:1074C00000000000000000000000000000000000BC
:1074D00000000000000000000000000000000000AC
:1074E000000000000000000000000000000000009C
:1074F000000000000000000000000000000000008C
:10750000000000000000000000000000000000007B
:10751000000000000000000000007FFE00000000EE
:107520000000000000007FFE0000000000000000DE
:10753000000000000000000000000000000000004B
:10754000000000000000000000000000000000003B
:10755000000000000000000000000000000000002B
:10756000000000000000000000000000000000001B
:10757000000000000000000000000000000000000B
:1075800000000000000000000000000020001000CB
:1075900008000400020001000080004000200010EC
:1075A00000080008001000200040008001000200D8
:1075B000040008001000200000000000000000008F
:1075C00000000000000000000000000000000000BB
:1075D00000000000000000000000000000000000AB
:1075E000000000000000000000000000000000009B
:1075F000000000000000000000000000000000008B
:1076000000000000000000000000000003E00C1873
:10761000180C10063006380638063806000C00181C
:10762000007000C00080008000800080000000002A
:10763000018003C003C001800000000000000000C2
:10764000000000000000000000000000000000003A
:10765000000000000000000000000000000000002A
:10766000000000000000000000000000000000001A
:10767000000000000000000000000000000000000A
:1076800000000000000000000000000003E0061001
:107690000C08180430D431B22132633263226622DE
:1076A0006622662266626664666426E833303002CB
:1076B0001004180C0C1803E000000000000000008B
:1076C00000000000000000000000000000000000BA
:1076D00000000000000000000000000000000000AA
:1076E000000000000000000000000000000000009A
:1076F000000000000000000000000000000000008A
:107700000000000000000000000000000380038073
:107710000380038004C004C004C004C00C4008609F
:107720000860086008201FF010301030103020185A
:1077300020182018601CF83E000000000000000027
:107740000000000000000000000000000000000039
:107750000000000000000000000000000000000029
:107760000000000000000000000000000000000019
:107770000000000000000000000000000000000009
:107780000000000000000000000000007FE018384A
:107790001818180C180C180C180C180C181818308D
:1077A0001FE01818180C18041806180618061806F2
:1077B0001806180C18187FF00000000000000000E8
:1077C00000000000000000000000000000000000B9
:1077D00000000000000000000000000000000000A9
:1077E0000000000000000000000000000000000099
:1077F0000000000000000000000000000000000089
:1078000000000000000000000000000003E0061C73
:10781000080C180630023002300060006000600082
:1078200060006000600060006000600030023002B4
:10783000100418080C1003E0000000000000000015
:107840000000000000000000000000000000000038
:107850000000000000000000000000000000000028
:107860000000000000000000000000000000000018
:107870000000000000000000000000000000000008
:107880000000000000000000000000007FC0187031
:1078900018181808180C180C1806180618061806D8
:1078A000180618061806180618061804180C180CDE
:1078B0001818181818607FC00000000000000000B1
:1078C00000000000000000000000000000000000B8
:1078D00000000000000000000000000000000000A8
:1078E0000000000000000000000000000000000098
:1078F0000000000000000000000000000000000088
:107900000000000000000000000000007FFC180CD8
:10791000180418021802180018001810181018304F
:107920001FF018301810181018001800180018024E
:1079300018021804180C7FFC000000000000000072
:107940000000000000000000000000000000000037
:107950000000000000000000000000000000000027
:107960000000000000000000000000000000000017
:107970000000000000000000000000000000000007
:107980000000000000000000000000007FFC181C48
:1079900018041802180218001800181018101830CF
:1079A0001FF01830181018101810180018001800C0
:1079B0001800180018007E00000000000000000001
:1079C00000000000000000000000000000000000B7
:1079D00000000000000000000000000000000000A7
:1079E0000000000000000000000000000000000097
:1079F0000000000000000000000000000000000087
:107A000000000000000000000000000003C00C3077
:107A1000081018183008300820006000600060006E
:107A200060006000607E6018601820183018301800
:107A3000101818180C2007C00000000000000000FB
:107A40000000000000000000000000000000000036
:107A50000000000000000000000000000000000026
:107A60000000000000000000000000000000000016
:107A70000000000000000000000000000000000006
:107A8000000000000000000000000000FC3F300C7F
:107A9000300C300C300C300C300C300C300C300C06
:107AA0003FFC300C300C300C300C300C300C300CF7
:107AB000300C300C300CFC3F0000000000000000D7
:107AC00000000000000000000000000000000000B6
:107AD00000000000000000000000000000000000A6
:107AE0000000000000000000000000000000000096
:107AF0000000000000000000000000000000000086
:107B00000000000000000000000000001FF80180DD
:107B1000018001800180018001800180018001805D
:107B2000018001800180018001800180018001804D
:107B30000180018001801FF80000000000000000AB
:107B40000000000000000000000000000000000035
:107B50000000000000000000000000000000000025
:107B60000000000000000000000000000000000015
:107B70000000000000000000000000000000000005
:107B800000000000000000000000000007FE006090
:107B900000600060006000600060006000600060E5
:107BA00000600060006000600060006000600060D5
:107BB0000060006000600060706070C071803F0015
:107BC00000000000000000000000000000000000B5
:107BD00000000000000000000000000000000000A5
:107BE0000000000000000000000000000000000095
:107BF0000000000000000000000000000000000085
:107C00000000000000000000000000007E7C183032
:107C100018201860184018801880190019001B00DF
:107C20001D801D8018C018C01860186018301830EA
:107C30001830181818187E3E0000000000000000E0
:107C40000000000000000000000000000000000034
:107C50000000000000000000000000000000000024
:107C60000000000000000000000000000000000014
:107C70000000000000000000000000000000000004
:107C80000000000000000000000000007E0018005E
:107C90001800180018001800180018001800180024
:107CA0001800180018001800180018001800180212
:107CB00018021804180C7FFC0000000000000000EF
:107CC00000000000000000000000000000000000B4
:107CD00000000000000000000000000000000000A4
:107CE0000000000000000000000000000000000094
:107CF0000000000000000000000000000000000084
:107D0000000000000000000000000000F00F381C20
:107D1000381C381C381C382C2C2C2C2C2C2C2C4C83
:107D20002C4C264C264C264C268C228C238C238CC7
:107D3000230C230C210CF13F000000000000000088
:107D40000000000000000000000000000000000033
:107D50000000000000000000000000000000000023
:107D60000000000000000000000000000000000013
:107D70000000000000000000000000000000000003
:107D8000000000000000000000000000F01F3804A8
:107D900038042C042C042604260423042304218400
:107DA000218420C420C42064206420342034201C7A
:107DB000201C200C200CF804000000000000000033
:107DC00000000000000000000000000000000000B3
:107DD00000000000000000000000000000000000A3
:107DE0000000000000000000000000000000000093
:107DF0000000000000000000000000000000000083
:107E000000000000000000000000000003C00C3073
:107E100018181008300C300C60046006600660060C
:107E2000600660066006600660062006300C300CB6
:107E3000100818180C3003C00000000000000000FB
:107E40000000000000000000000000000000000032
:107E50000000000000000000000000000000000022
:107E60000000000000000000000000000000000012
:107E70000000000000000000000000000000000002
:107E80000000000000000000000000007FF0181853
:107E9000180C180618061806180618061806180CE6
:107EA00018181FE018001800180018001800180013
:107EB0001800180018007E000000000000000000FC
:107EC00000000000000000000000000000000000B2
:107ED00000000000000000000000000000000000A2
:107EE0000000000000000000000000000000000092
:107EF0000000000000000000000000000000000082
:107F000000000000000000000000000003C00C3072
:107F100018181008300C300C600660066006600609
:107F2000600660066006600660066006278438CC3E
:107F3000386C18780C7003E00032003C001C000024
:107F40000000000000000000000000000000000031
:107F50000000000000000000000000000000000021
:107F60000000000000000000000000000000000011
:107F70000000000000000000000000000000000001
:107F80000000000000000000000000007FE0183842
:107F90001818180C180C180C180C180C1818183085
:107FA0001FE018C018C0186018601860183018302A
:107FB0001830181818187E1E00000000000000007D
:107FC00000000000000000000000000000000000B1
:107FD00000000000000000000000000000000000A1
:107FE0000000000000000000000000000000000091
:107FF0000000000000000000000000000000000081
:108000000000000000000000000000000FC8187809
:108010003018601860086008600070003C001F00A5
:1080200007C001F000780018001C400C400C600CE8
:10803000200C3018383027E000000000000000005D
:108040000000000000000000000000000000000030
:108050000000000000000000000000000000000020
:108060000000000000000000000000000000000010
:108070000000000000000000000000000000000000
:108080000000000000000000000000003FFC318400
:10809000218641824182018001800180018001802E
:1080A00001800180018001800180018001800180C8
:1080B00001800180018007E0000000000000000056
:1080C00000000000000000000000000000000000B0
:1080D00000000000000000000000000000000000A0
:1080E0000000000000000000000000000000000090
:1080F0000000000000000000000000000000000080
:10810000000000000000000000000000FC3E3008FD
:10811000300830083008300830083008300830089F
:10812000300830083008300830083008300830088F
:10813000300818101C2007C00000000000000000DC
:10814000000000000000000000000000000000002F
:10815000000000000000000000000000000000001F
:10816000000000000000000000000000000000000F
:1081700000000000000000000000000000000000FF
:108180000000000000000000000000007C1E180C31
:108190001808180818080C100C100C100C100C20E3
:1081A00006200620062006400340034003400380CB
:1081B00001800180010001000000000000000000BB
:1081C00000000000000000000000000000000000AF
:1081D000000000000000000000000000000000009F
:1081E000000000000000000000000000000000008F
:1081F000000000000000000000000000000000007F
:10820000000000000000000000000000F3CF6186C5
:1082100061842184208430C431C431C431C831C860
:1082200011C812481A681A681A701C700C700C7009
:108230000C300C2008200820000000000000000086
:10824000000000000000000000000000000000002E
:10825000000000000000000000000000000000001E
:10826000000000000000000000000000000000000E
:1082700000000000000000000000000000000000FE
:108280000000000000000000000000007C3E180814
:1082900018100C100C2006200640034003800180BB
:1082A0000180018001C002C00260046004700830D7
:1082B00008301818101C7C3E000000000000000070
:1082C00000000000000000000000000000000000AE
:1082D000000000000000000000000000000000009E
:1082E000000000000000000000000000000000008E
:1082F000000000000000000000000000000000007E
:108300000000000000000000000000007E3E380871
:10831000180818100C100C100C2006200620034022
:108320000340038001800180018001800180018081
:1083300001800180018007E00000000000000000D3
:10834000000000000000000000000000000000002D
:10835000000000000000000000000000000000001D
:10836000000000000000000000000000000000000D
:1083700000000000000000000000000000000000FD
:108380000000000000000000000000001FFE1C0CA8
:10839000180C3018201800300060006000C000C0C9
:1083A0000180018003000300060006000C00180293
:1083B00018063004301C7FFC0000000000000000A4
:1083C00000000000000000000000000000000000AD
:1083D000000000000000000000000000000000009D
:1083E000000000000000000000000000000000008D
:1083F000000000000000000000000000000000007D
:1084000000000000000003FC030003000300030061
:108410000300030003000300030003000300030044
:108420000300030003000300030003000300030034
:108430000300030003000300030003FC000000002E
:10844000000000000000000000000000000000002C
:10845000000000000000000000000000000000001C
:10846000000000000000000000000000000000000C
:1084700000000000000000000000000000000000FC
:1084800000000000000000000000180018000800B4
:108490000C00040006000600020003000100018039
:1084A0000180008000C000400060006000300030AB
:1084B000003000180018000C000C000C0006000032
:1084C00000000000000000000000000000000000AC
:1084D000000000000000000000000000000000009C
:1084E000000000000000000000000000000000008C
:1084F000000000000000000000000000000000007C
:108500000000000000003FC000C000C000C000C06C
:1085100000C000C000C000C000C000C000C000C05B
:1085200000C000C000C000C000C000C000C000C04B
:1085300000C000C000C000C000C03FC0000000007C
:10854000000000000000000000000000000000002B
:10855000000000000000000000000000000000001B
:10856000000000000000000000000000000000000B
:1085700000000000000000000000000000000000FB
:108580000000000003C003E0062008100000000007
:1085900000000000000000000000000000000000DB
:1085A00000000000000000000000000000000000CB
:1085B00000000000000000000000000000000000BB
:1085C00000000000000000000000000000000000AB
:1085D000000000000000000000000000000000009B
:1085E000000000000000000000000000000000008B
:1085F000000000000000000000000000000000007B
:10860000000000000000000000000000000000006A
:10861000000000000000000000000000000000005A
:10862000000000000000000000000000000000004A
:108630000000000000000000000000000000FFFF3C
:10864000000000000000000000000000000000002A
:10865000000000000000000000000000000000001A
:10866000000000000000000000000000000000000A
:1086700000000000000000000000000000000000FA
:10868000000000001E000300008000000000000049
:1086900000000000000000000000000000000000DA
:1086A00000000000000000000000000000000000CA
:1086B00000000000000000000000000000000000BA
:1086C00000000000000000000000000000000000AA
:1086D000000000000000000000000000000000009A
:1086E000000000000000000000000000000000008A
:1086F000000000000000000000000000000000007A
:108700000000000000000000000000000000000069
:108710000000000000000000000007E018303018E2
:1087200030183018003807D81C1830186018601836
:108730006018601930791F8E0000000000000000F2
:108740000000000000000000000000000000000029
:108750000000000000000000000000000000000019
:108760000000000000000000000000000000000009
:1087700000000000000000000000000000000000F9
:108780000000000000000000000008007800180051
:108790001800180018001800180019E01A381C18E2
:1087A0001C0C180C180C180C180C180C180C180CA5
:1087B00018081C181C3013E0000000000000000026
:1087C00000000000000000000000000000000000A9
:1087D0000000000000000000000000000000000099
:1087E0000000000000000000000000000000000089
:1087F0000000000000000000000000000000000079
:108800000000000000000000000000000000000068
:108810000000000000000000000003E00E100C1833
:1088200018183018300030003000300030003004AC
:10883000180418080C1003E00000000000000000FD
:108840000000000000000000000000000000000028
:108850000000000000000000000000000000000018
:108860000000000000000000000000000000000008
:1088700000000000000000000000000000000000F8
:108880000000000000000000000000080078001850
:108890000018001800180018001807D80C3818180D
:1088A00018183018301830183018301830183018A0
:1088B000101818380C5E079000000000000000003F
:1088C00000000000000000000000000000000000A8
:1088D0000000000000000000000000000000000098
:1088E0000000000000000000000000000000000088
:1088F0000000000000000000000000000000000078
:108900000000000000000000000000000000000067
:108910000000000000000000000003C00C30081838
:108920001808300C300C300C3FFC300030003000A8
:10893000180418080E1803E00000000000000000F2
:108940000000000000000000000000000000000027
:108950000000000000000000000000000000000017
:108960000000000000000000000000000000000007
:1089700000000000000000000000000000000000F7
:10898000000000000000000000000000007C0186E4
:10899000010603060300030003003FF80300030081
:1089A00003000300030003000300030003000300AF
:1089B0000300030003001FF000000000000000009F
:1089C00000000000000000000000000000000000A7
:1089D0000000000000000000000000000000000097
:1089E0000000000000000000000000000000000087
:1089F0000000000000000000000000000000000077
:108A00000000000000000000000000000000000066
:108A10000000000000000000000003EE0C36081803
:108A200018181818181808180C300FE0180018003B
:108A30001FC00FF8181C300C300C300C181807E051
:108A40000000000000000000000000000000000026
:108A50000000000000000000000000000000000016
:108A60000000000000000000000000000000000006
:108A700000000000000000000000000000000000F6
:108A8000000000000000000000000800780018004E
:108A90001800180018001800180019E01A301C18E7
:108AA0001818181818181818181818181818181846
:108AB0001818181818187E7E00000000000000002A
:108AC00000000000000000000000000000000000A6
:108AD0000000000000000000000000000000000096
:108AE0000000000000000000000000000000000086
:108AF0000000000000000000000000000000000076
:108B0000000000000000000000000000018003C021
:108B1000018000000000000000801F8001800180B3
:108B2000018001800180018001800180018001803D
:108B30000180018001801FF800000000000000009B
:108B40000000000000000000000000000000000025
:108B50000000000000000000000000000000000015
:108B60000000000000000000000000000000000005
:108B700000000000000000000000000000000000F5
:108B80000000000000000000000000000038007835
:108B90000030000000000000001003F00030003042
:108BA0000030003000300030003000300030003045
:108BB00000300030003000300030186018400F8066
:108BC00000000000000000000000000000000000A5
:108BD0000000000000000000000000000000000095
:108BE0000000000000000000000000000000000085
:108BF0000000000000000000000000000000000075
:108C000000000000000000000000080078001800CC
:108C100018001800180018001800187C18301820C8
:108C20001840188019801B801EC01CC018601830A6
:108C300018301818181C7E3E0000000000000000CC
:108C40000000000000000000000000000000000024
:108C50000000000000000000000000000000000014
:108C60000000000000000000000000000000000004
:108C700000000000000000000000000000000000F4
:108C80000000000000000000000000801F80018044
:108C900001800180018001800180018001800180CC
:108CA00001800180018001800180018001800180BC
:108CB0000180018001801FF800000000000000001A
:108CC00000000000000000000000000000000000A4
:108CD0000000000000000000000000000000000094
:108CE0000000000000000000000000000000000084
:108CF0000000000000000000000000000000000074
:108D00000000000000000000000000000000000063
:108D100000000000000000002000EF3C71C66186EA
:108D2000618661866186618661866186618661860B
:108D3000618661866186F3CF0000000000000000BC
:108D40000000000000000000000000000000000023
:108D50000000000000000000000000000000000013
:108D60000000000000000000000000000000000003
:108D700000000000000000000000000000000000F3
:108D800000000000000000000000000000000000E3
:108D90000000000000000000000009E07A301C180C
:108DA0001818181818181818181818181818181843
:108DB0001818181818187E7E000000000000000027
:108DC00000000000000000000000000000000000A3
:108DD0000000000000000000000000000000000093
:108DE0000000000000000000000000000000000083
:108DF0000000000000000000000000000000000073
:108E00000000000000000000000000000000000062
:108E10000000000000000000000003C00C30081833
:108E20001818100C300C300C300C300C300C300C8E
:108E3000181818180C3003C00000000000000000D3
:108E40000000000000000000000000000000000022
:108E50000000000000000000000000000000000012
:108E60000000000000000000000000000000000002
:108E700000000000000000000000000000000000F2
:108E800000000000000000000000000000000000E2
:108E90000000000000000000000009E07A301C180B
:108EA0001808180C180C180C180C180C180C180CA6
:108EB00018181C181E3019E01800180018007E0041
:108EC00000000000000000000000000000000000A2
:108ED0000000000000000000000000000000000092
:108EE0000000000000000000000000000000000082
:108EF0000000000000000000000000000000000072
:108F00000000000000000000000000000000000061
:108F10000000000000000000000003C80C781838B2
:108F20001818301830183018301830183018301819
:108F3000101818380C780798001800180018007ED0
:108F40000000000000000000000000000000000021
:108F50000000000000000000000000000000000011
:108F60000000000000000000000000000000000001
:108F700000000000000000000000000000000000F1
:108F800000000000000000000000000000000000E1
:108F900000000000000000000000061C7E6606863F
:108FA000078007000600060006000600060006000F
:108FB0000600060006007FE0000000000000000040
:108FC00000000000000000000000000000000000A1
:108FD0000000000000000000000000000000000091
:108FE0000000000000000000000000000000000081
:108FF0000000000000000000000000000000000071
:109000000000000000000000000000000000000060
:109010000000000000000000000003E4061C0C0C2F
:109020000C040C040E0007C001F00078001C100CAA
:10903000100C180C1C1813F00000000000000000B9
:109040000000000000000000000000000000000020
:109050000000000000000000000000000000000010
:109060000000000000000000000000000000000000
:1090700000000000000000000000000000000000F0
:1090800000000000000000000000000000000000E0
:10909000010001000100030007003FF80300030086
:1090A00003000300030003000300030003000300A8
:1090B00003040304018800F0000000000000000029
:1090C00000000000000000000000000000000000A0
:1090D0000000000000000000000000000000000090
:1090E0000000000000000000000000000000000080
:1090F0000000000000000000000000000000000070
:10910000000000000000000000000000000000005F
:1091100000000000000000000808787818181818EF
:1091200018181818181818181818181818181818BF
:10913000181818380C5E07900000000000000000AE
:10914000000000000000000000000000000000001F
:10915000000000000000000000000000000000000F
:1091600000000000000000000000000000000000FF
:1091700000000000000000000000000000000000EF
:1091800000000000000000000000000000000000DF
:10919000000000000000000000007C3E180C1808D1
:1091A00018180C100C100420062006200340034061
:1091B00003C00180018001000000000000000000E9
:1091C000000000000000000000000000000000009F
:1091D000000000000000000000000000000000008F
:1091E000000000000000000000000000000000007F
:1091F000000000000000000000000000000000006F
:10920000000000000000000000000000000000005E
:1092100000000000000000000000FBCF61862184F8
:109220003184318431C811C81AC81A481A700E70B6
:109230000C700C300C200420000000000000000026
:10924000000000000000000000000000000000001E
:10925000000000000000000000000000000000000E
:1092600000000000000000000000000000000000FE
:1092700000000000000000000000000000000000EE
:1092800000000000000000000000000000000000DE
:10929000000000000000000000003E7C0C100E10DA
:1092A0000620034003400180018001C00260046089
:1092B0000430081818187C7E000000000000000030
:1092C000000000000000000000000000000000009E
:1092D000000000000000000000000000000000008E
:1092E000000000000000000000000000000000007E
:1092F000000000000000000000000000000000006E
:10930000000000000000000000000000000000005D
:10931000000000000000000000007C3E181818103B
:1093200008100C10042006200620024003400140D3
:109330000180018001000100010002003E003C00AC
:10934000000000000000000000000000000000001D
:10935000000000000000000000000000000000000D
:1093600000000000000000000000000000000000FD
:1093700000000000000000000000000000000000ED
:1093800000000000000000000000000000000000DD
:10939000000000000000000000003FF830383030CE
:1093A000206020E000C001800380030006000E045E
:1093B0000C04180C30183FF80000000000000000FA
:1093C000000000000000000000000000000000009D
:1093D000000000000000000000000000000000008D
:1093E000000000000000000000000000000000007D
:1093F000000000000000000000000000000000006D
:1094000000000000000C00100020002000200020C0
:10941000002000200020002000200020002000C0AC
:1094200001800040002000200020002000200020BB
:10943000002000200020002000200010000C000070
:10944000000000000000000000000000000000001C
:10945000000000000000000000000000000000000C
:1094600000000000000000000000000000000000FC
:1094700000000000000000000000000000000000EC
:1094800000800080008000800080008000800080DC
:1094900000800080008000800080008000800080CC
:1094A00000800080008000800080008000800080BC
:1094B00000800080008000800080008000800080AC
:1094C000000000000000000000000000000000009C
:1094D000000000000000000000000000000000008C
:1094E000000000000000000000000000000000007C
:1094F000000000000000000000000000000000006C
:109500000000000018000400020002000200020037
:1095100002000200020002000200020002000180BC
:1095200000C001000200020002000200020002006E
:109530000200020002000200020004001800000005
:10954000000000000000000000000000000000001B
:10955000000000000000000000000000000000000B
:1095600000000000000000000000000000000000FB
:1095700000000000000000000000000000000000EB
:1095800000001E0023004182408200E400380000F9
:1095900000000000000000000000000000000000CB
:1095A00000000000000000000000000000000000BB
:1095B00000000000000000000000000000000000AB
:1095C000000000000000000000000000000000009B
:1099F000FFFFFFFFFFFFFFFFFFFFFFFFFFFFFFDF97
:109A0000F5F6EE16F719FF3BFF7CFF9DFFBEFFFF4B
:109A1000FFFFFFBEFF7CFF5CF71AF71BEEB8FEB935
:109A2000FFDFFFFFFFFFFFFFFFFFFFFFFFFFFFFF66
:109A3000FFFFFFFFFFFFFFFFFFFFFFFFFFFFFFFF36
:109A4000FFFFFFFFFFFFFFFFFFFFFFFFFFFFFFFF26
:109A5000FFFFFFFFFFFFFFFFFFFFFFFFFFFFFFFF16
:109A6000FFFFFFFFFFFFFFFFFFFFFFFFFFFFFFFF06
:109A7000FFFFFFFFFFFFFFFFFFFFFFFFFFFFFFFFF6
:109A8000FFFFFFFFFFFFFFFFFFFFFFFFFFFFFFFFE6
:109A9000FFFFFFFFFFFFFFFFFFFFFFFFFFFFFFFFD6
:109AA000FFFFFFFFFFFFFFFFFFFFFFFFFFFFFFFFC6
:109AB000FFFFFFFFFFFFFFFFFFFFFFFFFFFFFFFFB6
:109AC000FFFFFFFFFFFFFFFFFFFFFFFFFFFFFFFFA6
:109AD000FFFFFFFFFFFFFFFFFFFFFFFFFFFFFFFF96
:109AE000FFFFFFFFFFFFFFFFFFFFFFFFFFFFFFFF86
:109AF000FFFFFFFFFFFFFFFFFFFFFFFFFFFFFFFF76
:109B0000FFFFFFFFFFFFFFFFFFFFFFFFFFFFFFFF65
:109B1000FFFFFFFFFFFFFFFFFFFFFFFFFFFFFFFF55
:109B2000FFFFFFFFFFFFFFFFFFFFFFFFFFFFFFFF45
:109B3000FFFFFFFFFFFFFFFFFFFFFFFFFFFFFFFF35
:109B4000FFFFFFFFFFFFFFFFFFFFFFFFFFFFFFFF25
:109B5000FFFFFFFFFFFFFFFFFFFFFFFFFFFFFFFF15
:109B6000FFFFFFFFFFFFFFFFFFFFFFFFFFFFFFFF05
:109B7000FFFFFFFFFFFFFFFFFFFFFFFFFFFFFFFFF5
:109B8000FFFFFFFFFFFFFFFFFFFFFFFFFFFFFFFFE5
:109B9000FFFFFFFFFFFFFFFFFFFFFFFFFFFFFFFFD5
:109BA000FFFFFFFFFFFFFFFFFFFFFFFFFFFFFFFFC5
:109BB000FFFFFFFFFFFFFFFFFFFFFFFFFFFFFFFFB5
:109BC000FFFFFFFFFFFFFFFFFFFFFFFFFFFFFFFFA5
:109BD000FFFFFFFFFFFFFFFFFEFBC986FD51FED821
:109BE000FE98FED9F71AFF3BFF7CFF9DFFBEFFDE0C
:109BF000FFDEFFBDFF7CFF5CFF1AFEFAF6D8F677AA
:109C0000F697F4D0B8E4ED15FFDFFFFFFFFFFFFF8D
:109C1000FFFFFFFFFFFFFFFFFFFFFFFFFFFFFFFF54
:109C2000FFFFFFFFFFFFFFFFFFFFFFFFFFFFFFFF44
:109C3000FFFFFFFFFFFFFFFFFFFFFFFFFFFFFFFF34
:109C4000FFFFFFFFFFFFFFFFFFFFFFFFFFFFFFFF24
:109C5000FFFFFFFFFFFFFFFFFFFFFFFFFFFFFFFF14
:109C6000FFFFFFFFFFFFFFFFFFFFFFFFFFFFFFFF04
:109C7000FFFFFFFFFFFFFFFFFFFFFFFFFFFFFFFFF4
:109C8000FFFFFFFFFFFFFFFFFFFFFFFFFFFFFFFFE4
:109C9000FFFFFFFFFFFFFFFFFFFFFFFFFFFFFFFFD4
:109CA000FFFFFFFFFFFFFFFFFFFFFFFFFFFFFFFFC4
:109CB000FFFFFFFFFFFFFFFFFFFFFFFFFFFFFFFFB4
:109CC000FFFFFFFFFFFFFFFFFFFFFFFFFFFFFFFFA4
:109CD000FFFFFFFFFFFFFFFFFFFFFFFFFFFFFFFF94
:109CE000FFFFFFFFFFFFFFFFFFFFFFFFFFFFFFFF84
:109CF000FFFFFFFFFFFFFFFFFFFFFFFFFFFFFFFF74
:109D0000FFFFFFFFFFFFFFFFFFFFFFFFFFFFFFFF63
:109D1000FFFFFFFFFFFFFFFFFFFFFFFFFFFFFFFF53
:109D2000FFFFFFFFFFFFFFFFFFFFFFFFFFFFFFFF43
:109D3000FFFFFFFFFFFFFFFFFFFFFFFFFFFFFFFF33
:109D4000FFFFFFFFFFFFFFFFFFFFFFFFFFFFFFFF23
:109D5000FFFFFFFFFFFFFFFFFFFFFFFFFFFFFFFF13
:109D6000FFFFFFFFFFFFFFFFFFFFFFFFFFFFFFFF03
:109D7000FFFFFFFFFFFFFFFFFFFFFFFFFFFFFFFFF3
:109D8000FFFFFFFFFFFFFFFFFFFFFFFFFFFFFFFFE3
:109D9000FFFFFFFFFFFFFFFFFFFFFFFFFFFFFFFFD3
:109DA000FFFFFFFFFFFFFFFFFFFFFFFFFFFFFFFFC3
:109DB000FFFFFEBBD023E1A5FE14F615FE56F67795
:109DC000FEB8FED9FEFAFF3AFF5BFF7CFF9DFF9DC8
:109DD000FF9DFF7CFF5CFF5BFF1AF6D9F6B8F677B4
:109DE000F656EE15EDD4F5F4C144C002C209FF7D6C
:109DF000FFFFFFFFFFFFFFFFFFFFFFFFFFFFFFFF73
:109E0000FFFFFFFFFFFFFFFFFFFFFFFFFFFFFFFF62
:109E1000FFFFFFFFFFFFFFFFFFFFFFFFFFFFFFFF52
:109E2000FFFFFFFFFFFFFFFFFFFFFFFFFFFFFFFF42
:109E3000FFFFFFFFFFFFFFFFFFFFFFFFFFFFFFFF32
:109E4000FFFFFFFFFFFFFFFFFFFFFFFFFFFFFFFF22
:109E5000FFFFFFFFFFFFFFFFFFFFFFFFFFFFFFFF12
:109E6000FFFFFFFFFFFFFFFFFFFFFFFFFFFFFFFF02
:109E7000FFFFFFFFFFFFFFFFFFFFFFFFFFFFFFFFF2
:109E8000FFFFFFFFFFFFFFFFFFFFFFFFFFFFFFFFE2
:109E9000FFFFFFFFFFFFFFFFFFFFFFFFFFFFFFFFD2
:109EA000FFFFFFFFFFFFFFFFFFFFFFFFFFFFFFFFC2
:109EB000FFFFFFFFFFFFFFFFFFFFFFFFFFFFFFFFB2
:109EC000FFFFFFFFFFFFFFFFFFFFFFFFFFFFFFFFA2
:109ED000FFFFFFFFFFFFFFFFFFFFFFFFFFFFFFFF92
:109EE000FFFFFFFFFFFFFFFFFFFFFFFFFFFFFFFF82
:109EF000FFFFFFFFFFFFFFFFFFFFFFFFFFFFFFFF72
:109F0000FFFFFFFFFFFFFFFFFFFFFFFFFFFFFFFF61
:109F1000FFFFFFFFFFFFFFFFFFFFFFFFFFFFFFFF51
:109F2000FFFFFFFFFFFFFFFFFFFFFFFFFFFFFFFF41
:109F3000FFFFFFFFFFFFFFFFFFFFFFFFFFFFFFFF31
:109F4000FFFFFFFFFFFFFFFFFFFFFFFFFFFFFFFF21
:109F5000FFFFFFFFFFFFFFFFFFFFFFFFFFFFFFFF11
:109F6000FFFFFFFFFFFFFFFFFFFFFFFFFFFFFFFF01
:109F7000FFFFFFFFFFFFFFFFFFFFFFFFFFFFFFFFF1
:109F8000FFFFFFFFFFFFFFFFFFFFFFFFFFFFFEFBE6
:109F9000E002E001FDD3FDB3F5F3F614F636F676F4
:109FA000FE97FEB8FEF9FF1AFF3BFF5CFF5CFF7CEB
:109FB000FF7CFF5CFF3BFF1AF6FAF6B9F698F657FE
:109FC000F636EE15EDB4ED93ED52ED30C001C00262
:109FD000B842FEDBFFFFFFFFFFFFFFFFFFFFFFFFBA
:109FE000FFFFFFFFFFFFFFFFFFFFFFFFFFFFFFFF81
:109FF000FFFFFFFFFFFFFFFFFFFFFFFFFFFFFFFF71
:10A00000FFFFFFFFFFFFFFFFFFFFFFFFFFFFFFFF60
:10A01000FFFFFFFFFFFFFFFFFFFFFFFFFFFFFFFF50
:10A02000FFFFFFFFFFFFFFFFFFFFFFFFFFFFFFFF40
:10A03000FFFFFFFFFFFFFFFFFFFFFFFFFFFFFFFF30
:10A04000FFFFFFFFFFFFFFFFFFFFFFFFFFFFFFFF20
:10A05000FFFFFFFFFFFFFFFFFFFFFFFFFFFFFFFF10
:10A06000FFFFFFFFFFFFFFFFFFFFFFFFFFFFFFFF00
:10A07000FFFFFFFFFFFFFFFFFFFFFFFFFFFFFFFFF0
:10A08000FFFFFFFFFFFFFFFFFFFFFFFFFFFFFFFFE0
:10A09000FFFFFFFFFFFFFFFFFFFFFFFFFFFFFFFFD0
:10A0A000FFFFFFFFFFFFFFFFFFFFFFFFFFFFFFFFC0
:10A0B000FFFFFFFFFFFFFFFFFFFFFFFFFFFFFFFFB0
:10A0C000FFFFFFFFFFFFFFFFFFFFFFFFFFFFFFFFA0
:10A0D000FFFFFFFFFFFFFFFFFFFFFFFFFFFFFFFF90
:10A0E000FFFFFFFFFFFFFFFFFFFFFFFFFFFFFFFF80
:10A0F000FFFFFFFFFFFFFFFFFFFFFFFFFFFFFFFF70
:10A10000FFFFFFFFFFFFFFFFFFFFFFFFFFFFFFFF5F
:10A11000FFFFFFFFFFFFFFFFFFFFFFFFFFFFFFFF4F
:10A12000FFFFFFFFFFFFFFFFFFFFFFFFFFFFFFFF3F
:10A13000FFFFFFFFFFFFFFFFFFFFFFFFFFFFFFFF2F
:10A14000FFFFFFFFFFFFFFFFFFFFFFFFFFFFFFFF1F
:10A15000FFFFFFFFFFFFFFFFFFFFFFFFFFFFFFFF0F
:10A16000FFFFFFFFFFFFFFFFFFFFFDD7E002E00261
:10A17000FC6EF531F571F592F5D3F5F4F635F6563A
:10A18000F677F6B8FED8FEF9FF1AFF3AFF3BFF3B21
:10A19000FF3BFF3BFF1AFEFAF6D9F6B8F697F656E4
:10A1A000EE35EDF4EDB3ED72ED51E510E4CFDBCC1F
:10A1B000C002B822B822ECF4FFFFFFFFFFFFFFFF51
:10A1C000FFFFFFFFFFFFFFFFFFFFFFFFFFFFFFFF9F
:10A1D000FFFFFFFFFFFFFFFFFFFFFFFFFFFFFFFF8F
:10A1E000FFFFFFFFFFFFFFFFFFFFFFFFFFFFFFFF7F
:10A1F000FFFFFFFFFFFFFFFFFFFFFFFFFFFFFFFF6F
:10A20000FFFFFFFFFFFFFFFFFFFFFFFFFFFFFFFF5E
:10A21000FFFFFFFFFFFFFFFFFFFFFFFFFFFFFFFF4E
:10A22000FFFFFFFFFFFFFFFFFFFFFFFFFFFFFFFF3E
:10A23000FFFFFFFFFFFFFFFFFFFFFFFFFFFFFFFF2E
:10A24000FFFFFFFFFFFFFFFFFFFFFFFFFFFFFFFF1E
:10A25000FFFFFFFFFFFFFFFFFFFFFFFFFFFFFFFF0E
:10A26000FFFFFFFFFFFFFFFFFFFFFFFFFFFFFFFFFE
:10A27000FFFFFFFFFFFFFFFFFFFFFFFFFFFFFFFFEE
:10A28000FFFFFFFFFFFFFFFFFFFFFFFFFFFFFFFFDE
:10A29000FFFFFFFFFFFFFFFFFFFFFFFFFFFFFFFFCE
:10A2A000FFFFFFFFFFFFFFFFFFFFFFFFFFFFFFFFBE
:10A2B000FFFFFFFFFFFFFFFFFFFFFFFFFFFFFFFFAE
:10A2C000FFFFFFFFFFFFFFFFFFFFFFFFFFFFFFFF9E
:10A2D000FFFFFFFFFFFFFFFFFFFFFFFFFFFFFFFF8E
:10A2E000FFFFFFFFFFFFFFFFFFFFFFFFFFFFFFFF7E
:10A2F000FFFFFFFFFFFFFFFFFFFFFFFFFFFFFFFF6E
:10A30000FFFFFFFFFFFFFFFFFFFFFFFFFFFFFFFF5D
:10A31000FFFFFFFFFFFFFFFFFFFFFFFFFFFFFFFF4D
:10A32000FFFFFFFFFFFFFFFFFFFFFFFFFFFFFFFF3D
:10A33000FFFFFFFFFFFFFFFFFFFFFFFFFFFFFFFF2D
:10A34000FFFFFFFFFFFFFFFFD083E001D801F52FE4
:10A35000FD0FF530F571F592F5D3F5F4F615F635F8
:10A36000F676F697FEB8FED8FEF9FEFAFF1AFF1A47
:10A37000FF1AFF1AFEF9F6D9F6B8F698F677F63610
:10A38000EE15EDD4EDB3ED52E531E510DCCFE4AEE2
:10A39000DC6DB001B802B022B002FFBEFFFFFFFFCC
:10A3A000FFFFFFFFFFFFFFFFFFFFFFFFFFFFFFFFBD
:10A3B000FFFFFFFFFFFFFFFFFFFFFFFFFFFFFFFFAD
:10A3C000FFFFFFFFFFFFFFFFFFFFFFFFFFFFFFFF9D
:10A3D000FFFFFFFFFFFFFFFFFFFFFFFFFFFFFFFF8D
:10A3E000FFFFFFFFFFFFFFFFFFFFFFFFFFFFFFFF7D
:10A3F000FFFFFFFFFFFFFFFFFFFFFFFFFFFFFFFF6D
:10A40000FFFFFFFFFFFFFFFFFFFFFFFFFFFFFFFF5C
:10A41000FFFFFFFFFFFFFFFFFFFFFFFFFFFFFFFF4C
:10A42000FFFFFFFFFFFFFFFFFFFFFFFFFFFFFFFF3C
:10A43000FFFFFFFFFFFFFFFFFFFFFFFFFFFFFFFF2C
:10A44000FFFFFFFFFFFFFFFFFFFFFFFFFFFFFFFF1C
:10A45000FFFFFFFFFFFFFFFFFFFFFFFFFFFFFFFF0C
:10A46000FFFFFFFFFFFFFFFFFFFFFFFFFFFFFFFFFC
:10A47000FFFFFFFFFFFFFFFFFFFFFFFFFFFFFFFFEC
:10A48000FFFFFFFFFFFFFFFFFFFFFFFFFFFFFFFFDC
:10A49000FFFFFFFFFFFFFFFFFFFFFFFFFFFFFFFFCC
:10A4A000FFFFFFFFFFFFFFFFFFFFFFFFFFFFFFFFBC
:10A4B000FFFFFFFFFFFFFFFFFFFFFFFFFFFFFFFFAC
:10A4C000FFFFFFFFFFFFFFFFFFFFFFFFFFFFFFFF9C
:10A4D000FFFFFFFFFFFFFFFFFFFFFFFFFFFFFFFF8C
:10A4E000FFFFFFFFFFFFFFFFFFFFFFFFFFFFFFFF7C
:10A4F000FFFFFFFFFFFFFFFFFFFFFFFFFFFFFFFF6C
:10A50000FFFFFFFFFFFFFFFFFFFFFFFFFFFFFFFF5B
:10A51000FFFFFFFFFFFFFFFFFFFFFFFFFFFFFFFF4B
:10A52000FFFFFFFFFF5EE002E002D841ECCEF4EE59
:10A53000F4EFF510F551F571F5B2F5D3F5F4F61524
:10A54000F636F656F677F697F6B8F6B8F6D9F6D99F
:10A55000F6D9F6D9F6B8F6B8F697F657F636F615F0
:10A56000EDF4EDB3E572E552E511E4F0E4AFE48E0D
:10A57000DC4DDC6DB001B802B022B802B9C9FFFFF2
:10A58000FFFFFFFFFFFFFFFFFFFFFFFFFFFFFFFFDB
:10A59000FFFFFFFFFFFFFFFFFFFFFFFFFFFFFFFFCB
:10A5A000FFFFFFFFFFFFFFFFFFFFFFFFFFFFFFFFBB
:10A5B000FFFFFFFFFFFFFFFFFFFFFFFFFFFFFFFFAB
:10A5C000FFFFFFFFFFFFFFFFFFFFFFFFFFFFFFFF9B
:10A5D000FFFFFFFFFFFFFFFFFFFFFFFFFFFFFFFF8B
:10A5E000FFFFFFFFFFFFFFFFFFFFFFFFFFFFFFFF7B
:10A5F000FFFFFFFFFFFFFFFFFFFFFFFFFFFFFFFF6B
:10A60000FFFFFFFFFFFFFFFFFFFFFFFFFFFFFFFF5A
:10A61000FFFFFFFFFFFFFFFFFFFFFFFFFFFFFFFF4A
:10A62000FFFFFFFFFFFFFFFFFFFFFFFFFFFFFFFF3A
:10A63000FFFFFFFFFFFFFFFFFFFFFFFFFFFFFFFF2A
:10A64000FFFFFFFFFFFFFFFFFFFFFFFFFFFFFFFF1A
:10A65000FFFFFFFFFFFFFFFFFFFFFFFFFFFFFFFF0A
:10A66000FFFFFFFFFFFFFFFFFFFFFFFFFFFFFFFFFA
:10A67000FFFFFFFFFFFFFFFFFFFFFFFFFFFFFFFFEA
:10A68000FFFFFFFFFFFFFFFFFFFFFFFFFFFFFFFFDA
:10A69000FFFFFFFFFFFFFFFFFFFFFFFFFFFFFFFFCA
:10A6A000FFFFFFFFFFFFFFFFFFFFFFFFFFFFFFFFBA
:10A6B000FFFFFFFFFFFFFFFFFFFFFFFFFFFFFFFFAA
:10A6C000FFFFFFFFFFFFFFFFFFFFFFFFFFFFFFFF9A
:10A6D000FFFFFFFFFFFFFFFFFFFFFFFFFFFFFFFF8A
:10A6E000FFFFFFFFFFFFFFFFFFFFFFFFFFFFFFFF7A
:10A6F000FFFFFFFFFFFFFFFFFFFFFFFFFFFFFFFF6A
:10A70000FFFFD967E801E001E041EC4CF46DF4AEE5
:10A71000F4EFF50FED30ED51F677FF7CFFFFFFFF13
:10A72000FFFFFFFFFFFFFFFFFFFFFFFFFFFFFFFF39
:10A73000FFFFFFFFFFFFFFFFFFFFFFFFFF5BEE36A7
:10A74000EDB3ED93ED52ED31E510E4CFDCAEDC6E10
:10A75000DC2DD40CD3CBB001B802B022B002A84299
:10A76000FFBEFFFFFFFFFFFFFFFFFFFFFFFFFFFF3A
:10A77000FFFFFFFFFFFFFFFFFFFFFFFFFFFFFFFFE9
:10A78000FFFFFFFFFFFFFFFFFFFFFFFFFFFFFFFFD9
:10A79000FFFFFFFFFFFFFFFFFFFFFFFFFFFFFFFFC9
:10A7A000FFFFFFFFFFFFFFFFFFFFFFFFFFFFFFFFB9
:10A7B000FFFFFFFFFFFFFFFFFFFFFFFFFFFFFFFFA9
:10A7C000FFFFFFFFFFFFFFFFFFFFFFFFFFFFFFFF99
:10A7D000FFFFFFFFFFFFFFFFFFFFFFFFFFFFFFFF89
:10A7E000FFFFFFFFFFFFFFFFFFFFFFFFFFFFFFFF79
:10A7F000FFFFFFFFFFFFFFFFFFFFFFFFFFFFFFFF69
:10A80000FFFFFFFFFFFFFFFFFFFFFFFFFFFFFFFF58
:10A81000FFFFFFFFFFFFFFFFFFFFFFFFFFFFFFFF48
:10A82000FFFFFFFFFFFFFFFFFFFFFFFFFFFFFFFF38
:10A83000FFFFFFFFFFFFFFFFFFFFFFFFFFFFFFFF28
:10A84000FFFFFFFFFFFFFFFFFFFFFFFFFFFFFFFF18
:10A85000FFFFFFFFFFFFFFFFFFFFFFFFFFFFFFFF08
:10A86000FFFFFFFFFFFFFFFFFFFFFFFFFFFFFFFFF8
:10A87000FFFFFFFFFFFFFFFFFFFFFFFFFFFFFFFFE8
:10A88000FFFFFFFFFFFFFFFFFFFFFFFFFFFFFFFFD8
:10A89000FFFFFFFFFFFFFFFFFFFFFFFFFFFFFFFFC8
:10A8A000FFFFFFFFFFFFFFFFFFFFFFFFFFFFFFFFB8
:10A8B000FFFFFFFFFFFFFFFFFFFFFFFFFFFFFFFFA8
:10A8C000FFFFFFFFFFFFFFFFFFFFFFFFFFFFFFFF98
:10A8D000FFFFFFFFFFFFFFFFFFFFFFFFFFFFFFFF88
:10A8E000E002E002E802D821F40BF42CF46CEC6DE9
:10A8F000ED71FFBDFFFFFFFFFFFFFFFFFFFFFFFF4A
:10A90000FFFFFFFFFFFFFFFFFFFFFFFFFFFFFFFF57
:10A91000FFFFFFFFFFFFFFFFFFFFFFFFFFFFFFFF47
:10A92000FFFFFFFFF6D9DCF0E4F0E4AFDC8EDC6D76
:10A93000DC2CDBECD3ABCBAAB001B002B002B0028E
:10A94000B002E535FFFFFFFFFFFFFFFFFFFFFFFF47
:10A95000FFFFFFFFFFFFFFFFFFFFFFFFFFFFFFFF07
:10A96000FFFFFFFFFFFFFFFFFFFFFFFFFFFFFFFFF7
:10A97000FFFFFFFFFFFFFFFFFFFFFFFFFFFFFFFFE7
:10A98000FFFFFFFFFFFFFFFFFFFFFFFFFFFFFFFFD7
:10A99000FFFFFFFFFFFFFFFFFFFFFFFFFFFFFFFFC7
:10A9A000FFFFFFFFFFFFFFFFFFFFFFFFFFFFFFFFB7
:10A9B000FFFFFFFFFFFFFFFFFFFFFFFFFFFFFFFFA7
:10A9C000FFFFFFFFFFFFFFFFFFFFFFFFFFFFFFFF97
:10A9D000FFFFFFFFFFFFFFFFFFFFFFFFFFFFFFFF87
:10A9E000FFFFFFFFFFFFFFFFFFFFFFFFFFFFFFFF77
:10A9F000FFFFFFFFFFFFFFFFFFFFFFFFFFFFFFFF67
:10AA0000FFFFFFFFFFFFFFFFFFFFFFFFFFFFFFFF56
:10AA1000FFFFFFFFFFFFFFFFFFFFFFFFFFFFFFFF46
:10AA2000FFFFFFFFFFFFFFFFFFFFFFFFFFFFFFFF36
:10AA3000FFFFFFFFFFFFFFFFFFFFFFFFFFFFFFFF26
:10AA4000FFFFFFFFFFFFFFFFFFFFFFFFFFFFFFFF16
:10AA5000FFFFFFFFFFFFFFFFFFFFFFFFFFFFFFFF06
:10AA6000FFFFFFFFFFFFFFFFFFFFFFFFFFFFFFFFF6
:10AA7000FFFFFFFFFFFFFFFFFFFFFFFFFFFFFFFFE6
:10AA8000FFFFFFFFFFFFFFFFFFFFFFFFFFFFFFFFD6
:10AA9000FFFFFFFFFFFFFFFFFFFFFFFFFFFFFFFFC6
:10AAA000FFFFFFFFFFFFFFFFFFFFFFFFFFFFFFFFB6
:10AAB000FFFFFFFFFFFFFFFFFFFFFFFFFFFFD802CA
:10AAC000E802E802E002F3C9EBCAE40BFF5BFFFF18
:10AAD000FFFFFFFFFFFFFFFFFFFFFFFFFFFFFFFF86
:10AAE000FFFFFFFFFFFFFFFFFFFFFFFFFFFFFFFF76
:10AAF000FFFFFFFFFFFFFFFFFFFFFFFFFFFFFFFF66
:10AB0000FFFFFFFFFFFFFFFFFFFFEE16DC6DDC2DF9
:10AB1000D40CD3CBD38ACB6AD34AB002A822B002DA
:10AB2000B002B002BAACFFFFFFFFFFFFFFFFFFFF65
:10AB3000FFFFFFFFFFFFFFFFFFFFFFFFFFFFFFFF25
:10AB4000FFFFFFFFFFFFFFFFFFFFFFFFFFFFFFFF15
:10AB5000FFFFFFFFFFFFFFFFFFFFFFFFFFFFFFFF05
:10AB6000FFFFFFFFFFFFFFFFFFFFFFFFFFFFFFFFF5
:10AB7000FFFFFFFFFFFFFFFFFFFFFFFFFFFFFFFFE5
:10AB8000FFFFFFFFFFFFFFFFFFFFFFFFFFFFFFFFD5
:10AB9000FFFFFFFFFFFFFFFFFFFFFFFFFFFFFFFFC5
:10ABA000FFFFFFFFFFFFFFFFFFFFFFFFFFFFFFFFB5
:10ABB000FFFFFFFFFFFFFFFFFFFFFFFFFFFFFFFFA5
:10ABC000FFFFFFFFFFFFFFFFFFFFFFFFFFFFFFFF95
:10ABD000FFFFFFFFFFFFFFFFFFFFFFFFFFFFFFFF85
:10ABE000FFFFFFFFFFFFFFFFFFFFFFFFFFFFFFFF75
:10ABF000FFFFFFFFFFFFFFFFFFFFFFFFFFFFFFFF65
:10AC0000FFFFFFFFFFFFFFFFFFFFFFFFFFFFFFFF54
:10AC1000FFFFFFFFFFFFFFFFFFFFFFFFFFFFFFFF44
:10AC2000FFFFFFFFFFFFFFFFFFFFFFFFFFFFFFFF34
:10AC3000FFFFFFFFFFFFFFFFFFFFFFFFFFFFFFFF24
:10AC4000FFFFFFFFFFFFFFFFFFFFFFFFFFFFFFFF14
:10AC5000FFFFFFFFFFFFFFFFFFFFFFFFFFFFFFFF04
:10AC6000FFFFFFFFFFFFFFFFFFFFFFFFFFFFFFFFF4
:10AC7000FFFFFFFFFFFFFFFFFFFFFFFFFFFFFFFFE4
:10AC8000FFFFFFFFFFFFFFFFFFFFFFFFFFFFFFFFD4
:10AC9000FFFFFFFFFFFFFFFFFFFFFFBEE002E0023D
:10ACA000E802E002F368F5B3FFFFFFFFFFFFFFFFDD
:10ACB000FFFFFFFFFFFFFFFFFFFFFFFFFFFFFFFFA4
:10ACC000FFFFFFFFFFFFFFFFFFFFFFFFFFFFFFFF94
:10ACD000FFFFFFFFFFFFFFFFFFFFFFFFFFFFFFFF84
:10ACE000FFFFFFFFFFFFFFFFFFFFFFFFFFFFFFFF74
:10ACF000CBCBD3AACB8ACB49CB08CAC8B022B002EF
:10AD0000A802A802B002B1A8FFFFFFFFFFFFFFFFEC
:10AD1000FFFFFFFFFFFFFFFFFFFFFFFFFFFFFFFF43
:10AD2000FFFFFFFFFFFFFFFFFFFFFFFFFFFFFFFF33
:10AD3000FFFFFFFFFFFFFFFFFFFFFFFFFFFFFFFF23
:10AD4000FFFFFFFFFFFFFFFFFFFFFFFFFFFFFFFF13
:10AD5000FFFFFFFFFFFFFFFFFFFFFFFFFFFFFFFF03
:10AD6000FFFFFFFFFFFFFFFFFFFFFFFFFFFFFFFFF3
:10AD7000FFFFFFFFFFFFFFFFFFFFFFFFFFFFFFFFE3
:10AD8000FFFFFFFFFFFFFFFFFFFFFFFFFFFFFFFFD3
:10AD9000FFFFFFFFFFFFFFFFFFFFFFFFFFFFFFFFC3
:10ADA000FFFFFFFFFFFFFFFFFFFFFFFFFFFFFFFFB3
:10ADB000FFFFFFFFFFFFFFFFFFFFFFFFFFFFFFFFA3
:10ADC000FFFFFFFFFFFFFFFFFFFFFFFFFFFFFFFF93
:10ADD000FFFFFFFFFFFFFFFFFFFFFFFFFFFFFFFF83
:10ADE000FFFFFFFFFFFFFFFFFFFFFFFFFFFFFFFF73
:10ADF000FFFFFFFFFFFFFFFFFFFFFFFFFFFFFFFF63
:10AE0000FFFFFFFFFFFFFFFFFFFFFFFFFFFFFFFF52
:10AE1000FFFFFFFFFFFFFFFFFFFFFFFFFFFFFFFF42
:10AE2000FFFFFFFFFFFFFFFFFFFFFFFFFFFFFFFF32
:10AE3000FFFFFFFFFFFFFFFFFFFFFFFFFFFFFFFF22
:10AE4000FFFFFFFFFFFFFFFFFFFFFFFFFFFFFFFF12
:10AE5000FFFFFFFFFFFFFFFFFFFFFFFFFFFFFFFF02
:10AE6000FFFFFFFFFFFFFFFFFFFFFFFFFFFFFFFFF2
:10AE7000FFFFFFFFFFFFFFFFFFFFE002E002E00236
:10AE8000E802EB6CFFFFFFFFFFFFFFFFFFFFFFFF8D
:10AE9000FFFFFFFFFFFFFFFFFFFFFFFFFFFFFFFFC2
:10AEA000FFFFFFFFFFFFFFFFFFFFFFFFFFFFFFFFB2
:10AEB000FFFFFFFFFFFFFFFFFFFFFFFFFFFFFFFFA2
:10AEC000FFFFFFFFFFFFFFFFFFFFFFFFFFFFFFFF92
:10AED000FFFFFFBEBB08CB49C328CAC7B0E3A80227
:10AEE000A802A802A802A802A9A7FFFFFFFFFFFF70
:10AEF000FFFFFFFFFFFFFFFFFFFFFFFFFFFFFFFF62
:10AF0000FFFFFFFFFFFFFFFFFFFFFFFFFFFFFFFF51
:10AF1000FFFFFFFFFFFFFFFFFFFFFFFFFFFFFFFF41
:10AF2000FFFFFFFFFFFFFFFFFFFFFFFFFFFFFFFF31
:10AF3000FFFFFFFFFFFFFFFFFFFFFFFFFFFFFFFF21
:10AF4000FFFFFFFFFFFFFFFFFFFFFFFFFFFFFFFF11
:10AF5000FFFFFFFFFFFFFFFFFFFFFFFFFFFFFFFF01
:10AF6000FFFFFFFFFFFFFFFFFFFFFFFFFFFFFFFFF1
:10AF7000FFFFFFFFFFFFFFFFFFFFFFFFFFFFFFFFE1
:10AF8000FFFFFFFFFFFFFFFFFFFFFFFFFFFFFFFFD1
:10AF9000FFFFFFFFFFFFFFFFFFFFFFFFFFFFFFFFC1
:10AFA000FFFFFFFFFFFFFFFFFFFFFFFFFFFFFFFFB1
:10AFB000FFFFFFFFFFFFFFFFFFFFFFFFFFFFFFFFA1
:10AFC000FFFFFFFFFFFFFFFFFFFFFFFFFFFFFFFF91
:10AFD000FFFFFFFFFFFFFFFFFFFFFFFFFFFFFFFF81
:10AFE000FFFFFFFFFFFFFFFFFFFFFFFFFFFFFFFF71
:10AFF000FFFFFFFFFFFFFFFFFFFFFFFFFFFFFFFF61
:10B00000FFFFFFFFFFFFFFFFFFFFFFFFFFFFFFFF50
:10B01000FFFFFFFFFFFFFFFFFFFFFFFFFFFFFFFF40
:10B02000FFFFFFFFFFFFFFFFFFFFFFFFFFFFFFFF30
:10B03000FFFFFFFFFFFFFFFFFFFFFFFFFFFFFFFF20
:10B04000FFFFFFFFFFFFFFFFFFFFFFFFFFFFFFFF10
:10B05000FFFFFFFFFFFFFFDFE002E002E001D96733
:10B06000FFFFFFFFFFFFFFFFFFFFFFFFFFFFFFFFF0
:10B07000FFFFFFFFFFFFFFFFFFFFFFFFFFFEFFBE22
:10B08000FFBEFFDDFFFFFFFFFFFFFFFFFFFFFFFF33
:10B09000FFFFFFFFFFFFFFFFFFFFFFFFFFFFFFFFC0
:10B0A000FFFFFFFFFFFFFFFFFFFFFFFFFFFFFFFFB0
:10B0B000FFFFFFFFFFFFFF5BC2C7C2A7C286A80159
:10B0C000A802A802A802A802A802A126FFFFFFFF6B
:10B0D000FFFFFFFFFFFFFFFFFFFFFFFFFFFFFFFF80
:10B0E000FFFFFFFFFFFFFFFFFFFFFFFFFFFFFFFF70
:10B0F000FFFFFFFFFFFFFFFFFFFFFFFFFFFFFFFF60
:10B10000FFFFFFFFFFFFFFFFFFFFFFFFFFFFFFFF4F
:10B11000FFFFFFFFFFFFFFFFFFFFFFFFFFFFFFFF3F
:10B12000FFFFFFFFFFFFFFFFFFFFFFFFFFFFFFFF2F
:10B13000FFFFFFFFFFFFFFFFFFFFFFFFFFFFFFFF1F
:10B14000FFFFFFFFFFFFFFFFFFFFFFFFFFFFFFFF0F
:10B15000FFFFFFFFFFFFFFFFFFFFFFFFFFFFFFFFFF
:10B16000FFFFFFFFFFFFFFFFFFFFFFFFFFFFFFFFEF
:10B17000FFFFFFFFFFFFFFFFFFFFFFFFFFFFFFFFDF
:10B18000FFFFFFFFFFFFFFFFFFFFFFFFFFFFFFFFCF
:10B19000FFFFFFFFFFFFFFFFFFFFFFFFFFFFFFFFBF
:10B1A000FFFFFFFFFFFFFFFFFFFFFFFFFFFFFFFFAF
:10B1B000FFFFFFFFFFFFFFFFFFFFFFFFFFFFFFFF9F
:10B1C000FFFFFFFFFFFFFFFFFFFFFFFFFFFFFFFF8F
:10B1D000FFFFFFFFFFFFFFFFFFFFFFFFFFFFFFFF7F
:10B1E000FFFFFFFFFFFFFFFFFFFFFFFFFFFFFFFF6F
:10B1F000FFFFFFFFFFFFFFFFFFFFFFFFFFFFFFFF5F
:10B20000FFFFFFFFFFFFFFFFFFFFFFFFFFFFFFFF4E
:10B21000FFFFFFFFFFFFFFFFFFFFFFFFFFFFFFFF3E
:10B22000FFFFFFFFFFFFFFFFFFFFFFFFFFFFFFFF2E
:10B23000FFFFFFFFFFFFE002E802E002FF7EFFFFEB
:10B24000FFFFFFFFFFFFFFFFFFFFFFFFFFFFFFBD50
:10B25000F636E48EE44DEC6DECAEECCEECEFECEFBC
:10B26000ED10ED30ED31ED51ED51ED51E552E5725E
:10B27000EE36FF7DFFFFFFFFFFFFFFFFFFFFFFFF3A
:10B28000FFFFFFFFFFFFFFFFFFFFFFFFFFFFFFFFCE
:10B29000FFFFFFFFFFFFFFFFFFDFB287C267C2268E
:10B2A000B002A802A802A802A802A002EDD7FFFFE0
:10B2B000FFFFFFFFFFFFFFFFFFFFFFFFFFFFFFFF9E
:10B2C000FFFFFFFFFFFFFFFFFFFFFFFFFFFFFFFF8E
:10B2D000FFFFFFFFFFFFFFFFFFFFFFFFFFFFFFFF7E
:10B2E000FFFFFFFFFFFFFFFFFFFFFFFFFFFFFFFF6E
:10B2F000FFFFFFFFFFFFFFFFFFFFFFFFFFFFFFFF5E
:10B30000FFFFFFFFFFFFFFFFFFFFFFFFFFFFFFFF4D
:10B31000FFFFFFFFFFFFFFFFFFFFFFFFFFFFFFFF3D
:10B32000FFFFFFFFFFFFFFFFFFFFFFFFFFFFFFFF2D
:10B33000FFFFFFFFFFFFFFFFFFFFFFFFFFFFFFFF1D
:10B34000FFFFFFFFFFFFFFFFFFFFFFFFFFFFFFFF0D
:10B35000FFFFFFFFFFFFFFFFFFFFFFFFFFFFFFFFFD
:10B36000FFFFFFFFFFFFFFFFFFFFFFFFFFFFFFFFED
:10B37000FFFFFFFFFFFFFFFFFFFFFFFFFFFFFFFFDD
:10B38000FFFFFFFFFFFFFFFFFFFFFFFFFFFFFFFFCD
:10B39000FFFFFFFFFFFFFFFFFFFFFFFFFFFFFFFFBD
:10B3A000FFFFFFFFFFFFFFFFFFFFFFFFFFFFFFFFAD
:10B3B000FFFFFFFFFFFFFFFFFFFFFFFFFFFFFFFF9D
:10B3C000FFFFFFFFFFFFFFFFFFFFFFFFFFFFFFFF8D
:10B3D000FFFFFFFFFFFFFFFFFFFFFFFFFFFFFFFF7D
:10B3E000FFFFFFFFFFFFFFFFFFFFFFFFFFFFFFFF6D
:10B3F000FFFFFFFFFFFFFFFFFFFFFFFFFFFFFFFF5D
:10B40000FFFFFFFFFFFFFFFFFFFFFFFFFFFFFFFF4C
:10B41000FFFFFFFFE003E001D084FFFFFFFFFFFF1E
:10B42000FFFFFFFFFFFFFFDFF5B3EB69F3A9EBEAD7
:10B43000EC0BEC2BEC4CEC6DEC8DECAEECCEECCFE5
:10B44000ECEFED10ED10ED30ED30ED31ED31ED3193
:10B45000ED30ED31ED30E510E5D4FFBEFFFFFFFF2D
:10B46000FFFFFFFFFFFFFFFFFFFFFFFFFFFFFFFFEC
:10B47000FFFFFFFFFFFFFFFFFFFFFFFFEDB5BA4537
:10B48000A802A802A802A802A002A002A001FFDF51
:10B49000FFFFFFFFFFFFFFFFFFFFFFFFFFFFFFFFBC
:10B4A000FFFFFFFFFFFFFFFFFFFFFFFFFFFFFFFFAC
:10B4B000FFFFFFFFFFFFFFFFFFFFFFFFFFFFFFFF9C
:10B4C000FFFFFFFFFFFFFFFFFFFFFFFFFFFFFFFF8C
:10B4D000FFFFFFFFFFFFFFFFFFFFFFFFFFFFFFFF7C
:10B4E000FFFFFFFFFFFFFFFFFFFFFFFFFFFFFFFF6C
:10B4F000FFFFFFFFFFFFFFFFFFFFFFFFFFFFFFFF5C
:10B50000FFFFFFFFFFFFFFFFFFFFFFFFFFFFFFFF4B
:10B51000FFFFFFFFFFFFFFFFFFFFFFFFFFFFFFFF3B
:10B52000FFFFFFFFFFFFFFFFFFFFFFFFFFFFFFFF2B
:10B53000FFFFFFFFFFFFFFFFFFFFFFFFFFFFFFFF1B
:10B54000FFFFFFFFFFFFFFFFFFFFFFFFFFFFFFFF0B
:10B55000FFFFFFFFFFFFFFFFFFFFFFFFFFFFFFFFFB
:10B56000FFFFFFFFFFFFFFFFFFFFFFFFFFFFFFFFEB
:10B57000FFFFFFFFFFFFFFFFFFFFFFFFFFFFFFFFDB
:10B58000FFFFFFFFFFFFFFFFFFFFFFFFFFFFFFFFCB
:10B59000FFFFFFFFFFFFFFFFFFFFFFFFFFFFFFFFBB
:10B5A000FFFFFFFFFFFFFFFFFFFFFFFFFFFFFFFFAB
:10B5B000FFFFFFFFFFFFFFFFFFFFFFFFFFFFFFFF9B
:10B5C000FFFFFFFFFFFFFFFFFFFFFFFFFFFFFFFF8B
:10B5D000FFFFFFFFFFFFFFFFFFFFFFFFFFFFFFFF7B
:10B5E000FFFFFFFFFFFFFFFFFFFFFFFFFFFFFFFF6B
:10B5F000FFFFD9A8E002FE79FFFFFFFFFFFFFFFF7B
:10B60000FF9DE349EAA6EB07EB48EB68EB89EBCA41
:10B61000EBCAEBEBEC0BEC4CEC4CEC6DEC8DECAECC
:10B62000ECAEECCFECCFECEFECEFECEFECF0ECF0C1
:10B63000ECF0E4EFE4F0E4CFE4CFE4AFE48EDCCF71
:10B64000FF9DFFFFFFFFFFFFFFFFFFFFFFFFFFFF6C
:10B65000FFFFFFFFFFFFFFFFFFFFFFFFFFFFFFFFFA
:10B66000B985A801A802A002A002A002A002A0021F
:10B67000FFFFFFFFFFFFFFFFFFFFFFFFFFFFFFFFDA
:10B68000FFFFFFFFFFFFFFFFFFFFFFFFFFFFFFFFCA
:10B69000FFFFFFFFFFFFFFFFFFFFFFFFFFFFFFFFBA
:10B6A000FFFFFFFFFFFFFFFFFFFFFFFFFFFFFFFFAA
:10B6B000FFFFFFFFFFFFFFFFFFFFFFFFFFFFFFFF9A
:10B6C000FFFFFFFFFFFFFFFFFFFFFFFFFFFFFFFF8A
:10B6D000FFFFFFFFFFFFFFFFFFFFFFFFFFFFFFFF7A
:10B6E000FFFFFFFFFFFFFFFFFFFFFFFFFFFFFFFF6A
:10B6F000FFFFFFFFFFFFFFFFFFFFFFFFFFFFFFFF5A
:10B70000FFFFFFFFFFFFFFFFFFFFFFFFFFFFFFFF49
:10B71000FFFFFFFFFFFFFFFFFFFFFFFFFFFFFFFF39
:10B72000FFFFFFFFFFFFFFFFFFFFFFFFFFFFFFFF29
:10B73000FFFFFFFFFFFFFFFFFFFFFFFFFFFFFFFF19
:10B74000FFFFFFFFFFFFFFFFFFFFFFFFFFFFFFFF09
:10B75000FFFFFFFFFFFFFFFFFFFFFFFFFFFFFFFFF9
:10B76000FFFFFFFFFFFFFFFFFFFFFFFFFFFFFFFFE9
:10B77000FFFFFFFFFFFFFFFFFFFFFFFFFFFFFFFFD9
:10B78000FFFFFFFFFFFFFFFFFFFFFFFFFFFFFFFFC9
:10B79000FFFFFFFFFFFFFFFFFFFFFFFFFFFFFFFFB9
:10B7A000FFFFFFFFFFFFFFFFFFFFFFFFFFFFFFFFA9
:10B7B000FFFFFFFFFFFFFFFFFFFFFFFFFFFFFFFF99
:10B7C000FFFFFFFFFFFFFFFFFFFFFFFFFFFFFFFF89
:10B7D000FD96E002FFDFFFFFFFFFFFFFFDB6DA246B
:10B7E000EA45EA86EAC6EAE7EB27EB48EB69EB892C
:10B7F000EBAAEBCAEBEBEC0BEC2CEC4CEC6DEC8D10
:10B80000E48EECAEECAEECAEECAFE4CFE4CFE4CF44
:10B81000E4CFE4AFE4AFE4AEE48EE46EDC6DE44D7F
:10B82000DC4DD40CFF1BFFFFFFFFFFFFFFFFFFFFFF
:10B83000FFFFFFFFFFFFFFFFFFFFFFFFFFFFFFFF18
:10B84000FFFFA001A802A002A002A002A001A00286
:10B85000A0A4FFFFFFFFFFFFFFFFFFFFFFFFFFFFB2
:10B86000FFFFFFFFFFFFFFFFFFFFFFFFFFFFFFFFE8
:10B87000FFFFFFFFFFFFFFFFFFFFFFFFFFFFFFFFD8
:10B88000FFFFFFFFFFFFFFFFFFFFFFFFFFFFFFFFC8
:10B89000FFFFFFFFFFFFFFFFFFFFFFFFFFFFFFFFB8
:10B8A000FFFFFFFFFFFFFFFFFFFFFFFFFFFFFFFFA8
:10B8B000FFFFFFFFFFFFFFFFFFFFFFFFFFFFFFFF98
:10B8C000FFFFFFFFFFFFFFFF65DC55FD55FD55FD49
:10B8D00055FD55FD763DFFFFFFFFFFFFFFFFFFFF1B
:10B8E000FFFFFFFFFFFFFFFFFFFFFFFFFFFFFFFF68
:10B8F000FFFFFFFFFFFFFFFFFFFFFFFFFFFFFFFF58
:10B90000FFFFFFFFFFFFFFFFFFFFFFFFFFFFFFFF47
:10B91000FFFFFFFFFFFFFFFFFFFFFFFFFFFFFFFF37
:10B92000FFFFFFFFFFFFFFFFFFFFFFFFFFFFFFFF27
:10B93000FFFFFFFFFFFFFFFFFFFFFFFFFFFFFFFF17
:10B94000FFFFFFFFFFFFFFFFFFFFFFFFFFFFFFFF07
:10B95000FFFFFFFFFFFFFFFFFFFFFFFFFFFFFFFFF7
:10B96000FFFFFFFFFFFFFFFFFFFFFFFFFFFFFFFFE7
:10B97000FFFFFFFFFFFFFFFFFFFFFFFFFFFFFFFFD7
:10B98000FFFFFFFFFFFFFFFFFFFFFFFFFFFFFFFFC7
:10B99000FFFFFFFFFFFFFFFFFFFFFFFFFFFFFFFFB7
:10B9A000FFFFFFFFFFFFFFFFFFFFFFFFFFFFFFDFC7
:10B9B000D823FFFFFFFFFFFFEB6EE002E144E9E465
:10B9C000EA24EA65EA86EAC6EAE7E327E348EB48C1
:10B9D000EB69EBA9EBAAE3A9DB69DBAADBCBDBEB29
:10B9E000DBCBDC0BE44CEC8DEC6EE48EE48DE48E72
:10B9F000E46EE46DE46EDC6DDC4DDC4DDC2DDC0CC6
:10BA0000DC0CDBEBD3CBD3AADCF1FFFFFFFFFFFFA6
:10BA1000FFFFFFFFFFFFFFFFFFFFFFFFFFFFFFFF36
:10BA2000FFFFFFFF9842A002A002A002A002A00216
:10BA30009802FF5DFFFFFFFFFFFFFFFFFFFFFFFF1C
:10BA4000FFFFFFFFFFFFFFFFFFFFFFFFFFFF051DE2
:10BA5000051D051D051D051D051D051D051D051DD6
:10BA6000051D051D051D051D051D051D051D051DC6
:10BA7000051D051D051D051D051D051D051D051DB6
:10BA8000051D051D051D051D051D051D04FD051CC8
:10BA9000FFFFFFFFFFFFFFFFFFFFFFFFFFFFFFFFB6
:10BAA000FFFFFFFFFFFFFFFF1D1C051D051D051DFF
:10BAB000051D04FD359CFFFFFFFFFFFFFFFFFFFF9C
:10BAC000FFFFFFFFFFFFFFFFFFFFFFFFFFFFFFFF86
:10BAD000FFFFFFFFFFFFFFFFFFFFFFFFFFFFFFFF76
:10BAE000FFFFFFFFFFFFEFFF04FC04FC04FC04FC6E
:10BAF00004FC04FC04FC04FC04FC04FC04FC04FC46
:10BB000004FC04FC04FC04FC04FC04FC04FC04FC35
:10BB100004FC04FC04FC04FC04FC04FC04FC04FC25
:10BB200004FC04FC04FC04FC04FCFFFFFFFFFFFF1B
:10BB3000FFFFFFFFD7DF051D04FD051D051D051DCA
:10BB4000051D051D051D051D051D051D051D051DE5
:10BB5000051D051D051D051D051D051D051D051DD5
:10BB6000051D051D051D051D051D051D051D051DC5
:10BB7000051D04FC051CEFDFFFFFFFFFFFFFFFFFBC
:10BB8000FFFFFFFFFFFFFFFFFFFFFFFFFFFFC8A457
:10BB9000FFFFFFFFFD96E802E802E002E164E9C46E
:10BBA000E204EA25EA65EA85EAA6DAC6F46EFEB89A
:10BBB000FFDFFFFFFFFFFFFFFFFFFFFFFFFFFFFFB5
:10BBC000FFFFFFFFFFFFFFFFFFFFFFBEF657E48E03
:10BBD000DC2CDC4DDC4DDC4CDC2CDC0CDBECD3EB6E
:10BBE000D3CBD3ABD38AD36AD349C2E7FF9DFFFF40
:10BBF000FFFFFFFFFFFFFFFFFFFFFFFFFFFFFFFF55
:10BC0000FFFFFFFFFFFFA002A001A001A00298011B
:10BC100098019802FFFFFFFFFFFFFFFFFFFFFFFFFD
:10BC2000FFFFFFFFFFFFFFFFFFFFFFFFFFFF051D00
:10BC3000051D051D051D051D051D051D051D051DF4
:10BC4000051D051D051D051D051D051D051D051DE4
:10BC5000051D051D051D051D051D051D051D051DD4
:10BC6000051D051D051D051D051D051D051C151CB6
:10BC7000FFFFFFFFFFFFFFFFFFFFFFFFFFFFFFFFD4
:10BC8000FFFFFFFFFFFFFFFF1D1C051D051D051D1D
:10BC9000051D04FC053D151C151C151C151C151C4B
:10BCA000151C151C151C151C151C151C151C151C0C
:10BCB000151C151C151C151C151C151C153CFFFF0F
:10BCC000FFFFFFFFFFFFEFFF051D051D051D051D04
:10BCD000051D051D051D051D051D051D051D051D54
:10BCE000051D051D051D051D051D051D051D051D44
:10BCF000051D051D051D051D051D051D051D051D34
:10BD0000051D051D051D051D1D5CFFFFFFFFFFFF38
:10BD1000FFFFFFFFD7BF04FD04FD051D051D051D29
:10BD2000051D051D051D051D051D051D051D051D03
:10BD3000051D051D051D051D051D051D051D051DF3
:10BD4000051D051D051D051D051D051D051D051DE3
:10BD5000051D04FD04FCEFDFFFFFFFFFFFFFFFFFFA
:10BD6000FFFFFFFFFFFFFFFFFFFFFFFFFFFFFFFFE3
:10BD7000FFFFD947E802E802E802E002E103E963D5
:10BD8000E1E4E1C3DB29FF9DFFFFFFFFFFFFFFFFB2
:10BD9000FFFFFFFFFFFFFFFFFFFFFFFFFFFFFFFFB3
:10BDA000FFFFFFFFFFFFFFFFFFFFFFFFFFFFFFFFA3
:10BDB000FFFFFFDFF6FAD44DDBCBD3EBDBCBDBAA07
:10BDC000D3AAD38AD369D349D328CB08CAE8BAC83F
:10BDD000FFFFFFFFFFFFFFFFFFFFFFFFFFFFFFFF73
:10BDE000FFFFFFFFFFFFFFFFA021A002A0029801BD
:10BDF000A0019801DCB3FFFFFFFFFFFFFFFFFFFF84
:10BE0000FFFFFFFFFFFFFFFFFFFFFFFFFFFF04FD3F
:10BE100004FD04FD04FD04FD04FD04FD04FD04FD1A
:10BE200004FD04FD04FD04FD04FD04FD04FD04FD0A
:10BE300004FD04FD04FD04FD04FD04FD04FD04FDFA
:10BE400004FD04FD04FD04FD04FD04FD04FDEFDF1D
:10BE5000FFFFFFFFFFFFFFFFFFFFFFFFFFFFFFFFF2
:10BE6000FFFFFFFFFFFFFFFF151C04FD04FD04FDA6
:10BE700004FD051D051C051D04FD04FD051D04FD37
:10BE800004FD051D04FD04FD051D04FD04FD051D47
:10BE900004FD04FD051D04FD04FD051C45BDFFFF5B
:10BEA000FFFFFFFFFFFFEFFF04FD04FD04FD04FDA6
:10BEB00004FD04FD04FD04FD04FD04FD04FD04FD7A
:10BEC00004FD04FD04FD04FD04FD04FD04FD04FD6A
:10BED00004FD04FD04FD04FD04FD04FD04FD04FD5A
:10BEE00004FD04FD04FD04FDEFFFFFFFFFFFFFFF66
:10BEF000FFFFFFFFD7BF04FD04FD04FD04FD04FDAB
:10BF000004FD04FD04FD04FD04FD04FD04FD04FD29
:10BF100004FD04FD04FD04FD04FD04FD04FD04FD19
:10BF200004FD04FD04FD04FD04FD04FD04FD04FD09
:10BF300004FD04FD04FCEFDFFFFFFFFFFFFFFFFF39
:10BF4000FFFFFFFFFFFFFFFFFFFFFFFFFFFFFFBF41
:10BF5000E002E002E002E002E002E062E8A3E3CDFA
:10BF6000FFFFFFFFFFFFFFFFFFFFFFFFFFFFFFFFE1
:10BF7000FFFFFFFFFFFFFFFFFFFFFFFFFFFFFFFFD1
:10BF8000FFFFFFFFFFFFFFFFFFFFFFFFFFFFFFFFC1
:10BF9000FFFFFFFFFFFFFFFFFFFFFFDFDCB0D389E5
:10BFA000D369D329CB29CB08CAE8CAC8C2C7C2877C
:10BFB000C266FF5CFFFFFFFFFFFFFFFFFFFFFFFF0A
:10BFC000FFFFFFFFFFFFFFFFA0029802980198010B
:10BFD000980198029801FFFFFFFFFFFFFFFFFFFF9F
:10BFE000FFFFFFFFFFFFFFFFFFFFFFFFFFFF04FC5F
:10BFF00004FC04FC04FC04FC04FC04FC04FC04FC41
:10C0000004FC04FC04FC04FC04DC04FC04FC04FC50
:10C0100004FC04FC04FC04FC04FC04FC04FC04FC20
:10C0200004FC04FC04FC04FC04FC04FC04FCFFFF12
:10C03000FFFFFFFFFFFFFFFFFFFFFFFFFFFFFFFF10
:10C04000FFFFFFFFFFFFFFFF14FB04FC04FC04FCE9
:10C0500004FC04FC04FC04FC04FC04FC04FC04FCE0
:10C0600004FC04FC04FC04FC04FC04FC04FC04FCD0
:10C0700004FC04FC04FC04FC04FC04FCFFFFFFFFC4
:10C08000FFFFFFFFFFFFEFFF04FC04FC04FC04FCC8
:10C0900004FC04FC04FC04FC04FC04FC04DC04FCC0
:10C0A00004FC04DC04FC04FC04FC04FC04FC04FCB0
:10C0B00004FC04FC04DC04DC04FC04DC04DC04FC00
:10C0C00004DC04DC04DD051DFFFFFFFFFFFFFFFFB5
:10C0D000FFFFFFFFD7BF04DD04FC04FC04FC04FCED
:10C0E00004FC04FC04FC04FC04FC04FC04FC04FC50
:10C0F00004FC04FC04FC04FC04FC04FC04FC04FC40
:10C1000004FC04FC04FC04FC04FC04FC04FC04FC2F
:10C1100004FC04FC04FCEFDFFFFFFFFFFFFFFFFF59
:10C12000FFFFFFFFFFFFFFFFFFFFFFFFFFDFE0015C
:10C13000E002E002E802E802E002FE79FFFFFFFF12
:10C14000FFFFFFFFFFFFFFFFFFFFFFFFFFFFFFFFFF
:10C15000FFFFFFFFFFFFFFFFFFFFFFFFFFFFFFFFEF
:10C16000FFFFFFFFFFFFFFFFFFFFFFFFFFFFFFFFDF
:10C17000FFFFFFFFFFFFFFFFFFFFFFFFFFFFFFFFCF
:10C18000EDF5CAE7CB08CAE8CAC7C2A7CA67C24664
:10C19000C225C226D46FFFFFFFFFFFFFFFFFFFFF97
:10C1A000FFFFFFFFFFFFA001A00298029801980186
:10C1B000980198029802B2ECFFFFFFFFFFFFFFFF1C
:10C1C000FFFFFFFFFFFFFFFFFFFFFFFFFFFF96DF08
:10C1D00096DF96DF96DF96DF96DF96DF96DF96DFB7
:10C1E00096DF96DF96DF96DF665E04FC04DC04DCF7
:10C1F00004DC04DC04DC96FF96DF96DF96DF96DF36
:10C2000096DF96DF96DF96DF96DF96DFCF7FFFFF24
:10C21000FFFFFFFFFFFFFFFFFFFFFFFFFFFFFFFF2E
:10C22000FFFFFFFFFFFFFFFF14FB04DC04DC04DC67
:10C2300004DC04DC04DC04DC04DC04DC04DC04DCFE
:10C2400004DC04DC04DC04DC04DC04DC04DC04DCEE
:10C2500004DC04DC04DC04DC04DC24DAFFDFFFFFA4
:10C26000FFFFFFFFFFFFEFFF04FC04DC04DC04DC46
:10C2700004DD14DBFFFFFFFFFFFFFFFFFFFFFFFFFA
:10C28000FFFFFFFFFFFFFFFFFFFFF7FFF7FFF7FFD6
:10C29000F7FFF7FFFFFFFFFFFFFFFFFFFFFFFFFFBE
:10C2A000FFFFFFFFFFFFFFFFFFFFFFFFFFFFFFFF9E
:10C2B000FFFFFFFFDFDF251B251C253C253C253C20
:10C2C000253C253C253C253C253C253C253C253C66
:10C2D0001CFB0CDB0CDB0CDB0CDB0CDB0CDB0CDBF6
:10C2E0000CDB0CDB0CDA04DC04DC04DC04DC04DC3A
:10C2F00004DC04DC04FCEFBFFFFFFFFFFFFFFFFFD8
:10C30000FFFFFFFFFFFFFFFFFFFFFFFFE802E0026D
:10C31000E802E803D043FF9DFFFFFFFFFFFFFFFFA1
:10C32000FFFFFFFFFFFFFFFFFFFFFFFFFFFFFFFF1D
:10C33000FFFFFFFFFFFFFFFFFFFFFFFFFFFFFFFF0D
:10C34000FFFFFFFFFFFFFFFFFFFFFFFFFFFFFFFFFD
:10C35000FFFFFFFFFFFFFFFFFFFFFFFFFFFFFFFFED
:10C36000FFFFFFFFFF3BBA46CA87C267C246BA2536
:10C37000BA05B9E5B1A4A9C5FFFFFFFFFFFFFFFFA5
:10C38000FFFFFFFF9801A002A00298019801980109
:10C390009801980190029001FFFFFFFFFFFFFFFF50
:10C3A000FFFFFFFFFFFFFFFFFFFFFFFFFFFFFFFF9D
:10C3B000FFFFFFFFFFFFFFFFFFFFFFFFFFFFFFFF8D
:10C3C000FFFFFFFFFFFFFFFFA71F04DC04DC04DC0F
:10C3D00004DC04DC04DCFFFFFFFFFFFFFFFFFFFFC7
:10C3E000FFFFFFFFFFFFFFFFFFFFFFFFFFFFFFFF5D
:10C3F000FFFFFFFFFFFFFFFFFFFFFFFFFFFFFFFF4D
:10C40000FFFFFFFFFFFFFFFF14FB04DC04DC04DC85
:10C4100004DC04DC2D5CBF9FBF9FBF9FBF9FBF9FFD
:10C42000BF9FBF9FBF9FBF9FBF9FBF9FBF9FBF9F1C
:10C43000BF9FBF9FBF9FBF9FBF9FFFFFFFFFFFFF2C
:10C44000FFFFFFFFFFFFEFFF04DC04DC04DC04DC84
:10C4500004DC1CDAFFFFFFFFFFFFFFFFFFFFFFFF12
:10C46000FFFFFFFFFFFFFFFF459C04DC04DC04DC53
:10C4700004DC04DBB73FFFFFFFFFFFFFFFFFFFFF11
:10C48000FFFFFFFFFFFFFFFFFFFFFFFFFFFFFFFFBC
:10C49000FFFFFFFFFFFFFFFFFFFFFFFFFFFFFFFFAC
:10C4A000FFFFFFFFFFFFFFFFFFFFFFFFFFFFFFFF9C
:10C4B000FFFFFFFFFFFFFFFFFFFFFFFFFFFFFFFF8C
:10C4C000FFFFFFFFD7BF04DC04DC04DC04DC04DC7A
:10C4D00004DC04DCAF3FFFFFFFFFFFFFFFFFFFFFB8
:10C4E000FFFFFFFFFFFFFFFFFFFFD042E002E80278
:10C4F000E002FE18FFFFFFFFFFFFFFFFFFFFFFFF50
:10C50000FFFFFFFFFFFFFFFFFFFFFFFFFFFFF7FF43
:10C51000FFFFF7DFF7DFFFFFFFFFFFFFFFFFFFFF7B
:10C52000FFFFFFFFFFFFFFFFFFFFFFFFFFFFFFFF1B
:10C53000FFFFFFFFFFFFFFFFFFFFFFFFFFFFFFFF0B
:10C54000FFFFFFFFFFFFFFFFF656C246BA26BA0500
:10C55000B9C5B9A4B184B1449881FFFFFFFFFFFFC3
:10C56000FFFF9801A002A00298019801980198018C
:10C570009801980190019002FE59FFFFFFFFFFFF15
:10C58000FFFFFFFFFFFFFFFFFFFFFFFFFFFFFFFFBB
:10C59000FFFFFFFFFFFFFFFFFFFFFFFFFFFFFFFFAB
:10C5A000FFFFFFFFFFFFFFFFA71F04BC04DC04DC4D
:10C5B00004DC04DC04DCFFFFFFFFFFFFFFFFFFFFE5
:10C5C000FFFFFFFFFFFFFFFFFFFFFFFFFFFFFFFF7B
:10C5D000FFFFFFFFFFFFFFFFFFFFFFFFFFFFFFFF6B
:10C5E000FFFFFFFFFFFFFFFF14FB04DC04DC04DCA4
:10C5F00004DC04BC355CFFFFFFFFFFFFFFFFFFFF14
:10C60000FFFFFFFFFFFFFFFFFFFFFFFFFFFFFFFF3A
:10C61000FFFFFFFFFFFFFFFFFFFFFFFFFFFFFFFF2A
:10C62000FFFFFFFFFFFFEFFF04DC04DC04DC04DCA2
:10C6300004DC1CBAEFFF765E765E765E765E765E32
:10C64000765E765E765E763E04DC04DC04DC04DC3A
:10C6500004DC04BC7E5E765E765E765E765E765E3A
:10C66000765E765E765E765EB73EFFFFFFFFFFFF8B
:10C67000FFFFFFFFFFFFFFFFFFFFFFFFFFFFFFFFCA
:10C68000FFFFFFFFFFFFFFFFFFFFFFFFFFFFFFFFBA
:10C69000FFFFFFFFFFFFFFFFFFFFFFFFFFFFFFFFAA
:10C6A000FFFFF7FF04DC04DC04BB04DC04DC04DC77
:10C6B00004DC65FCFFFFFFFFFFFFFFFFFFFFFFFF45
:10C6C000FFFFFFFFFFFFFFFFF4B4E802E802E26BA9
:10C6D000FFFFFFFFFFFFFFFFFFFFFFFFFFFFFFFF6A
:10C6E000F7FFCF7F763C451B4D5C557C557C5D7BD1
:10C6F0005D5B655B655B6D5B6D5B6D7B6D5C6D1A3A
:10C700007D39BE9DF7BFFFFFFFFFFFFFFFFFFFFF6C
:10C71000FFFFFFFFFFFFFFFFFFFFFFFFFFFFFFFF29
:10C72000FFFFFFFFFFFFFFFFFFFFFFFEB1C4C1C51B
:10C73000B9A4B184B143B103A8C39904FFFFFFDFDB
:10C740009002A002A0029801980198019801980215
:10C7500098019001900190018822FFFFFFFFFFFFE9
:10C76000FFFFFFFFFFFFFFFFFFFFFFFFFFFFFFFFD9
:10C77000FFFFFFFFFFFFFFFFFFFFFFFFFFFFFFFFC9
:10C78000FFFFFFFFFFFFFFFFA71F04BC04BC04BCAB
:10C7900004BC04BC04BCFFFFFFFFFFFFFFFFFFFF63
:10C7A000FFFFFFFFFFFFFFFFFFFFFFFFFFFFFFFF99
:10C7B000FFFFFFFFFFFFFFFFFFFFFFFFFFFFFFFF89
:10C7C000FFFFFFFFFFFFFFFF14DB04BC04BC04BC42
:10C7D00004BC04DB353BFFFFFFFFFFFFFFFFFFFF54
:10C7E000FFFFFFFFFFFFFFFFFFFFFFFFFFFFFFFF59
:10C7F000FFFFFFFFFFFFFFFFFFFFFFFFFFFFFFFF49
:10C80000FFFFFFFFFFFFEFFF04BC04BC04BC04BC40
:10C8100004BC1CBADFBF04BB04BC04BC04BC04BC25
:10C8200004BC04BC04BC04BC04BC04BC04BC04BC08
:10C8300004BC04BC04BC04BC04BC04BC04BC04BCF8
:10C8400004BC04BC04BC04BC865DFFFFFFFFFFFF0B
:10C85000FFFFFFFFFFFFFFFFFFFFFFFFFFFFFFFFE8
:10C86000FFFFFFFFFFFFFFFFFFFFFFFFFFFFFFFFD8
:10C87000FFFFFFFFFFFFFFFFFFFFFFFFFFFFFFFFC8
:10C88000FFFF04BB04BC04BC04BC04BC04BC04BC6B
:10C890000CBBFFFFFFFFFFFFFFFFFFFFFFFFFFFFDF
:10C8A000FFFFFFFFFFFFFFFFE802E002FFDFFFFFE8
:10C8B000FFFFFFFFFFFFFFFFFFFF967D353B2D3C96
:10C8C0002D3B2D5B355C3D5C453C455B4D5B553BF5
:10C8D000553B5D3B5D3B653B653B653B6D3B6D3A69
:10C8E0006D1A6D1A6D1A6D1A6CFA7D1AE79FFFFFAB
:10C8F000FFFFFFFFFFFFFFFFFFFFFFFFFFFFFFFF48
:10C90000FFFFFFFFFFFFFFFFFFFFFFFFFFFFFEDA5D
:10C91000B144B143B103A8C3A882A8429821A0E5BD
:10C92000A001A002A0029801980198019801980125
:10C9300098019001900190019021FFDFFFFFFFFF20
:10C94000FFFFFFFFFFFFFFFFFFFFFFFFFFFFFFFFF7
:10C95000FFFFFFFFFFFFFFFFFFFFFFFFFFFFFFFFE7
:10C96000FFFFFFFFFFFFFFFFAF1F04BB04BB04BBC4
:10C9700004BB04BB04BBFFFFFFFFFFFFFFFFFFFF84
:10C98000FFFFFFFFFFFFFFFFFFFFFFFFFFFFFFFFB7
:10C99000FFFFFFFFFFFFFFFFFFFFF7FFEFFFEFFFCF
:10C9A000EFFFEFFFEFFFEFFF1CBA04BB04BB04BBBC
:10C9B00004BB04BB353BEFFFEFFFEFFFEFFFEFFFE3
:10C9C000EFFFEFFFEFFFEFFFEFFFEFFFEFFFEFFFF7
:10C9D000EFFFEFFFEFFFEFFFEFFFEFFFFFFFFFFFC7
:10C9E000FFFFFFFFFFFFEFFF04BB04BB04BB04BB63
:10C9F00004BB1C99DFBF04BB04BB04BB04BB04BB6A
:10CA000004BB04BB04BB04BB04BB04BB04BB04BB2E
:10CA100004BB04BB04BB04BB04BB04BB04BB04BB1E
:10CA200004BB04BB04BB04BB865DFFFFFFFFFFFF2D
:10CA3000FFFFFFFFFFFFFFFFFFFFFFFFFFFFFFFF06
:10CA4000FFFFFFFFFFFFFFFFFFFFFFFFFFFFFFFFF6
:10CA5000FFFFFFFFFFFFFFFFFFFFFFFFFFFFFFFFE6
:10CA600004BB04BB04BB04BB04BB04BB04BB047A0F
:10CA7000FFFFFFFFFFFFFFFFFFFFFFFFFFFFFFFFC6
:10CA8000FFFFFFFFFFFFFFFFE1A8FFFFFFFFFFFF2B
:10CA9000FFFFFFFFC77F355B2D3C2D3C2D3C2D3C20
:10CAA0002D3C253C2D1B353B3D1B3D1B451B451B94
:10CAB0004D1B551B551B5D1A5CFA64FA64FA64FA47
:10CAC00064FA64DA64DA64DA64DA6CD964B96C99A9
:10CAD00074D9FFFFFFFFFFFFFFFFFFFFFFFFFFFF17
:10CAE000FFFFFFFFFFFFFFFFFFFFFFFFFFFFFFFF56
:10CAF000FF7DB0E3A8C3A882A842A002A002A002C2
:10CB0000A002A002A0029801980198019801980142
:10CB10009001900190019001880199E8FFFFFFFFCB
:10CB2000FFFFFFFFFFFFFFFFFFFFFFFFFFFFFFFF15
:10CB3000FFFF6DFC6E3D761D761D761D6E3DBF5F61
:10CB4000FFFFFFFFFFFFFFFFAEFF049B049B049B63
:10CB5000049B049B049BFFFFFFFFFFFFFFFFFFFF02
:10CB6000FFFFFFFFFFFFFFFFFFFFFFFFFFFFFFFFD5
:10CB7000FFFFFFFFFFFFFFFFDFBF049B049B049B42
:10CB8000049B049B049B049B049B049B049B049BAD
:10CB9000049B049B049B049B049B049B049B049B9D
:10CBA000049B049B049B049B049B049B049B049B8D
:10CBB000049B049B049B049B049B049BF7FFFFFFC7
:10CBC000FFFFFFFFFFFFEFFF049B049B049B049B01
:10CBD000049B1C99DFBF049A049B049B049B049B49
:10CBE000049B049B049B049B049B049B049B049B4D
:10CBF000049B049B049B049B049B049C049B049B3C
:10CC0000049B049B049B049B863DFFFFFFFFFFFFEB
:10CC1000FFFFFFFFFFFFFFFFFFFFFFFFFFFFFFFF24
:10CC2000FFFFFFFFFFFFFFFFFFFFFFFFFFFFFFFF14
:10CC3000FFFFFFFFFFFFFFFFFFFFFFFFFFFF24D905
:10CC4000049B049B049B049B049B049B04BBFFFF6D
:10CC5000FFFFFFFFFFFFFFFFFFFFFFFFFFFFFFFFE4
:10CC6000FFFFFFFFFFFFFFFFFFFFFFFFFFFFFFFFD4
:10CC70004D9B2D5C255B2D3C2D3C2D3C2D3C2D3CB6
:10CC8000253B251B251B24FB2CFB34FB34FB3CFBE9
:10CC90003CFA44DA44FA4CDA54DA54DA54DA5CBA3C
:10CCA0005CB95CB95C995C995C995C995C795C79DC
:10CCB0005C585C3854389DDCFFFFFFFFFFFFFFFF2F
:10CCC000FFFFFFFFFFFFFFFFFFFFFFFFFFFFFFFF74
:10CCD000FFFFFFFFA842A822A002A002A002A0021C
:10CCE000A002A0029801980198019801980198016A
:10CCF000900190019001900190018801FFFFFFFFDA
:10CD0000FFFFFFFFFFFFFFFFFFFFFFFFFFFFFFFF33
:10CD1000FFFF0C9A049A047B047B047B047B8E9EA9
:10CD2000FFFFFFFFFFFFFFFFAEFF049A049B049B82
:10CD3000049B049B049BFFFFFFFFFFFFFFFFFFFF20
:10CD4000FFFFFFFFFFFFFFFFFFFFFFFFFFFFFFFFF3
:10CD5000FFFFFFFFFFFFFFFFDFBF049B049B049B60
:10CD6000049B049B049B049B049B049B049B049BCB
:10CD7000049B049B049B049B049B049B049B049BBB
:10CD8000049B049B049B049B049B049B049B049BAB
:10CD9000049B049B049B049B049B047AF7FFFFFF06
:10CDA000FFFFFFFFFFFFEFFF047B049B049B049B3F
:10CDB000049B1C79DFBF049A049B049B049B049B87
:10CDC000353BDFBFDFDFDFDFDFDFDFDFDFDFDFDFE1
:10CDD000DFDFDFDFDFDFDFDFDFDFE7BF6E1E047AED
:10CDE000049B049B049B049B863DFFFFFFFFFFFF0A
:10CDF000FFFFFFFFFFFFFFFFFFFFFFFFFFFFFFFF43
:10CE0000FFFFFFFFFFFFFFFFFFFFFFFFFFFFFFFF32
:10CE1000FFFFFFFFFFFFFFFFFFFFFFFF34FA049B51
:10CE2000049B049B049B049B049A049BFFFFFFFF4D
:10CE3000FFFFFFFFFFFFFFFFFFFFFFFFFFFFFFFF02
:10CE4000FFFFFFFFFFFFFFFFFFFFFFFF55BB253B7E
:10CE50002D3C2D3C2D3C2D3C2D3C255C2D3C253B7B
:10CE6000251B24FB24FB24FB24DA24DA2CDA34DA15
:10CE700034BA3CBA44BA44BA44B94C994CB95499FE
:10CE8000549954995479547954785458545854585E
:10CE9000543854385437D71EFFFFFFFFFFFFFFFF02
:10CEA000FFFFFFFFFFFFFFFFFFFFFFFFFFFFFFFF92
:10CEB000FFFFFFFFFFFFA802A001A002A002A00247
:10CEC000A002980198019801980198029801900198
:10CED000900190019001900188018801FF7DFFFF82
:10CEE000FFFFFFFFFFFFFFFFFFFFFFFFFFFFFFFF52
:10CEF000FFFF0C7A047B047B047B047B047A8E9E08
:10CF0000FFFFFFFFFFFFFFFFAEFF047A047B047B00
:10CF1000047B047B047BFFFFFFFFFFFFFFFFFFFF9E
:10CF2000FFFFFFFFFFFFFFFFFFFFFFFFFFFFFFFF11
:10CF3000FFFFFFFFFFFFFFFFDFBF047A047B047BDF
:10CF4000047B047B047A047B049B047B047B047BCA
:10CF5000047B047B047B047B047B047B047B047BD9
:10CF6000047B047B047B047B047B047B047B047BC9
:10CF7000047B047B047B047B047B049AFFFFFFFF9C
:10CF8000FFFFFFFFFFFFEFFF049B047B047B047A9E
:10CF9000047A1C79DFBF049A047B047B047B047B46
:10CFA000353BFFFFFFFFFFFFFFFFFFFFFFFFFFFF1F
:10CFB000FFFFFFFFFFFFFFFFFFFFFFFF7E5D049B03
:10CFC000047B047B047B047B863DFFFFFFFFFFFFA8
:10CFD000FFFFFFFFFFFFFFFFFFFFFFFFFFFFFFFF61
:10CFE000FFFFFFFFFFFFFFFFFFFFFFFFFFFFFFFF51
:10CFF000FFFFFFFFFFFFFFFFFFFF7E3D047B047B82
:10D00000047B047B049A047B047BCF9FFFFFFFFF1C
:10D01000FFFFFFFFFFFFFFFFFFFFFFFFFFFFFFFF20
:10D02000FFFFFFFFFFFFFFFF6E1C2D3C2D3C255C2B
:10D030002D5B2D3C2D3C2D3C2D3C253B251B251BE4
:10D0400024FB24FB24DA24DA24BA24BA249A2C9A66
:10D050002C99349934993C794499447944794C79A0
:10D060004C584C584C584C584C384C384C384C1840
:10D070004C184BF7F7DFFFFFFFFFFFFFFFFFFFFF3E
:10D08000FFFFFFFFFFFFFFFFFFFFFFFFFFFFFFFFB0
:10D09000FFFFFFFFFFFFFE18A002A002A001A002F9
:10D0A00098019801980298019801980198019001BF
:10D0B000900190019001900190018801A209FFFF69
:10D0C000FFFFFFFFFFFFFFFFFFFFFFFFFFFFFFFF70
:10D0D000FFFF0C79045A047A047A047A047A8E9E4B
:10D0E000FFFFFFFFFFFFFFFFAEFF047A047A047A21
:10D0F000047A047A047AFFFFFFFFFFFFFFFFFFFFC0
:10D10000FFFFFFFFFFFFFFFFFFFFFFFFFFFFFFFF2F
:10D11000FFFFFFFFFFFFFFFFDFBF047A047A047AFF
:10D12000047A047A047A047A047A047A047A047A0F
:10D13000047A047A047A047A047A047A047A047AFF
:10D14000047A047A047A047A047A047A047A045A0F
:10D15000047A047A047A047A047A047AFFFFFFFFDF
:10D16000FFFFFFFFFFFFEFFF047A047A047A047ADF
:10D17000047A1C59DFBF045A047A047A047A047AC8
:10D180003D1BFFFFFFFFFFFFFFFFFFFFFFFFFFFF55
:10D19000FFFFFFFFFFFFFFFFFFFFFFFF765D047A4A
:10D1A000047A047A047A047A863CFFFFFFFFFFFFCB
:10D1B000FFFFFFFFFFFFFFFFFFFFFFFFFFFFFFFF7F
:10D1C000FFFFFFFFFFFFFFFFFFFFFFFFFFFFFFFF6F
:10D1D000FFFFFFFFFFFFFFFFFFFF045A047A047AFF
:10D1E000047A047A047A047A8E7EFFFFFFFFFFFF41
:10D1F000FFFFFFFFFFFFFFFFFFFFFFFFFFFFFFFF3F
:10D20000FFFFFFFFFFFF2D3B2D5B255C2D3C2D3CE1
:10D210002D3C2D3C2D3C253C251B251B24FB24FBB4
:10D2200024DB24DA24BA24BA24BA249A249924794F
:10D2300024592C592C59345934383C383C583C38F2
:10D240003C3844384418441843F843F743F743D76D
:10D2500043D6FFFFFFFFFFFFFFFFFFFFFFFFFFFFC3
:10D26000FFFFFFFFFFFFFFFFFFFFFFFFFFFFFFFFCE
:10D27000FFFFFFFFED55A002A001A002A002A00247
:10D2800098019801980198029801980190019001E5
:10D290009001900190018801880188018801FFFFB9
:10D2A000FFFFFFFFFFFFFFFFFFFFFFFFFFFFFFFF8E
:10D2B000FFFF0C59045A045A045A045A045A8E7E29
:10D2C000FFFFFFFFFFFFFFFFAEFE045A045A045AA0
:10D2D000045A045A045A969E969E969E969E969E30
:10D2E000969E969E969E969E969E969E969E969E9E
:10D2F000BEFEFFFFFFFFFFFFDFBF045A045A045AC0
:10D30000045A045A045AFFFFFFFFFFFFFFFFFFFF0D
:10D31000FFFFFFFFFFFFFFFFFFFFFFFFFFFFFFFF1D
:10D32000FFFFFFFFFFFFFFFFFFFFFFFFFFFFFFFF0D
:10D33000045A045A045A045A045A045AFFFFFFFFBD
:10D34000FFFFFFFFFFFFEFFF045A045A045A045A7D
:10D35000045A1458DFBF045A045A045A045A045A8F
:10D36000045A045A045A045A045A045A045A045ACD
:10D37000045A045A045A04590459045A7E3D045A62
:10D38000045A045A045A045A861CFFFFFFFFFFFF89
:10D39000FFFFFFFFFFFFFFFFFFFFFFFFFFFFFFFF9D
:10D3A000FFFFFFFFFFFFFFFFFFFFFFFFFFFFFFFF8D
:10D3B000FFFFFFFFFFFFFFFFFFFF045A045A045A5D
:10D3C000045A045A045A147AFFFFFFFFFFFFFFFFBD
:10D3D000FFFFFFFFFFFFFFFFFFFFFFFFFFFFFFFF5D
:10D3E000FFFFFFFF457B2D3B2D3C2D3C2D3C2D3C75
:10D3F0002D3C2D3C253B251B251B251B24FB24DB1D
:10D4000024DA24BA24BA249A249A2479247924592F
:10D4100024592C392C382C382C382C183418341822
:10D42000341733F73BF733D73BD733D73BB72B55BD
:10D43000FFFFFFFFFFFFFFFFFFFFFFFFFFFFFFFFFC
:10D44000FFFFFFFFFFFFFFFFFFFFFFFFFFFFFFFFEC
:10D45000FFFFCB4EA002A002A002A002A002A002E9
:10D460009801980198019802980198019001900103
:10D470009001900190018801880188018801FFFFD7
:10D48000FFFFFFFFFFFFFFFFFFFFFFFFFFFFFFFFAC
:10D49000FFFF0C59045A045A045A045A045A8E7E47
:10D4A000FFFFFFFFFFFFFFFFAEDF045A045A045ADD
:10D4B000045A045A045A045A045A045A045A045A7C
:10D4C000045A045A045A045A045A045A043A043BAB
:10D4D000FFFFFFFFFFFFFFFFDFBF045A045A045A9C
:10D4E000045A045A045AFFFFFFFFFFFFFFFFFFFF2C
:10D4F000FFFFFFFFFFFFFFFFFFFFFFFFFFFFFFFF3C
:10D50000FFFFFFFFFFFFFFFFFFFFFFFFFFFFFFFF2B
:10D51000045A045A045A045A045A0459F7FFFFFFE4
:10D52000FFFFFFFFFFFFEFFF045A045A045A045A9B
:10D53000045A1458DFBF045A045A045A045A045AAD
:10D54000045A045A045A045A045A045A045A045AEB
:10D55000045A045A045A045A045AB6FE7E1D045A48
:10D56000045A045A045A045A861CFFFFFFFFFFFFA7
:10D57000FFFF045A045A045A045A045A045A045A1B
:10D58000045A045A045A045A045A045A045A045AAB
:10D59000045A045A045A045A045A043A045A045ABB
:10D5A000045A045A045A045A045A045A045A045A8B
:10D5B000045A045A0439FFFFFFFFFFFFFFFFFFFF7C
:10D5C000FFFFFFFF2D3B2D5B2D3C2D3C2D3C2D3CCB
:10D5D0002D3C253B251B251B24FB24FB24DA24DAC8
:10D5E00024BA24BA249A24992479245924592459F0
:10D5F000243924382418241823F823F823D723D7D0
:10D600002BD72BB72BB72BB72B972B972B76FFFF4F
:10D61000FFFFFFFFFFFFFFFFFFFFFFFFFFFFFFFF1A
:10D62000FFFFFFFFFFFFFFFFFFFFFFFFFFFFFFFF0A
:10D63000A968A002A002A002A002A002A002980174
:10D64000980198019801980198019001900190012A
:10D650009001880190018801880188018801FFFFFD
:10D66000FFFFFFFFFFFFFFFFFFFFFFFFFFFFFFFFCA
:10D67000FFFF0C39043A043A043A043A043A8E7E25
:10D68000FFFFFFFFFFFFFFFFAEDF043A043A043A5B
:10D69000043A043A043A043A043A043A043A043A9A
:10D6A000043A043A043A043A043A043A043A249A0A
:10D6B000FFFFFFFFFFFFFFFFDFBF043A043A043A1A
:10D6C000043A043A0439FFFFFFFFFFFFFFFFFFFFAB
:10D6D000FFFFFFFFFFFFFFFFFFFFFFFFFFFFFFFF5A
:10D6E000FFFFFFFFFFFFFFFFFFFFFFFFFFFFFFFF4A
:10D6F000043A043A043A043A043A0439F7FFFFFFC3
:10D70000FFFFFFFFFFFFEFFF043A043A043A04393A
:10D7100004391438DFBF043A043A043A043A043AAC
:10D72000043A043A043A043A043A043A043A043A09
:10D73000043A043A043A041A0439FFFF7E1D0439FE
:10D74000043A043A043A043A861CFFFFFFFFFFFF45
:10D75000FFFF0439043A04390439043A043904391E
:10D76000043A04390439043A04390439043A0439CE
:10D770000439043A04390439043A043A043A043ABC
:10D78000043A043A043A043A043A043A043A0439AA
:10D79000043A043A865DFFFFFFFFFFFFFFFFFFFF34
:10D7A000FFFFFFFF2D3C2D3C2D3C2D3C2D3C253B10
:10D7B000251B251B24FB24FB24DA24DA24BA24BAF3
:10D7C000249A249A247924792459245924592438D0
:10D7D0002418241823F823F823F71BD71BB71BB7EB
:10D7E0001B971B971B97237623764C16FFFFFFFF93
:10D7F000FFFFFFFFFFFFFFFFFFFFFFFFFFFFFFFF39
:10D80000FFFFFFFFFFFFFFFFFFFFFFFFFFFF98424C
:10D81000A802A002A002A002A002A0029801980102
:10D820009801980198019801900190019001900150
:10D830009001900190018801880188018801F6BA61
:10D84000FFFFFFFFFFFFFFFFFFFFFFFFFFFFFFFFE8
:10D85000FFFF0C38043904390439043904398E7E49
:10D86000FFFFFFFFFFFFFFFFAEDE0439043904397D
:10D8700004390439043904390439043904390439C0
:10D880000439043904390439043904390419FFFF0F
:10D89000FFFFFFFFFFFFFFFFDFBF0439043904393B
:10D8A000043904390439FFFFFFFFFFFFFFFFFFFFCB
:10D8B000FFFFFFFFFFFFFFFFFFFFFFFFFFFFFFFF78
:10D8C000FFFFFFFFFFFFFFFFFFFFFFFFFFFFFFFF68
:10D8D000043904390439043904390439F7FFFFFFE6
:10D8E000FFFFFFFFFFFFEFFF04390439043904395C
:10D8F00004391438DFBF04390439043904390439D0
:10D90000041A04390439043904390439043904394E
:10D91000043904390439043A6DBCFFFF7E1D043A12
:10D9200004390439043904397DFCFFFFFFFFFFFF90
:10D93000FFFF04390439043904390439043904393E
:10D9400004390439043904390439043904390439EF
:10D9500004390439043904390439043904390439DF
:10D9600004390439043904390439043904390439CF
:10D9700004390439FFFFFFFFFFFFFFFFFFFFFFFF39
:10D98000FFFFFFFF2D3C2D3C2D3C2D3C253B251B57
:10D99000251B24FB24FB24DA24DA24BA24BA249A93
:10D9A000249A247924792459245924392438241890
:10D9B000241823F81BF71BD71BD71BB71BB71B97C4
:10D9C0001B761B761B561B558DBBFFFFFFFFFFFF12
:10D9D000FFFFFFFFFFFFFFFFFFFFFFFFFFFFFFFF57
:10D9E000FFFFFFFFFFFFFFFFFFFFFFFFA002A002FF
:10D9F000A002A002A002A002A002A0029801980129
:10DA00009801980198019001900190019001900176
:10DA10009001900188018801880188018001C3F08C
:10DA2000FFFFFFFFFFFFFFFFFFFFFFFFFFFFFFFF06
:10DA3000FFFF0C18041904190419041904198E5D48
:10DA4000FFFFFFFFFFFFFFFFAEDE041904190419FB
:10DA500004190419041904190419041904190419DE
:10DA60000419041904190419041904190BF8FFFF07
:10DA7000FFFFFFFFFFFFFFFFDF9F041904190419D9
:10DA8000041904190419FFFFFFFFFFFFFFFFFFFF49
:10DA9000FFFFFFFFFFFFFFFFFFFFFFFFFFFFFFFF96
:10DAA000FFFFFFFFFFFFFFFFFFFFFFFFFFFFFFFF86
:10DAB000041904190419041904190419FFFFFFFFBC
:10DAC000FFFFFFFFFFFFEFFF0419041904190419FA
:10DAD00004191418DFBF04190419041904190419CE
:10DAE0003CF9FFFFFFFFFFFFFFFFFFFFFFFFFFFF0F
:10DAF000FFFFFFFFFFFFFFFFFFFFFFFF7E1D04395A
:10DB00000419041904190419861CFFFFFFFFFFFF05
:10DB1000FFFF04190419041904190419041904193C
:10DB2000041904190419041904190419041904190D
:10DB300004190419041904190419041904190419FD
:10DB400004190419041904190419041904190419ED
:10DB5000041985FCFFFFFFFFFFFFFFFFFFFFFFFF33
:10DB6000FFFFFFFF2D3C2D3C253C251B251B24FBE7
:10DB700024FB24DA24DA24BA24BA249A249A249995
:10DB8000247924592459245924382418241823F892
:10DB900023F723F71BD71BB71BB71B971B961B76C7
:10DBA0001B761B561355CF3FFFFFFFFFFFFFFFFF05
:10DBB000FFFFFFFFFFFFFFFFFFFFFFFFFFFFFFFF75
:10DBC000FFFFFFFFFFFFFFFFFF9EA802A802A802C2
:10DBD000A002A002A002A002A00298019801980150
:10DBE0009802980198019001900190019001900194
:10DBF000900188018801880188018801880191E8E5
:10DC0000FFFFFFFFFFFFFFFFFFFFFFFFFFFFFFFF24
:10DC1000FFFF0C18041904190419041904198E5D66
:10DC2000FFFFFFFFFFFFFFFFAEDE04190419041919
:10DC3000041904190419FFFFFFFFFFFFFFFFFFFF97
:10DC4000FFFFFFFFFFFFFFFFFFFFFFFFFFFFFFFFE4
:10DC5000FFFFFFFFFFFFFFFFDF9F041904190419F7
:10DC6000041904190419FFFFFFFFFFFFFFFFFFFF67
:10DC7000FFFFFFFFFFFFFFFFFFFFFFFFFFFFFFFFB4
:10DC8000FFFFFFFFFFFFFFFFFFFFFFFFFFFFFFFFA4
:10DC9000041904190419041904190418FFFFFFFFDB
:10DCA000FFFFFFFFFFFFEFFF041904190419041918
:10DCB00004191417DFBF04180419041904190419EE
:10DCC0003CD9FFFFFFFFFFFFFFFFFFFFFFFFFFFF4D
:10DCD000FFFFFFFFFFFFFFFFFFFFFFFF7E1C041999
:10DCE00004190419041804197DFCFFFFFFFFFFFF4E
:10DCF000FFFF0C18141814181418141814181418FA
:10DD000014181418141814181418141814181418B3
:10DD100014181418141814181418041904190419D0
:10DD200004190419041904191418141814181418CF
:10DD30001418FFFFFFFFFFFFFFFFFFFFFFFFFFFFC5
:10DD4000FFFFFFFF2D3C253B251B251B24FB24FB50
:10DD500024DA24DA24BA24BA249A249A2479245975
:10DD60002459245924392C382418241823F823F74B
:10DD70001BD71BD71BB71B971B971B961B761B76B6
:10DD80001B561B56EFDFFFFFFFFFFFFFFFFFFFFFED
:10DD9000FFFFFFFFFFFFFFFFFFFFFFFFFFFFFFFF93
:10DDA000FFFFFFFFFFFFFEBAA801A002A802A0022A
:10DDB000A002A002A002A002A0029801980198016E
:10DDC00098029801900190019001900190019001BA
:10DDD00090018801880188018801880180018945B6
:10DDE000FFFFFFFFFFFFFFFFFFFFFFFFFFFFFFFF43
:10DDF000FFFF0C1803F903F903F903F903F98E5D2A
:10DE0000FFFFFFFFFFFFFFFFAEBE03F903F903F9BA
:10DE100003F903F903F9FFFFFFFFFFFFFFFFFFFF18
:10DE2000FFFFFFFFFFFFFFFFFFFFFFFFFFFFFFFF02
:10DE3000FFFFFFFFFFFFFFFFDF9F03F903F903F978
:10DE400003F903F903F934992C992C792C792C795D
:10DE50002C792C792C792C792C792C792C792C799A
:10DE60002C792C792C792C792C792C792C782C986C
:10DE700003F903F903F903F903D8EFFFFFFFFFFFED
:10DE8000FFFFFFFFFFFFEFFF03F903F903F903F9BA
:10DE900003F91417DFBF03F803F903F903F903F9D2
:10DEA00034DAF7FFF7DFEFFFEFFFEFFFEFFFEFFFF2
:10DEB000EFFFEFFFEFFFEFFFEFFFF7FF6DFC041841
:10DEC00003F903F903F90418FFFFFFFFFFFFFFFF4A
:10DED000FFFFFFFFFFFFFFFFFFFFFFFFFFFFFFFF52
:10DEE000FFFFFFFFFFFFFFFFFFFFFFFFFFFFFFFF42
:10DEF000FFFFFFFFFFFFFFFFFFFF03F803F903F939
:10DF000003F903F903F80C19FFFFFFFFFFFFFFFF01
:10DF1000FFFFFFFFFFFFFFFFFFFFFFFFFFFFFFFF11
:10DF2000FFFFFFFF253B251B251B24FB24DB24DAF9
:10DF300024DA24BA249A249A249924792479245915
:10DF40002459243824382418241823F81BF71BD705
:10DF50001BB71BB71B971B971B961B761B561B5695
:10DF60001B36FFFFFFFFFFFFFFFFFFFFFFFFFFFF6E
:10DF7000FFFFFFFFFFFFFFFFFFFFFFFFFFFFFFFFB1
:10DF8000FFFFFFFFDC93A822A802A802A002A002C4
:10DF9000A002A002A002A002980198019801980294
:10DFA00098019801900190019001900190019001D9
:10DFB000880188018801880188018801800180C367
:10DFC000FFFFFFFFFFFFFFFFFFFFFFFFFFFFFFFF61
:10DFD000FFFF0BF703F803F803F803F803F88E5D6F
:10DFE000FFFFFFFFFFFFFFFFAEBE03F803F803F8DC
:10DFF00003F803F803F8FFFFFFFFFFFFFFFFFFFF3A
:10E00000FFFFFFFFFFFFFFFFFFFFFFFFFFFFFFFF20
:10E01000FFFFFFFFFFFFFFFFDF9F03F803F803F899
:10E0200003F803F803F803F803F803F803F803F818
:10E0300003F803F803F803F803F803F803F803F808
:10E0400003F803F803F803F803F803F803F803F8F8
:10E0500003F803F903F903D8FFFFFFFFFFFFFFFFFA
:10E06000FFFFFFFFFFFFF7FF03F803F803F803F8D4
:10E0700003F813F7DFBF03F803F803F803F803F816
:10E0800003F803F803F803F803F803F803F803F8B8
:10E0900003F803F803F803F803F803F803F803F9A7
:10E0A00003F803F81418FFFFFFFFFFFFFFFFFFFF58
:10E0B000FFFFFFFFFFFFFFFFFFFFFFFFFFFFFFFF70
:10E0C000FFFFFFFFFFFFFFFFFFFFFFFFFFFFFFFF60
:10E0D000FFFFFFFFFFFFFFFFFFFF03F803F803F859
:10E0E00003F803F803F913F8FFFFFFFFFFFFFFFF3B
:10E0F000FFFFFFFFFFFFFFFFFFFFFFFFFFFFFFFF30
:10E10000FFFFFFFF251B24FB24FB24DA24DA24BABB
:10E1100024BA249A24992479247924592459243816
:10E120002C382418241823F823F71BD71BD71BB728
:10E130001BB71B971B961B761B761B561B351B3478
:10E14000FFFFFFFFFFFFFFFFFFFFFFFFFFFFFFFFDF
:10E15000FFFFFFFFFFFFFFFFFFFFFFFFFFFFFFFFCF
:10E16000FFFFB20AA802A802A802A802A002A00209
:10E17000A002A002A00298019801980198019801BC
:10E1800098019001900190019001900190019001FF
:10E19000880188018801880188018001800180A3AD
:10E1A000FFFFFFFFFFFFFFFFFFFFFFFFFFFFFFFF7F
:10E1B000FFFF0BD703D803D803D803D803D88E3D6D
:10E1C000FFFFFFFFFFFFFFFFAEBE03D803D803D85A
:10E1D00003D803D803D8FFFFFFFFFFFFFFFFFFFFB8
:10E1E000FFFFFFFFFFFFFFFFFFFFFFFFFFFFFFFF3F
:10E1F000FFFFFFFFFFFFFFFFDFBF03D803D803D8F8
:10E2000003D803D803D803D803D803D803D803D836
:10E2100003D803D803D803D803D803D803D803D826
:10E2200003D803D803D803D803D803D803D803D816
:10E2300003D803D94CD9FFFFFFFFFFFFFFFFFFFF0C
:10E24000FFFFFFFFFFFFF7FF03D803D803D803D872
:10E2500003D813D7DF9F03D803D803D803D803D834
:10E2600003D803D803D803D803D803D803D803D8D6
:10E2700003D803D803D803D803D803D803D803D8C6
:10E2800003B8D77FFFFFFFFFFFFFFFFFFFFFFFFF89
:10E29000FFFFFFFFFFFFFFFFFFFFFFFFFFFFFFFF8E
:10E2A000FFFFFFFFFFFFFFFFFFFFFFFFFFFFFFFF7E
:10E2B000FFFFFFFFFFFFFFFFFFFF03D803D803D8D7
:10E2C00003D803D803D813F8FFFFFFFFFFFFFFFFBA
:10E2D000FFFFFFFFFFFFFFFFFFFFFFFFFFFFFFFF4E
:10E2E000FFFFFFFF24FB24DB24DA24DA24BA24BA5C
:10E2F000249A249924792479245924592C382C38A7
:10E300002418241823F823F71BD71BD71BB71B97F8
:10E310001B971B961B761B56135713353374FFFF41
:10E32000FFFFFFFFFFFFFFFFFFFFFFFFFFFFFFFFFD
:10E33000FFFFFFFFFFFFFFFFFFFFFFFFFFFFFFFFED
:10E34000A0C5A802A802A802A802A002A002A002DA
:10E35000A002A002A00298019801980198029801D9
:10E360009001900190019001900190018801880135
:10E370008801880188018801800180018001894528
:10E38000FFFFFFFFFFFFFFFFFFFFFFFFFFFFFFFF9D
:10E39000FFFF0BB703D803B803B803B803B88E5D0B
:10E3A000FFFFFFFFFFFFFFFFAEDE03B803B803B8B8
:10E3B00003B803B803B8FFFFFFFFFFFFFFFFFFFF36
:10E3C000FFFFFFFFFFFFFFFFFFFFFFFFFFFFFFFF5D
:10E3D000FFFFFFFFFFFFFFFFE79F03B703B803B88F
:10E3E00003B803B803B803B803B803B803B803B855
:10E3F00003B803B803B803B803B803B803B803B845
:10E4000003B803B803B803B803B803B803B803B834
:10E4100003D8B6DEFFFFFFFFFFFFFFFFFFFFFFFF99
:10E42000FFFFFFFFFFFFEFFF03D803B803B803B8F8
:10E4300003D813D7DF9F03B803D803D803D803D872
:10E4400003D803D803D803B803D803B803B803B874
:10E4500003B803D803B803D803D803B803B803D864
:10E46000F7FFFFFFFFFFFFFFFFFFFFFFFFFFFFFFC4
:10E47000FFFFFFFFFFFFFFFFFFFFFFFFFFFFFFFFAC
:10E48000FFFFFFFFFFFFFFFFFFFFFFFFFFFFFFFF9C
:10E49000FFFFFFFFFFFFFFFFFFFF03B703B803B856
:10E4A00003B803B803B80BD7FFFFFFFFFFFFFFFF61
:10E4B000FFFFFFFFFFFFFFFFFFFFFFFFFFFFFFFF6C
:10E4C000FFFFFFFF24DB24BA24BA24BA249A249A3B
:10E4D00024792479245924592C392C3824182418C7
:10E4E00023F823F81BD71BD71BB71BB71B971B970A
:10E4F0001B761B761B561B5613566CB8FFFFFFFF8F
:10E50000FFFFFFFFFFFFFFFFFFFFFFFFFFFFFFFF1B
:10E51000FFFFFFFFFFFFFFFFFFFFFFFFFFFFA8025F
:10E52000A802A802A802A802A002A002A002A002BB
:10E53000A002A00298019801980198019801980101
:10E540009001900190019001900190018801880153
:10E55000880188018801880180018001800191E89B
:10E56000FFFFFFFFFFFFFFFFFFFFFFFFFFFFFFFFBB
:10E57000FFFF0BB703B803B803B803B803B88E3D69
:10E58000FFFFFFFFFFFFFFFFAEBD03B803B803B8F7
:10E5900003B803B803B8FFFFFFFFFFFFFFFFFFFF54
:10E5A000FFFFFFFFFFFFFFFFFFFFFFFFFFFFFFFF7B
:10E5B000FFFFFFFFFFFFFFFFE77F1C182417241753
:10E5C0002417241724172417241724172417241773
:10E5D0002417241724172417241724172417241763
:10E5E0002417241724172417241724171C3724173B
:10E5F000FFFFFFFFFFFFFFFFFFFFFFFFFFFFFFFF2B
:10E60000FFFFFFFFFFFFF7FF03B803B803B803B82E
:10E6100003B713D6EFBF6D5A6D5A6D5A6D5A6D5AC6
:10E620006D5A6D5A6D7A6D5A13F803B803B803B872
:10E6300003B803B7657B6D5A6D5A6D5A7D9BFFFF1A
:10E64000FFFFFFFFFFFFFFFFFFFFFFFFFFFFFFFFDA
:10E65000FFFFFFFFFFFFFFFFFFFFFFFFFFFFFFFFCA
:10E66000FFFFFFFFFFFFFFFFFFFFFFFFFFFFFFFFBA
:10E67000FFFFFFFFFFFFFFFFFFFF039703B803B894
:10E6800003B803B803B813D7FFFFFFFFFFFFFFFF77
:10E69000FFFFFFFFFFFFFFFFFFFFFFFFFFFFFFFF8A
:10E6A000FFFFFFFF24DA24BA24BA249A249924799C
:10E6B00024792459245924382C182418241823F890
:10E6C00023D71BD71BD71BB71B971B971B761B7614
:10E6D0001B761B561B561B35A63CFFFFFFFFFFFF9B
:10E6E000FFFFFFFFFFFFFFFFFFFFFFFFFFFFFFFF3A
:10E6F000FFFFFFFFFFFFFFFFFFFFFFDFB002B002E2
:10E70000A802A802A802A802A002A002A002A002D9
:10E71000A00298019801980198029801980190012F
:10E720009001900190019001900190018801880171
:10E730008801880188018001800180018001A2ECAC
:10E74000FFFFFFFFFFFFFFFFFFFFFFFFFFFFFFFFD9
:10E75000FFFF0BB6039703970397039703988E3D2C
:10E76000FFFFFFFFFFFFFFFFAEBE03970397039777
:10E77000039703970397FFFFFFFFFFFFFFFFFFFFD5
:10E78000FFFFFFFFFFFFFFFFFFFFFFFFFFFFFFFF99
:10E79000FFFFFFFFFFFFFFFFFFFFFFFFFFFFFFFF89
:10E7A000FFFFFFFFFFFFFFFFFFFFFFFFFFFFFFFF79
:10E7B000FFFFFFFFFFFFFFFFFFFFFFFFFFFFFFFF69
:10E7C000FFFFFFFFFFFFFFFFFFFFFFFFFFFFFFFF59
:10E7D000FFFFFFFFFFFFFFFFFFFFFFFFFFFFFFFF49
:10E7E000FFFFFFFFFFFFF7FF0397039703970397D1
:10E7F00003971396FFFFFFFFFFFFFFFFFFFFFFFFE2
:10E80000FFFFFFFFFFFFFFFF13D703970397039758
:10E8100003970397E7DFFFFFFFFFFFFFFFFFFFFF08
:10E82000FFFFFFFFFFFFFFFFFFFFFFFFFFFFFFFFF8
:10E83000FFFFFFFFFFFFFFFFFFFFFFFFFFFFFFFFE8
:10E84000FFFFFFFFFFFFFFFFFFFFFFFFFFFFFFFFD8
:10E85000FFFFFFFFFFFFFFFFFFFF039703970397F4
:10E860000397039703980BB7FFFFFFFFFFFFFFFF1F
:10E87000FFFFFFFFFFFFFFFFFFFFFFFFFFFFFFFFA8
:10E88000FFFFFFFF24BA249A249A2479247924597B
:10E89000245924382C382418241823F823F81BD79B
:10E8A0001BD71BB71BB71B971B971B761B761B56DB
:10E8B0001B561B561B35E77FFFFFFFFFFFFFFFFFC8
:10E8C000FFFFFFFFFFFFFFFFFFFFFFFFFFFFFFFF58
:10E8D000FFFFFFFFFFFFFFFFFF7EA822B002A8029D
:10E8E000A802A802A802A002A002A002A002A00200
:10E8F000A00298019801980198029801980190014E
:10E900009001900190019001900188018801880197
:10E910008801880180018001800180018001DD96ED
:10E92000FFFFFFFFFFFFFFFFFFFFFFFFFFFFFFFFF7
:10E93000FFFF0B96039703970397039703978E3D6B
:10E94000FFFFFFFFFFFFFFFFAEBE03970397039795
:10E95000039703970397FFFFFFFFFFFFFFFFFFFFF3
:10E96000FFFFFFFFFFFFFFFFFFFFFFFFFFFFFFFFB7
:10E97000FFFFFFFFFFFFFFFFFFFFFFFFFFFF03970B
:10E9800003970397039703970397FFFF23D71BD79B
:10E990001BD71BD71BD723D7FFFFFFFF1BD71BD7C7
:10E9A0001BD71BD71BD71BD6FFFFFFFF0375039792
:10E9B0000397039703970397FFFFFFFFFFFFFFFFF7
:10E9C000FFFFFFFFFFFFF7FF0397039703970397EF
:10E9D00003971396FFFFFFFFFFFF0397039703972C
:10E9E000039703972C17FFFF13B60397039703971B
:10E9F00003970397E7DF9E9E039703970397039779
:10EA00000396FFFFFFFFFFFFFFFFFFFFFFFFFFFF7B
:10EA1000FFFFFFFFFFFFFFFFFFFFFFFFFFFFFFFF06
:10EA2000FFFFFFFFFFFFFFFFFFFFFFFFFFFFFFFFF6
:10EA3000FFFFFFFFFFFFFFFFFFFF03970397039712
:10EA40000397039703970BB7FFFFFFFFFFFFFFFF3E
:10EA5000FFFFFFFFFFFFFFFFFFFFFFFFFFFFFFFFC6
:10EA6000FFFFFFFF2499247A24792459245924593B
:10EA700024382C382418241823F81BF71BD71BB76D
:10EA80001BB71B971B971B761B761B561B561B35FC
:10EA90001B361B36FFFFFFFFFFFFFFFFFFFFFFFFE0
:10EAA000FFFFFFFFFFFFFFFFFFFFFFFFFFFFFFFF76
:10EAB000FFFFFFFFFFFFF5B7B002A802A802A80200
:10EAC000A802A802A802A002A002A002A002A0021E
:10EAD000980198019801980298019801900190017D
:10EAE00090019001900190018801880188018801BE
:10EAF0008801880180018001800180018001FF9EE2
:10EB0000FFFFFFFFFFFFFFFFFFFFFFFFFFFFFFFF15
:10EB1000FFFF0B76037703770377037703778E1D69
:10EB2000FFFFFFFFFFFFFFFFAE9E03770377037733
:10EB3000037703770377FFFFFFFFFFFFFFFFFFFF71
:10EB4000FFFFFFFFFFFFFFFFFFFFFFFFFFFFFFFFD5
:10EB5000FFFFFFFFFFFFFFFFFFFFFFFFE7BF0377A1
:10EB600003770377037703770356FFFF54D90377BF
:10EB70000377037703770377FFFFFFFF4C98037753
:10EB80000377037703770377FFFFFFFF9E5D03772C
:10EB90000377037703770377DF9FFFFFFFFFFFFF15
:10EBA000FFFFFFFFFFFFF7FF03770377037703778D
:10EBB00003771396FFFFFFFFA69E03770377037784
:10EBC00003770377FFFFFFFF13960377037703773E
:10EBD00003770397E7BFFFFF037603770377037796
:10EBE00003972418FFFFFFFFFFFFFFFFFFFFFFFF5B
:10EBF000FFFFFFFFFFFFFFFFFFFFFFFFFFFFFFFF25
:10EC0000FFFFFFFFFFFFFFFFFFFFFFFFFFFFFFFF14
:10EC1000FFFFFFFFFFFFFFFFFFFF03760377037791
:10EC20000377037703770B96FFFFFFFFFFFFFFFFDD
:10EC3000FFFFFFFFFFFFFFFFFFFFFFFFFFFFFFFFE4
:10EC4000FFFFFFFF2C7924792479245924392438B3
:10EC50002C38241823F823F81BD71BD71BD71BB736
:10EC60001B971B971B761B761B561B561B351B369B
:10EC70001B14FFFFFFFFFFFFFFFFFFFFFFFFFFFF73
:10EC8000FFFFFFFFFFFFFFFFFFFFFFFFFFFFFFFF94
:10EC9000FFFFFFDFCBAFB022A802B002A802A8029C
:10ECA000A802A802A002A002A002A002A002A00244
:10ECB000980198019801980298019801900190019B
:10ECC00090019001900190018801880188018801DC
:10ECD0008801880180018001800180017801FFFFA7
:10ECE000FFFFFFFFFFFFFFFFFFFFFFFFFFFFFFFF34
:10ECF000FFFF0B76035703570357037603578E1D09
:10ED0000FFFFFFFFFFFFFFFFAE9D035703570357B2
:10ED1000035703570357FFFFFFFFFFFFFFFFFFFFEF
:10ED2000FFFFFFFFFFFFFFFFFFFFFFFFFFFFFFFFF3
:10ED3000FFFFFFFFFFFFFFFFFFFFFFFF23B603768D
:10ED400003570357035703766D5AFFFFF7FF037707
:10ED500003760357035703779E5CFFFFEFDF0377CC
:10ED600003570357035703579E5DFFFFFFFF0357EA
:10ED7000035703570357035733F7FFFFFFFFFFFF07
:10ED8000FFFFFFFFFFFFF7FF03570357035703572B
:10ED900003761376FFFFFFFF0356037603570357EF
:10EDA00003760B96FFFFFFFF139603570357035796
:10EDB00003570377E7BFFFFF54D9035703570357A0
:10EDC00003570377FFFFFFFFFFFFFFFFFFFFFFFF7B
:10EDD000FFFFFFFFFFFFFFFFFFFFFFFFFFFFFFFF43
:10EDE000FFFFFFFFFFFFFFFFFFFFFFFFFFFFFFFF33
:10EDF000FFFFFFFFFFFFFFFFFFFF03560357035710
:10EE00000357035703770B96FFFFFFFFFFFFFFFF3B
:10EE1000FFFFFFFFFFFFFFFFFFFFFFFFFFFFFFFF02
:10EE2000FFFFFFFF4CFA2459245924382C392418A9
:10EE3000241823F823F81BD71BD71BB71B971B9746
:10EE40001B961B761B761B561B561B351B352B340E
:10EE5000FFFFFFFFFFFFFFFFFFFFFFFFFFFFFFFFC2
:10EE6000FFFFFFFFFFFFFFFFFFFFFFFFFFFFFFFFB2
:10EE7000FFFFA822B002B002B002A802A802A802B6
:10EE8000A802A802A002A002A002A002A00298026A
:10EE900098019801980198019801900190019001C2
:10EEA0009001900190018801880188018801880102
:10EEB0008801800180018001800180018001FFFFC5
:10EEC000FFFFFFFFFFFFFFFFFFFFFFFFFFFFFFFF52
:10EED000FFFF0B5603560356035603560356961C64
:10EEE000FFFFFFFFFFFFFFFFAE9D035603560356D4
:10EEF000035603560356FFFFFFFFFFFFFFFFFFFF11
:10EF0000FFFFFFFFFFFFFFFFFFFFFFFFFFFFFFFF11
:10EF1000FFFFFFFFFFFFFFFFFFFFFFFF035603564B
:10EF20000356035603560356FFFFFFFFFFFF03562A
:10EF300003560356035603570336FFFFFFFF0356DE
:10EF400003560356035603560355FFFFFFFF0B56A8
:10EF500003560356035603560356FFFFFFFFFFFFFA
:10EF6000FFFFFFFFFFFFF7FF03560356035603564D
:10EF700003561355FFFFE7BF0335035603560356E9
:10EF80000336E79FFFFFFFFF137603560356035632
:10EF900003560356EFBFFFFFFFFF0356035603560A
:10EFA000035603566D59FFFFFFFFFFFFFFFFFFFFF3
:10EFB000FFFFFFFFFFFFFFFFFFFFFFFFFFFFFFFF61
:10EFC000FFFFFFFFFFFFFFFFFFFFFFFFFFFFFFFF51
:10EFD000FFFFFFFFFFFFFFFFFFFF03360356035650
:10EFE0000356035603561355FFFFFFFFFFFFFFFFB6
:10EFF000FFFFFFFFFFFFFFFFFFFFFFFFFFFFFFFF21
:10F00000FFFFFFFF963C2C3924382418241823F8DE
:10F0100023F823F71BD71BB71BB71B971B971B7630
:10F020001B761B561B561B35133513354BF5FFFF4F
:10F03000FFFFFFFFFFFFFFFFFFFFFFFFFFFFFFFFE0
:10F04000FFFFFFFFFFFFFFFFFFFFFFFFFFFFFFDFF0
:10F05000A843B002A802A802A802A802A802A80217
:10F06000A802A002A002A002A002A002980198019A
:10F0700098019801980298019801900190019001DF
:10F080009001900188018801880188018801880128
:10F09000800180018001800180017800EDB7FFFFD1
:10F0A000FFFFFFFFFFFFFFFFFFFFFFFF44370336B8
:10F0B0000335035603360336033603360336033669
:10F0C000033603350335033603350336033603367B
:10F0D000033603360336033503550335033503354D
:10F0E0000335033503350335033503350335033560
:10F0F0000336FFFFFFFFFFFFFFFFC71F0336033687
:10F100000336033603360356FFFFFFFFFFFF2BB521
:10F1100003360336033603560356FFFFFFFF33F66D
:10F1200003360336033603360356FFFFFFFF95DB36
:10F1300003360336033603360336EFBFFFFFFFFF08
:10F14000FFFFFFFFFFFFF7FF0356033603360336CB
:10F1500003361355FFFF0B760336033603360336AB
:10F160000356FFFFEFDFF7DF1B7503360336035649
:10F1700003560356F7FFFFFFFFFF23D60336033680
:10F18000033603360336FFFFFFFFFFFFFFFFFFFFDE
:10F19000FFFFFFFFFFFFFFFF033603360336033693
:10F1A0000336033603360336033603360336033697
:10F1B0000336033603360336033503360336033688
:10F1C0000356035733F6FFFFFFFFFFFFFFFFFFFF6D
:10F1D000FFFFFFFFFFFFFFFFFFFFFFFFFFFFFFFF3F
:10F1E000FFFFFFFFE7BF2C382418241823F823F86B
:10F1F0001BD71BD71BB71B971B971B961B761B7622
:10F200001B561B351B351B351B158539FFFFFFFFB3
:10F21000FFFFFFFFFFFFFFFFFFFFFFFFFFFFFFFFFE
:10F22000FFFFFFFFFFFFFFFFFFFFFFFFFFFFA82321
:10F23000B002B002A802A802A802A802A802A8026E
:10F24000A002A002A002A002A002A00298019801C0
:10F250009801980198019801900190019001900106
:10F260009001900188018801880188018801880146
:10F2700080018001800180017001FF5DFFFFFFFFC1
:10F28000FFFFFFFFFFFFFFFFFFFFFFFF4C9803366D
:10F2900003360336033603360336033603160336C6
:10F2A00003360336033603360336031603360336B6
:10F2B0000336033603360336033603360336033686
:10F2C0000336033603360336033603360336033676
:10F2D0000B15FFFFFFFFFFFFFFFF0B350336033664
:10F2E0000336033603365498FFFFFFFFFFFFCF3F7F
:10F2F00003360336033603360336EFFFFFFFE7BF5F
:10F3000003160316033603360336B6DEFFFFFFFF90
:10F31000033603360336033603363C37FFFFFFFF61
:10F32000FFFFFFFFFFFFF7FF033603360336033609
:10F3300003361334FFFF0336033603360336033632
:10F3400085BBFFFF0316033603160336033603158A
:10F350000B14FFFFFFFFFFFFFFFFF7FF033603362E
:10F36000033603360335CF3FFFFFFFFFFFFFFFFFED
:10F37000FFFFFFFFFFFFFFFF0316033603360336D1
:10F3800003360336033603360336033603360336B5
:10F3900003360336033603360335033603360336A6
:10F3A0000335DF9FFFFFFFFFFFFFFFFFFFFFFFFFB3
:10F3B000FFFFFFFFFFFFFFFFFFFFFFFFFFFFFFFF5D
:10F3C000FFFFFFFFFFFF241823F823F823F71BD7C5
:10F3D0001BB71BB71B971B971B961B761B561B5601
:10F3E0001B351B351B151B151AF41AF4FFFFFFFF05
:10F3F000FFFFFFFFFFFFFFFFFFFFFFFFFFFFFFFF1D
:10F40000FFFFFFFFFFFFFFFFFFFFFFBFB022B002C4
:10F41000B002A802A802A802A802A802A802A80294
:10F42000A002A002A002A002A002A00198019801DF
:10F43000980198029801900190019001900190012B
:10F44000900190018801880188018801880180016C
:10F45000800180007801F6BBFFFFFFFFFFFFFFFF89
:10F46000FFFFFFFFFFFFFFFFFFFFFFFF54980315A4
:10F4700003150315031503150315031503150315CC
:10F4800003150315031503150315031503150315BC
:10F4900003150315031503150315031503150315AC
:10F4A000031503150315031503150315031503169B
:10F4B000F7FFFFFFFFFFFFFFFFFF03160315031515
:10F4C000031503150315F7FFFFFFFFFFFFFFFFFF06
:10F4D000031603150315031503164437FFFFFFFF3B
:10F4E000031503160315031503161335FFFFFFFF5E
:10F4F0000B150AF60B15031503150AF5FFFFFFFFA1
:10F50000FFFFFFFFFFFFF7FF0315031603150B16A1
:10F510002BD6FFFF4C5703160315031503160315CF
:10F52000FFFFFFFF0B150315031503160AF54438FB
:10F53000FFFFFFFFFFFFFFFFFFFFFFFF03150315A7
:10F540000315031503150AF4FFFFFFFFFFFFFFFF7D
:10F55000FFFFFFFFFFFFFFFF031603150315031552
:10F5600003150315031503150315031503150315DB
:10F5700003150315031503150316031603163BF7AE
:10F58000FFDEFFFFFFFFFFFFFFFFFFFFFFFFFFFFAC
:10F59000FFFFFFFFFFFFFFFFFFFFFFFFFFFFFFFF7B
:10F5A000FFFFFFFFFFFF33F623F71BD71BD71BB768
:10F5B0001BB71B971B961B761B561B561B561B35E2
:10F5C0001B351B151B151AF41AF41AD41AB3FFFFB6
:10F5D000FFFFFFFFFFFFFFFFFFFFFFFFFFFFFFFF3B
:10F5E000FFFFFFFFFFFFFFFFFFFFD3AFB002B0023F
:10F5F000B002A802A802A802A802A802A802A002BB
:10F60000A002A002A002A00298029801980198010D
:10F610009801980190019001900190019001900152
:10F62000900188018801880188018801800180019A
:10F630008001F659FFFFFFFFFFFFFFFFFFFFFFFF06
:10F64000FFFFFFFFFFFFFFFFFFFFFFFF54770B15DB
:10F650000B150B150B150B150B150B150B150B15AA
:10F660000B150B150B150B150B150B150B150B159A
:10F670000B150B150B150B150B150B150B150B158A
:10F680000B150B150B150B150B150AF50AF51B348D
:10F69000FFFFFFFFFFFFFFFF95DB0B160B150B15A1
:10F6A0000B150B150AF5FFFFFFFFFFFFFFFFFFFF25
:10F6B0000B150B150B150B150B150B15FFFFFFFF8E
:10F6C0000AF40AF50B150B150B150AF5FFFFFFFFE2
:10F6D0008D9A0B150AF60B150B150B15EFDFFFFFB7
:10F6E000FFFFFFFFFFFFF7FF0B150AF52355FFFF95
:10F6F000FFFFFFFF0B150AF50B150B150AF51AF4A2
:10F70000FFFFFFFF0AF50B150B150B15BEBEFFFF24
:10F71000FFFFFFFFFFFFFFFFFFFFFFFF7D7B0B15DD
:10F720000B150B150B150B15FFFFFFFFFFFFFFFF61
:10F73000FFFFFFFFFFFFFFFF0AF50B150B150B1572
:10F740000B150B150B150B150B150B150B150B15B9
:10F750000B150B150B150B150AF50B15DF7FFFFFAE
:10F76000FFFFFFFFFFFFFFFFFFFFFFFFFFFFFFFFA9
:10F77000FFFFFFFFFFFFFFFFFFFFFFFFFFFFFFFF99
:10F78000FFFFFFFFFFFFB6BE1BD71BD71BB71B97A3
:10F790001B971B761B761B561B561B351B351B35C3
:10F7A0001B151AF512F51AD41AD41AD41AB322B4A6
:10F7B000FFFFFFFFFFFFFFFFFFFFFFFFFFFFFFFF59
:10F7C000FFFFFFFFFFFFFFFFFFFFFFFFFFFFE4B3B0
:10F7D000A802A802A801A802A801A022A802A002CB
:10F7E000A002A002A002A00298019801980198012D
:10F7F0009801980190019001900190019001900171
:10F800008801900188018801800188008022F6BA71
:10F81000FFFFFFFFFFFFFFFF6BD61150FFFFFFFF52
:10F82000FFFFFFFFFFFFFFFFFFFFFFFF5C7712F40B
:10F830001AF412F412F41AF412F412F41AF412F480
:10F8400012F41AF412F412F41AF41AF412F41AF468
:10F850001AF412F41AF41AF412F41AF41AF412F450
:10F860001AF41AF412F41AF41AF41AF41AF3F7DF69
:10F87000FFFFFFFFFFFFFFFF2B543BD73BD63BD6DD
:10F880003BD63BD66CB9FFFFFFFFFFFFFFFFFFFF3B
:10F89000855964D964D964D964D96CB8FFFFFFFF76
:10F8A000AE3C6CB964D964D964D964D9FFFFFFFF59
:10F8B000FFFFCF1ECF1ECF1FCF1FCF1EEF9FFFFF1B
:10F8C000FFFFFFFFFFFFF7FF2B54FFFFFFFFFFFFCF
:10F8D000FFFFEFFF12F512F512F512F512F5E77FB3
:10F8E000FFFFFFFF0AF512F512F5F7FFFFFFFFFF1D
:10F8F000FFFFFFFFFFFFFFFFFFFFFFFFFFFF0AD537
:10F9000012F512F512F512F5855AFFFFFFFFFFFF02
:10F91000FFFFFFFFFFFFFFFF1AF412F412D412F4EF
:10F9200012D412F412F412D412F412F412D412F407
:10F9300012F412D412F412F41AF4FFFFFFFFFFFFC7
:10F94000FFFFFFFFFFFFFFFFFFFFFFFFFFFFFFFFC7
:10F95000FFFFFFFFFFFFFFFFFFFFFFFFFFFFFFFFB7
:10F96000FFFFFFFFFFFFFFFF1BB71BB71B971B9797
:10F970001B761B761B561B561B351B351B151B1583
:10F980001AF51AF523141AD51AB41AB41AB31A941C
:10F990001A748D5AFFFFFFFFFFFFFFFFFFFFFFFFFE
:10F9A000FFFFFFFFFFFFFFFFFFFFFFFFFFFFFFFF67
:10F9B000FFFFFFFFDC52A083A801A802A002A00263
:10F9C000A002A002A0029802980198019801980153
:10F9D0009801900190019001900190019001900197
:10F9E00088018801880188A3EE38FFFFFFFFFFFF31
:10F9F000FFFFFFFFFFFF114F0970FFFFFFFFFFFF3A
:10FA0000FFFFFFFFFFFFFFFFFFFFFFFFFFFFFFFF06
:10FA1000FFFFFFFFFFFFFFFFFFFFFFFFFFFFFFFFF6
:10FA2000FFFFFFFFFFFFFFFFFFFFFFFFFFFFFFFFE6
:10FA3000FFFFFFFFFFFFFFFFFFFFFFFFFFFFFFFFD6
:10FA4000FFFFFFFFFFFFFFFFFFFFFFFFFFFFFFFFC6
:10FA5000FFFFFFFFFFFFFFFFFFFFFFFFFFFFFFFFB6
:10FA6000FFFFFFFFFFFFFFFFFFFFFFFFFFFFFFFFA6
:10FA7000FFFFFFFFFFFFFFFFFFFFFFFFFFFFFFFF96
:10FA8000FFFFFFFFFFFFFFFFFFFFFFFFFFFFFFFF86
:10FA9000FFFFFFFFFFFFFFFFFFFFFFFFFFFFFFFF76
:10FAA000FFFFFFFFFFFFFFFFFFFFFFFFFFFFFFFF66
:10FAB000FFFFFFFFFFFFFFFFFFFFFFFFFFFFFFFF56
:10FAC000FFFFFFFFFFFFFFFFFFFFFFFFFFFFFFFF46
:10FAD000FFFFFFFFFFFFFFFFFFFFFFFFFFFFFFFF36
:10FAE000FFFFFFFFFFFFFFFFFFFFFFFFFFFFFFFF26
:10FAF000FFFFFFFFFFFFFFFFFFFFFFFFFFFFFFFF16
:10FB0000FFFFFFFFFFFFFFFFFFFFFFFFFFFFFFFF05
:10FB1000FFFFFFFFFFFFFFFFFFFFFFFFFFFFFFFFF5
:10FB2000FFFFFFFFFFFFFFFFFFFFFFFFFFFFFFFFE5
:10FB3000FFFFFFFFFFFFFFFFFFFFFFFFFFFFFFFFD5
:10FB4000FFFFFFFFFFFFFFFF13961B971B761B7640
:10FB50001B561B561B351B351B351B151AF51AF486
:10FB60001AF48D7AFFFF1AB31A931A931A731A7341
:10FB70001A531A532252FFFFFFFFFFFFFFFFFFFF41
:10FB8000FFFFFFFFFFFFFFFFFFFFFFFFFFFFFFFF85
:10FB9000FFFFFFFFFFFFFFFFFFFFFF5DCBAFA06396
:10FBA000A002A001A0019802980298029802980170
:10FBB0009002900290029001900188019001884289
:10FBC000BBAFFF9EFFFFFFFFFFFFFFFFFFFFFFFF3A
:10FBD000FFFFBE1D1171115142D3FFFFFFFFFFFF59
:10FBE000FFFFFFFFFFFFFFFFFFFFFFFFFFFFFFFF25
:10FBF000FFFFFFFFFFFFFFFFFFFFFFFFFFFFFFFF15
:10FC0000FFFFFFFFFFFFFFFFFFFFFFFFFFFFFFFF04
:10FC1000FFFFFFFFFFFFFFFFFFFFFFFFFFFFFFFFF4
:10FC2000FFFFFFFFFFFFFFFFFFFFFFFFFFFFFFFFE4
:10FC3000FFFFFFFFFFFFFFFFFFFFFFFFFFFFFFFFD4
:10FC4000FFFFFFFFFFFFFFFFFFFFFFFFFFFFFFFFC4
:10FC5000FFFFFFFFFFFFFFFFFFFFFFFFFFFFFFFFB4
:10FC6000FFFFFFFFFFFFFFFFFFFFFFFFFFFFFFFFA4
:10FC7000FFFFFFFFFFFFFFFFFFFFFFFFFFFFFFFF94
:10FC8000FFFFFFFFFFFFFFFFFFFFFFFFFFFFFFFF84
:10FC9000FFFFFFFFFFFFFFFFFFFFFFFFFFFFFFFF74
:10FCA000FFFFFFFFFFFFFFFFFFFFFFFFFFFFFFFF64
:10FCB000FFFFFFFFFFFFFFFFFFFFFFFFFFFFFFFF54
:10FCC000FFFFFFFFFFFFFFFFFFFFFFFFFFFFFFFF44
:10FCD000FFFFFFFFFFFFFFFFFFFFFFFFFFFFFFFF34
:10FCE000FFFFFFFFFFFFFFFFFFFFFFFFFFFFFFFF24
:10FCF000FFFFFFFFFFFFFFFFFFFFFFFFFFFFFFFF14
:10FD0000FFFFFFFFFFFFFFFFFFFFFFFFFFFFFFFF03
:10FD1000FFFFFFFFFFFFFFFFFFFFFFFFFFFFFFFFF3
:10FD2000FFFFFFFFFFFFFFFFC6FE1B761B761B5684
:10FD30001B561B351B351B151B151AF51AF41AF526
:10FD4000BE9DFFFFFFFFFFFF3B131A731A731A5389
:10FD50001A531A331A3312338CF9FFFFFFFFFFFFD8
:10FD6000FFFFFFFFFFFFFFFFFFFFFFFFFFFFFFFFA3
:10FD7000FFFFFFFFFFFFFFFFFFFFFFFFFFFFFFFF93
:10FD8000FFFFFFFFFFFFFFFFFFDEF6BAFE9AE576FB
:10FD9000DD96F69AFF9EFFDFFFFFFFFFFFFFFFFFED
:10FDA000FFFFFFFFFFFFFFFFFFFFFFFFFFFFFFDF83
:10FDB0001950117011511152FFFFFFFFFFFFFFFF9C
:10FDC000FFFFFFFFFFFFFFFFFFFFFFFFFFFFFFFF43
:10FDD000FFFFFFFFFFFFFFFFFFFFFFFFFFFFFFFF33
:10FDE000FFFFFFFFFFFFFFFFFFFFFFFFFFFFFFFF23
:10FDF000FFFFFFFFFFFFFFFFFFFFFFFFFFFFFFFF13
:10FE0000FFFFFFFFFFFFFFFFFFFFFFFFFFFFFFFF02
:10FE1000FFFFFFFFFFFFFFFFFFFFFFFFFFFFFFFFF2
:10FE2000FFFFFFFFFFFFFFFFFFFFFFFFFFFFFFFFE2
:10FE3000FFFFFFFFFFFFFFFFFFFFFFFFFFFFFFFFD2
:10FE4000FFFFFFFFFFFFFFFFFFFFFFFFFFFFFFFFC2
:10FE5000FFFFFFFFFFFFFFFFFFFFFFFFFFFFFFFFB2
:10FE6000FFFFFFFFFFFFFFFFFFFFFFFFFFFFFFFFA2
:10FE7000FFFFFFFFFFFFFFFFFFFFFFFFFFFFFFFF92
:10FE8000FFFFFFFFFFFFFFFFFFFFFFFFFFFFFFFF82
:10FE9000FFFFFFFFFFFFFFFFFFFFFFFFFFFFFFFF72
:10FEA000FFFFFFFFFFFFFFFFFFFFFFFFFFFFFFFF62
:10FEB000FFFFFFFFFFFFFFFFFFFFFFFFFFFFFFFF52
:10FEC000FFFFFFFFFFFFFFFFFFFFFFFFFFFFFFFF42
:10FED000FFFFFFFFFFFFFFFFFFFFFFFFFFFFFFFF32
:10FEE000FFFFFFFFFFFFFFFFFFFFFFFFFFFFFFFF22
:10FEF000FFFFFFFFFFFFFFFFFFFFFFFFFFFFFFFF12
:10FF0000FFFFFFFFFFFFFFFFFFFF1B761B561B35A9
:10FF10001B351B351B151B151AF51AF51AF57CD860
:10FF2000FFFFFFFFFFFFFFFFFFFF2A931A521A5345
:10FF30001A321A331A12121219F211F2EFBFFFFF1E
:10FF4000FFFFFFFFFFFFFFFFFFFFFFFFFFFFFFFFC1
:10FF5000FFFFFFFFFFFFFFFFFFFFFFFFFFFFFFFFB1
:10FF6000FFFFFFFFFFFFFFFFFFFFFFFFFFFFFFFFA1
:10FF7000FFFFFFFFFFFFFFFFFFFFFFFFFFFFFFFF91
:10FF8000FFFFFFFFFFFFFFFFFFFFFFFF3A5211518F
:10FF9000117011501150EF5FFFFFFFFFFFFFFFFFD8
:10FFA000FFFFFFFFFFFFFFFFFFFFFFFFFFFFFFFF61
:10FFB000FFFFFFFFFFFFFFFFFFFFFFFFFFFFFFFF51
:10FFC000FFFFFFFFFFFFFFFFFFFFFFFFFFFFFFFF41
:10FFD000FFFFFFFFFFFFFFFFFFFFFFFFFFFFFFFF31
:10FFE000FFFFFFFFFFFFFFFFFFFFFFFFFFFFFFFF21
:10FFF000FFFFFFFFFFFFFFFFFFFFFFFFFFFFFFFF11
:020000040801F1
:10000000FFFFFFFFFFFFFFFFFFFFFFFFFFFFFFFF00
:10001000FFFFFFFFFFFFFFFFFFFFFFFFFFFFFFFFF0
:10002000FFFFFFFFFFFFFFFFFFFFFFFFFFFFFFFFE0
:10003000FFFFFFFFFFFFFFFFFFFFFFFFFFFFFFFFD0
:10004000FFFFFFFFFFFFFFFFFFFFFFFFFFFFFFFFC0
:10005000FFFFFFFFFFFFFFFFFFFFFFFFFFFFFFFFB0
:10006000FFFFFFFFFFFFFFFFFFFFFFFFFFFFFFFFA0
:10007000FFFFFFFFFFFFFFFFFFFFFFFFFFFFFFFF90
:10008000FFFFFFFFFFFFFFFFFFFFFFFFFFFFFFFF80
:10009000FFFFFFFFFFFFFFFFFFFFFFFFFFFFFFFF70
:1000A000FFFFFFFFFFFFFFFFFFFFFFFFFFFFFFFF60
:1000B000FFFFFFFFFFFFFFFFFFFFFFFFFFFFFFFF50
:1000C000FFFFFFFFFFFFFFFFFFFFFFFFFFFFFFFF40
:1000D000FFFFFFFFFFFFFFFFFFFFFFFFFFFFFFFF30
:1000E000FFFFFFFFFFFFFFFFFFFF8DBB1B351B3532
:1000F0001B151B151AF51AF51AD41AF474B7FFFF5D
:10010000FFFFFFFFFFFFFFFFFFFFFFFF64151A5216
:100110001A12121211F211F211F111D211B111B021
:10012000EFBFFFFFFFFFFFFFFFFFFFFFFFFFFFFF2F
:10013000FFFFFFFFFFFFFFFFFFFFFFFFFFFFFFFFCF
:10014000FFFFFFFFFFFFFFFFFFFFFFFFFFFFFFFFBF
:10015000FFFFFFFFFFFFFFFFFFFFFFFFFFFFFFFFAF
:10016000FFFFFFFFFFFFFFFF63941151115011517B
:1001700011510970ADBAFFFFFFFFFFFFFFFFFFFF47
:10018000FFFFFFFFFFFFFFFFFFFFFFFFFFFFFFFF7F
:10019000FFFFF7FF551A54FA5519551954F9551917
:1001A000551954F9551A54D85CD7FFFFFFFFFFFFCC
:1001B000FFFF64D854F95D1A54FA54F954F95519EB
:1001C00054F954F9551954F9551AFFFFFFFFFFFF71
:1001D000FFFFFFFFFFFFFFFFE7DF54F95519551938
:1001E00054F95519551954F9551954FA5CF9551A19
:1001F000FFFF54F954F9551954F954F9551954F9A4
:1002000054F9551954F954F9551954F954F9551923
:1002100054F954F954FAFFFFFFFF4CF94D1954F902
:100220005519551954F94D1A4CFAF7FFFFFF5CF8B0
:1002300054F95519551954F955195519551A551A8E
:100240004CF95CF95519551954F954F9551954F9E3
:1002500054F9551954F954F9551954F954F954F9F4
:100260005519FFFF553B551954F9551954F954F9CF
:100270005519551954F95519551954F95519551950
:1002800054F95519551954F9FFFFFFFF55194CF949
:10029000551954F95519551954F954F954F954F993
:1002A000F7FF54F954F954F9551954F954F95519FB
:1002B00054F954F954F9FFFFFFFFFFFFFFFFFFFF61
:1002C000FFFFFFFFFFFFFFFFFFFFFFFF1B351B15BA
:1002D0001AF51AF41AD41AD41AD4ADDCFFFFFFFFB2
:1002E000FFFFFFFFFFFFFFFFFFFFFFFFFFFFFFFF1E
:1002F00011F211F211F211D211D211B209B1119110
:100300001171117184B9FFFFFFFFFFFFFFFFFFFFB6
:10031000FFFFFFFFFFFFFFFFFFFFFFFFFFFFFFFFED
:10032000FFFFFFFFFFFFFFFFFFFFFFFFFFFFFFFFDD
:10033000FFFFFFFFFFFFFFFFFFFFFFFFFFFFFFFFCD
:10034000FFFFD6FE194F1151115111511151115189
:100350001151E71EFFFFFFFFFFFFFFFFFFFFFFFF42
:10036000FFFFFFFFFFFFFFFFFFFFFFFFFFFFFFFF9D
:10037000FFFFFFFFFFFF03B703D703D803B803B89E
:1003800003B803B803F9EFFFFFFFFFFFFFFFFFFF15
:10039000FFFFFFFFFFFF03B603D803B803B803B89E
:1003A00003B803B803D8EFFFFFFFFFFFFFFFFFFF16
:1003B000FFFFFFFFFFFFFFFFFFFFFFFF33D403D966
:1003C00003B803B803D803D803B803D8E7FFFFFF87
:1003D000FFFFFFFFEFFF03B703D803B803B803B86D
:1003E00003B803D803B803B803B803D803B703D9D5
:1003F00003B703D803D7F7FFFFFFFFFFCFBF03D833
:1004000003D803B803B803B803B803D91395FFFFA3
:10041000FFFF139603B803B703D803B803D8EFFF61
:10042000FFFF0BB703B703B803B803D803D703B86C
:1004300003B803B803B803D903B703B803B803D8A4
:1004400003B8FFFFFFFFE7FF03B8039803B803B843
:1004500003D803B803B803B803B803B803B803B8A4
:1004600003D803B803D803D8FFFFFFFFFFFFDFFF68
:1004700003B803D803B803B803B803B803B7F7FF4A
:10048000FFFFFFFF23B503B803B703B803D803D8B2
:1004900003B7F7FFFFFFFFFFFFFFFFFFFFFFFFFFB8
:1004A000FFFFFFFFFFFFFFFFFFFFFFFFB69D1AF5F6
:1004B0001AF41AD41AD41AB422B4FFFFFFFFFFFFB4
:1004C000FFFFFFFFFFFFFFFFFFFFFFFFFFFFFFFF3C
:1004D000FFFF329409F111D109B1119111911191DC
:1004E0001171117111501150114FAD9BFFFFFFFFA2
:1004F000FFFFFFFFFFFFFFFFFFFFFFFFFFFFFFFF0C
:10050000FFFFFFFFFFFFFFFFFFFFFFFFFFFFFFFFFB
:10051000FFFFFFFFFFFFFFFFFFFFFFFFEF7F5B75A9
:10052000117011701170115111511151117011513F
:10053000DF1FFFFFDF1DFFFFFFFFFFFFFFFFFFFFCD
:10054000FFFFFFFFFFFFFFFFFFFFFFFFFFFFFFFFBB
:10055000FFFFFFFFFFFF03B703B703B703B803D8DD
:1005600003B803B803D8FFFFFFFFFFFFFFFFFFFF44
:10057000FFFFFFFFFFFFFFFFEFFF03B803B803B864
:1005800003B80B75FFFFFFFFFFFFFFFFFFFFFFFF3C
:10059000FFFFFFFFFFFFFFFFFFFFFFFFFFFFFFFF6B
:1005A00003D803B803B803D803B7FFFFFFFFFFFF6B
:1005B000FFFFFFFFFFFFFFFF0BB703D803B803B830
:1005C00003B8FFFFFFFFFFFFFFFFFFFFEFFFFFFF8E
:1005D000EFFF03B803B8F7FFFFFFFFFFFFFFFFFFC9
:1005E00003D803B803B803B803B803D803D803B8D3
:1005F000FFFFFFFFF7FF03B703D713B5FFFFFFFFB1
:10060000FFFF03D803B70B96FFFFFFFFEFFF03B811
:1006100003B803B803B81B74FFFFFFFF33F503B83B
:1006200003B9FFFFFFFFFFFFFFFF03D703B803B8C6
:1006300003B803B8FFFFFFFFFFFFFFFFFFFFF7FF58
:10064000FFFFF7FF03D803D8FFFFFFFFFFFFFFFF08
:10065000FFFF03B803B803B803B803B8FFFFFFFFF9
:10066000FFFFF7FF0BB603B703B903B80B96FFFF05
:10067000FFFFFFFFFFFFFFFFFFFFFFFFFFFFFFFF8A
:10068000FFFFFFFFFFFFFFFFFFFFFFFFFFFF12F571
:100690001AD41AD41AB41AB41A931A94FFFFFFFF8B
:1006A000FFFFFFFFFFFFFFFFFFFFFFFFFFFFFFFF5A
:1006B000FFFFFFFFF7FF119109910991117111716E
:1006C00011501151115011501151115111710971E5
:1006D00019708457D6FEFFFFFFFFFFFFFFFFFFFFEC
:1006E000FFFFFFFFFFFFFFFFFFFFFFFFFFFFFFFF1A
:1006F000FFFFFFFFB5DB4292115011511151115113
:100700001150115111501151115111513211FFFF5E
:10071000FFFF21B0FFFFFFFFFFFFFFFFFFFFFFFF16
:10072000FFFFFFFFFFFFFFFFFFFFFFFFFFFFFFFFD9
:10073000FFFFFFFF039803D803B88E3DEFFF03D7F9
:1007400003B803B803D803B8FFFFFFFFFFFFFFFFA5
:10075000FFFFFFFFFFFFFFFFF7FF03B803B803B87A
:1007600003B81396FFFFFFFFFFFFFFFFFFFFFFFF31
:10077000FFFFFFFFFFFFFFFFFFFFFFFFFFFFFFFF89
:1007800003D803B803B803B803B7FFFFFFFFFFFFA9
:10079000FFFFFFFFFFFFFFFF0B9603B803B803B88F
:1007A00003B803D803B803B803B803B803D8EFFFFE
:1007B000FFFFFFFFE7FFF7FFFFFFFFFFFFFFFFFF69
:1007C00003D803B803B803D803B803D803B803B8F1
:1007D00003D82BB5F7FF03D803D71395FFFFFFFF0F
:1007E000FFFF03B8F7FFFFFFFFFFFFFFEFFF03B8B7
:1007F00003B803B803B81B74FFFFFFFFFFFFFFFF41
:100800001396F7FFFFFFFFFFFFFF03B903B803B81D
:1008100003D803B803B803B803D803B9039703B8E0
:10082000EFFFFFFFFFFFDFFFFFFFFFFFFFFFFFFF08
:10083000FFFF03B803B803B803B803B8FFFF44567B
:1008400003D803B803D803B803B8BF5FFFFFFFFFA7
:10085000FFFFFFFFFFFFFFFFFFFFFFFFFFFFFFFFA8
:10086000FFFFFFFFFFFFFFFFFFFFFFFFFFFFE79F10
:100870001AD51AB41A941A931A731A531A53FFFFFB
:10088000FFFFFFFFFFFFFFFFFFFFFFFFFFFFFFFF78
:10089000FFFFFFFFFFFFFFFF9D3911711170115125
:1008A0001170115111511151115111511151115119
:1008B0001151115111511170117111511170114FCC
:1008C000114F325232523252114F11701150117079
:1008D000115011511130117111511151115111510A
:1008E00011511151115111511151D6FEFFDFFFFF6E
:1008F0004AB3CE9DFFFFFFFFFFFFFFFFFFFFFFFF9C
:10090000FFFFFFFFFFFFFFFFFFFFFFFFFFFFFFFFF7
:10091000FFFF441503B903B803B7E7FFE7FFC7FFBD
:1009200003B803B803B803B803D8FFFFFFFFFFFF06
:10093000FFFFFFFFFFFFFFFFF7FF03B803B803B898
:1009400003B81395FFFFFFFFFFFFFFFFFFFFFFFF50
:10095000FFFFFFFF23F623D6FFFFFFFFFFFFFFFF91
:1009600003B803B803B803D803B7FFFFFFFFFFFFC7
:10097000FFFFFFFFFFFFFFFF0BB703B803B803B88C
:1009800003B703B803D803D803D703D803D8EFFFBE
:10099000FFFFFFFFFFFF33D3FFFFFFFFFFFFFFFF5F
:1009A00003D803B803D8F7FF03D803B803B803B8D4
:1009B00003B803B803B703D803D81395FFFFFFFFAD
:1009C000FFDEFFFFFFFFFFFFFFFFFFFFEFFF03B8AB
:1009D00003B803B803B82373FFFFFFFFFFFFFFFF58
:1009E000FFFFFFFFFFFFFFFFFFFF03B803B803B8E0
:1009F00003B703D803D803D803D803B803D803D860
:100A0000EFFFFFFFFFFFFFFF2BB4FFFFFFFFFFFF25
:100A1000FFFF03B803B803B803B803B803D803B89B
:100A200003B703B803D803B803B803D8E7FFFFFF41
:100A3000FFFFFFFFFFFFFFFFFFFFFFFFFFFFFFFFC6
:100A4000FFFFFFFFFFFFFFFFFFFFFFFFFFFFFFFFB6
:100A50004B951A941A941A731A731A531A321A323B
:100A6000FFFFFFFFFFFFFFFFFFFFFFFFFFFFFFFF96
:100A7000FFFFFFFFFFFFFFFFFFFFFFFF6395115128
:100A80001151115111511151115111511151115156
:100A90001151115111511151115111501170117009
:100AA0001151115111511151115011511151115137
:100AB0001150115111511151115111511151115127
:100AC000115111501151B5FBFFFFFFFFFFFF29F13D
:100AD000114FFFFFFFFFFFFFFFFFFFFFFFFFFFFFC4
:100AE000FFFFFFFFFFFFFFFFFFFFFFFFFFFFFFFF16
:100AF000C79F03D803B803B803B803D803B803B833
:100B000003B803B803B803B803D81B54FFFFFFFFB3
:100B1000FFFFFFFFFFFFFFFFF7FF03B803B803B8B6
:100B200003B81395FFFFFFFFFFFFFFFFFFFFFFFF6E
:100B3000F7FF03D803B723D6FFFFFFFFFFFFFFFF39
:100B400003B803B803B803D803B7FFFFFFFFFFFFE5
:100B5000FFFFFFFFFFFFFFFF0BB703B803B803B8AA
:100B600003B8FFFFFFFFFFFFFFFFF7FF0BB7EFFF2C
:100B7000FFFF0B9603F92BB4FFFFFFFFFFFFFFFF03
:100B800003D803B803D8FFFFFFFF039703B803B8E8
:100B900003B803B803B803D703D81395FFFFFFFFCB
:100BA000FFFFFFFFFFFFFFFFFFFFFFFFEFFF03B8A8
:100BB00003B803B803B82373FFFFFFFFFFFFFFFF76
:100BC000FFFFFFFFFFFFFFFFFFFF03B803B803B8FE
:100BD00003B803B8FFFFFFFFFFFFFFFFFFFF0BB6E8
:100BE000EFFFFFFF0BB6039723D5FFFFFFFFFFFFCC
:100BF000FFFF03B803B803B803B803B803B82C1752
:100C0000FFFFFFFF239403B703B703B803B7B73F52
:100C1000FFFFFFFFFFFFFFFFFFFFFFFFFFFFFFFFE4
:100C2000FFFFFFFFFFFFFFFFFFFFFFFFFFFFFFFFD4
:100C3000FFFF22731A731A531A531A331A321A12F5
:100C400009F1FFFFFFFFFFFFFFFFFFFFFFFFFFFFB8
:100C5000FFFFFFFFFFFFFFFFFFFFFFFFFFFFFFFFA4
:100C6000E73E1150115011511150115111511151B4
:100C70001151115111511151115111511151115164
:100C80001151115111511151115111511151115154
:100C90001151115111511170115111511150117106
:100CA0006395FFFFFFFFFFFFFFFFFFFF1150114F95
:100CB000FFFFFFFFFFFFFFFFFFFFFFFFFFFFFFFF44
:100CC000FFFFFFFFFFFFFFFFFFFFFFFFFFFF0B9592
:100CD00003D803B803B86D39FFFFFFFFFFFFFFFF25
:100CE000F7FF03D803B803B803D703B703D8F7FF58
:100CF000FFFFFFFFFFFFF7FF03B703B803B803B819
:100D000003B80BB80BB70B960B970BB70BB603B822
:100D100003B703D803B823D6FFFFFFFFFFFF0BB6CF
:100D200003B803B803B803D803B8C77FFFFFFFFFBA
:100D3000FFFFFFFFFFFF95FC03B703B803B803B83D
:100D400003B80BB70B970B970B970B970BB60BB81A
:100D500003D803B803D82BB4FFFFFFFFFFFF3436DF
:100D600003B703D803961375FFFFFFFFDFFF03B838
:100D700003B803B803B803B803D81395FFFFFFFF08
:100D8000FFFFFFFFFFFFFFFFFFFFF7FF03B803B801
:100D900003B803B803B80397E7FFFFFFFFFFFFFFA8
:100DA000FFFFFFFFFFFFFFFF8DFB03F803B803B852
:100DB00003D803D80B960B970B970B970B970BB693
:100DC0000B970BD803B803D823D5FFFFFFFFFFFF16
:100DD0003BF503D903B803B803B803B82BF5FFFFFD
:100DE000FFFFFFFFFFFF03D803D803B803B803D802
:100DF00003D8FFFFFFFFFFFFFFFFFFFFFFFFFFFF26
:100E0000FFFFFFFFFFFFFFFFFFFFFFFFFFFFFFFFF2
:100E1000FFFFFFFF1A331A531A331A331A121A122A
:100E20001A1311F2CEDEFFFFFFFFFFFFFFFFFFFFF0
:100E3000FFFFFFFFFFFFFFFFFFFFFFFFFFFFFFFFC2
:100E4000FFFFFFFFFFFF84B71150117011511151C7
:100E50001151115111511151115111511151115182
:100E60001151115111511151115111511151115172
:100E70001151115111511171115073F6FFFFFFFF04
:100E8000FFFFFFFFFFFFFFFFDF1E11511171FFFF8B
:100E9000FFFFFFFFFFFFFFFFFFFFFFFFFFFFFFFF62
:100EA000FFFFFFFFFFFFFFFFFFFFFFFF03B803B8D8
:100EB00003B803B803B8039703D8EFFFF7FF03B7EE
:100EC00003B803B803B803B803D803B803D803B80A
:100ED0000BB6FFFF0B9603B803B803B803B803B80B
:100EE00003B803B703B803B803B803B803B803B82B
:100EF00003D803B703B823D6FFFF1BB503D803D825
:100F000003B803B803B803B803B803B80BB7CFFFEF
:100F1000FFFFE7FF03D903D703D803B803B803B82B
:100F200003B803D803B803B803B803B803B803B9C8
:100F300003D803D803B82BB4FFFFAEFF03B703B841
:100F400003D803B803B803B803D84478FFFFF7FF0A
:100F500003D903D803B803B803D81395FFFFFFFFE5
:100F6000FFFFFFFFFFFFFFFF0BB603B803D803B877
:100F700003B803B803B803B803D70397F7FFFFFF1D
:100F8000FFFFFFFFE7FF03B703D703D803B803B89A
:100F900003B803D703B803B803B803B803B803B85A
:100FA00003B803B803D703D823D5FFFFAF3F03B877
:100FB00003D903B803B803B803B803B803B803D818
:100FC000FFFF1B9403B703D803B803B803B803B8F3
:100FD00003B703D81B94FFFFFFFFFFFFFFFFFFFFD7
:100FE000FFFFFFFFFFFFFFFFFFFFFFFFFFFFFFFF11
:100FF000FFFFFFFFDF5F1A3212321A12121211F2D4
:1010000011F209D211B23272FFFFFFFFFFFFFFFFA3
:10101000FFFFFFFFFFFFFFFFFFFFFFFFFFFFFFFFE0
:10102000FFFFFFFFFFFFFFFFFFFFFFFFF7BF8CD8B2
:101030003232115011511170117111701151115141
:10104000115111511151115111501150115119706B
:101050005B75CEBEFFFFFFFFFFFFFFFFFFFFFFFF40
:10106000FFFFFFFFFFFF197011711150F7DFFFFF46
:10107000FFFFFFFFFFFFFFFFFFFFFFFFFFFFFFFF80
:10108000FFFFFFFFFFFFFFFFFFFFFFFFFFFFFFFF70
:10109000FFFFFFFFFFFFFFFFFFFFFFFFFFFFFFFF60
:1010A000FFFFFFFFFFFFFFFFFFFFFFFFFFFFFFFF50
:1010B000FFFFFFFFFFFFFFFFFFFFFFFFFFFFFFFF40
:1010C000FFFFFFFFFFFFFFFFFFFFFFFFFFFFFFFF30
:1010D000FFFFFFFFFFFFFFFFF7DFFFFFFFFFFFFF48
:1010E000FFFFFFFFFFFFFFFFFFFFFFFFFFFFFFFF10
:1010F000FFFFFFFFFFFFFFFFFFFFFFFFFFFFFFFF00
:10110000FFFFFFFFFFFFFFFFFFFFFFFFFFFFFFFFEF
:10111000FFFFFFFFFFFFFFFFFFFFFFFFFFFFFFFFDF
:10112000FFFFFFFFFFFFFFFFFFFFFFFFFFFFFFFFCF
:10113000FFFFFFFFFFFFFFFFFFFFFFFFFFFFFFFFBF
:10114000FFFFFFFFFFFFFFFFFFFFFFFFFFFFFFFFAF
:10115000FFFFFFFFFFFFFFFFFFFFFFFFFFFFFFFF9F
:10116000FFFFFFFFFFFFFFFFFFFFFFFFFFFFFFFF8F
:10117000FFFFFFFFFFFFFFFFFFFFFFFFFFFFFFFF7F
:10118000FFFFFFFFFFFFFFFFFFFFFFFFFFFFFFFF6F
:10119000FFFFFFFFFFFFFFFFFFFFFFFFFFFFFFFF5F
:1011A000FFFFFFFFFFFFFFFFFFFFFFFFFFFFFFFF4F
:1011B000FFFFFFFFFFFFFFFFFFFFFFFFFFFFFFFF3F
:1011C000FFFFFFFFFFFFFFFFFFFFFFFFFFFFFFFF2F
:1011D000FFFFFFFFFFFF9D9B121211F211F211D2D0
:1011E00011D211B109B211911171E73FFFFFFFFF59
:1011F000FFFFFFFFFFFFFFFFFFFFFFFFFFFFFFFFFF
:10120000FFFFFFFFFFFFFFFFFFFFFFFFFFFFFFFFEE
:10121000FFFFFFFFFFFFFFFFF7DFEF5FCEBDCE9DBC
:10122000CE9DCE9DE75FF7DFFFFFFFFFFFFFFFFFD4
:10123000FFFFFFFFFFFFFFFFFFFFFFFFFFFFFFFFBE
:10124000FFFFC65C11711150115084B7FFFFFFFF03
:10125000FFFFFFFFFFFFFFFFFFFFFFFFFFFFFFFF9E
:10126000FFFFFFFFFFFFFFFFFFFFFFFFFFFFFFFF8E
:10127000FFFFFFFFFFFFFFFFFFFFFFFFFFFFFFFF7E
:10128000FFFFFFFFFFFFFFFFFFFFFFFFFFFFFFFF6E
:10129000FFFFFFFFFFFFFFFFFFFFFFFFFFFFFFFF5E
:1012A000FFFFFFFFFFFFFFFFFFFFFFFFFFFFFFFF4E
:1012B000FFFFFFFFFFFFFFFFFFFFFFFFFFFFFFFF3E
:1012C000FFFFFFFFFFFFFFFFFFFFFFFFFFFFFFFF2E
:1012D000FFFFFFFFFFFFFFFFFFFFFFFFFFFFFFFF1E
:1012E000FFFFFFFFFFFFFFFFFFFFFFFFFFFFFFFF0E
:1012F000FFFFFFFFFFFFFFFFFFFFFFFFFFFFFFFFFE
:10130000FFFFFFFFFFFFFFFFFFFFFFFFFFFFFFFFED
:10131000FFFFFFFFFFFFFFFFFFFFFFFFFFFFFFFFDD
:10132000FFFFFFFFFFFFFFFFFFFFFFFFFFFFFFFFCD
:10133000FFFFFFFFFFFFFFFFFFFFFFFFFFFFFFFFBD
:10134000FFFFFFFFFFFFFFFFFFFFFFFFFFFFFFFFAD
:10135000FFFFFFFFFFFFFFFFFFFFFFFFFFFFFFFF9D
:10136000FFFFFFFFFFFFFFFFFFFFFFFFFFFFFFFF8D
:10137000FFFFFFFFFFFFFFFFFFFFFFFFFFFFFFFF7D
:10138000FFFFFFFFFFFFFFFFFFFFFFFFFFFFFFFF6D
:10139000FFFFFFFFFFFFFFFFFFFFFFFFFFFFFFFF5D
:1013A000FFFFFFFFFFFFFFFFFFFFFFFFFFFFFFFF4D
:1013B000FFFFFFFFFFFFFFFF745711F111F211D282
:1013C00009B109B10991119111711171114FF7DF33
:1013D000FFFFFFFFFFFFFFFFFFFFFFFFFFFFFFFF1D
:1013E000FFFFFFFFFFFFFFFFFFFFFFFFFFFFFFFF0D
:1013F000FFFFFFFFFFFFFFFFFFFFFFFFFFFFFFFFFD
:10140000FFFFFFFFFFFFFFFFFFFFFFFFFFFFFFFFEC
:10141000FFFFFFFFFFFFFFFFFFFFFFFFFFFFFFFFDC
:10142000112F1151117011515334FFFFFFFFFFFFB6
:10143000FFFFFFFFFFFFFFFFFFFFFFFFFFFFFFFFBC
:10144000FFFFFFFFFFFFFFFFFFFFFFFFFFFFFFFFAC
:10145000FFFFFFFFFFFFFFFFFFFFFFFFFFFFFFFF9C
:10146000FFFFFFFFFFFFFFFFFFFFFFFFFFFFFFFF8C
:10147000FFFFFFFFFFFFFFFFFFFFFFFFFFFFFFFF7C
:10148000FFFFFFFFFFFFFFFFFFFFFFFFFFFFFFFF6C
:10149000FFFFFFFFFFFFFFFFFFFFFFFFFFFFFFFF5C
:1014A000FFFFFFFFFFFFFFFFFFFFFFFFFFFFFFFF4C
:1014B000FFFFFFFFFFFFFFFFFFFFFFFFFFFFFFFF3C
:1014C000FFFFFFFFFFFFFFFFFFFFFFFFFFFFFFFF2C
:1014D000FFFFFFFFFFFFFFFFFFFFFFFFFFFFFFFF1C
:1014E000FFFFFFFFFFFFFFFFFFFFFFFFFFFFFFFF0C
:1014F000FFFFFFFFFFFFFFFFFFFFFFFFFFFFFFFFFC
:10150000FFFFFFFFFFFFFFFFFFFFFFFFFFFFFFFFEB
:10151000FFFFFFFFFFFFFFFFFFFFFFFFFFFFFFFFDB
:10152000FFFFFFFFFFFFFFFFFFFFFFFFFFFFFFFFCB
:10153000FFFFFFFFFFFFFFFFFFFFFFFFFFFFFFFFBB
:10154000FFFFFFFFFFFFFFFFFFFFFFFFFFFFFFFFAB
:10155000FFFFFFFFFFFFFFFFFFFFFFFFFFFFFFFF9B
:10156000FFFFFFFFFFFFFFFFFFFFFFFFFFFFFFFF8B
:10157000FFFFFFFFFFFFFFFFFFFFFFFFFFFFFFFF7B
:10158000FFFFFFFFFFFFFFFFFFFFFFFFFFFFFFFF6B
:10159000FFFFFFFFFFFFFFFFFFFF743611B111B127
:1015A000119111911171117111711151115111514B
:1015B0001970DEFEFFFFFFFFFFFFFFFFFFFFFFFFD2
:1015C000FFFFFFFFFFFFFFFFFFFFFFFFFFFFFFFF2B
:1015D000FFFFFFFFFFFFFFFFFFFFFFFFFFFFFFFF1B
:1015E000FFFFFFFFFFFFFFFFFFFFFFFFFFFFFFFF0B
:1015F000FFFFFFFFFFFFFFFFFFFFDF1F19700970F5
:1016000011511151095094F8FFFFFFFFFFFFFFFF39
:10161000FFFFFFFFFFFFFFFFFFFFFFFFFFFFFFFFDA
:10162000FFFFFFFFFFFFFFFFFFFFFFFFFFFFFFFFCA
:10163000FFFFFFFFFFFFFFFFFFFFFFFFFFFFFFFFBA
:10164000FFFFFFFFFFFFFFFFFFFFFFFFFFFFFFFFAA
:10165000FFFFFFFFFFFFFFFFFFFFFFFFFFFFFFFF9A
:10166000FFFFFFFFFFFFFFFFFFFFFFFFFFFFFFFF8A
:10167000FFFFFFFFFFFFFFFFFFFFFFFFFFFFFFFF7A
:10168000FFFFFFFFFFFFFFFFFFFFFFFFFFFFFFFF6A
:10169000FFFFFFFFFFFFFFFFFFFFFFFFFFFFFFFF5A
:1016A000FFFFFFFFFFFFFFFFFFFFFFFFFFFFFFFF4A
:1016B000FFFFFFFFFFFFFFFFFFFFFFFFFFFFFFFF3A
:1016C000FFFFFFFFFFFFFFFFFFFFFFFFFFFFFFFF2A
:1016D000FFFFFFFFFFFFFFFFFFFFFFFFFFFFFFFF1A
:1016E000FFFFFFFFFFFFFFFFFFFFFFFFFFFFFFFF0A
:1016F000FFFFFFFFFFFFFFFFFFFFFFFFFFFFFFFFFA
:10170000FFFFFFFFFFFFFFFFFFFFFFFFFFFFFFFFE9
:10171000FFFFFFFFFFFFFFFFFFFFFFFFFFFFFFFFD9
:10172000FFFFFFFFFFFFFFFFFFFFFFFFFFFFFFFFC9
:10173000FFFFFFFFFFFFFFFFFFFFFFFFFFFFFFFFB9
:10174000FFFFFFFFFFFFFFFFFFFFFFFFFFFFFFFFA9
:10175000FFFFFFFFFFFFFFFFFFFFFFFFFFFFFFFF99
:10176000FFFFFFFFFFFFFFFFFFFFFFFFFFFFFFFF89
:10177000FFFFFFFFFFFFFFFFFFFFFFFF951911B105
:1017800011911171117111511151115111511151C9
:10179000115111511150A57AFFFFFFFFFFFFFFFF0D
:1017A000FFFFFFFFFFFFFFFFFFFFFFFFFFFFFFFF49
:1017B000FFFFFFFFFFFFFFFFFFFFFFFFFFFFFFFF39
:1017C000FFFFFFFFFFFFFFFFFFFFFFFFFFFFFFFF29
:1017D000FFFFFFFFFFFFB5FB1150115111511170B9
:1017E0001151115073F6FFFFFFFFFFFFFFFFFFFFD7
:1017F000FFFFFFFFFFFFFFFFFFFFFFFFFFFFFFFFF9
:10180000FFFFFFFFFFFFFFFFFFFFFFFFFFFFFFFFE8
:10181000FFFFFFFFFFFFFFFFFFFFFFFFFFFFFFFFD8
:10182000FFFFFFFFFFFFFFFFFFFFFFFFFFFFFFFFC8
:10183000FFFFFFFFFFFFFFFFFFFFFFFFFFFFFFFFB8
:10184000FFFFFFFFFFFFFFFFFFFFFFFFFFFFFFFFA8
:10185000FFFFFFFFFFFFFFFFFFFFFFFFFFFFFFFF98
:10186000FFFFFFFFFFFFFFFFFFFFFFFFFFFFFFFF88
:10187000FFFFFFFFFFFFFFFFFFFFFFFFFFFFFFFF78
:10188000FFFFFFFFFFFFFFFFFFFFFFFFFFFFFFFF68
:10189000FFFFFFFFFFFFFFFFFFFFFFFFFFFFFFFF58
:1018A000FFFFFFFFFFFFFFFFFFFFFFFFFFFFFFFF48
:1018B000FFFFFFFFFFFFFFFFFFFFFFFFFFFFFFFF38
:1018C000FFFFFFFFFFFFFFFFFFFFFFFFFFFFFFFF28
:1018D000FFFFFFFFFFFFFFFFFFFFFFFFFFFFFFFF18
:1018E000FFFFFFFFFFFFFFFFFFFFFFFFFFFFFFFF08
:1018F000FFFFFFFFFFFFFFFFFFFFFFFFFFFFFFFFF8
:10190000FFFFFFFFFFFFFFFFFFFFFFFFFFFFFFFFE7
:10191000FFFFFFFFFFFFFFFFFFFFFFFFFFFFFFFFD7
:10192000FFFFFFFFFFFFFFFFFFFFFFFFFFFFFFFFC7
:10193000FFFFFFFFFFFFFFFFFFFFFFFFFFFFFFFFB7
:10194000FFFFFFFFFFFFFFFFFFFFFFFFFFFFFFFFA7
:10195000FFFFFFFFFFFFFFFFFFFFFFFFFFFFF7DFBF
:10196000097111711151115111511151115111512F
:1019700011511151115111511151115173D5F7DFFD
:10198000FFFFFFFFFFFFFFFFFFFFFFFFFFFFFFFF67
:10199000FFFFFFFFFFFFFFFFFFFFFFFFFFFFFFFF57
:1019A000FFFFFFFFFFFFFFFFFFFFFFFFFFFFFFFF47
:1019B0009D19197009711151115111511151115184
:1019C0001171E73FFFFFFFFFFFFFFFFFFFFFFFFF7B
:1019D000FFFFFFFFFFFFFFFFFFFFFFFFFFFFFFFF17
:1019E000FFFFFFFFFFFFFFFFFFFFFFFFFFFFFFFF07
:1019F000FFFFFFFFFFFFFFFFFFFFFFFFFFFFFFFFF7
:101A0000FFFFFFFFFFFFFFFFFFFFFFFFFFFFFFFFE6
:101A1000FFFFFFFFFFFFFFFFFFFFFFFFFFFFFFFFD6
:101A2000FFFFFFFFFFFFFFFFFFFFFFFFFFFFFFFFC6
:101A3000FFFFFFFFFFFFFFFFFFFFFFFFFFFFFFFFB6
:101A4000FFFFFFFFFFFFFFFFFFFFFFFFFFFFFFFFA6
:101A5000FFFFFFFFFFFFFFFFFFFFFFFFFFFFFFFF96
:101A6000FFFFFFFFFFFFFFFFFFFFFFFFFFFFFFFF86
:101A7000FFFFFFFFFFFFFFFFFFFFFFFFFFFFFFFF76
:101A8000FFFFFFFFFFFFFFFFFFFFFFFFFFFFFFFF66
:101A9000FFFFFFFFFFFFFFFFFFFFFFFFFFFFFFFF56
:101AA000FFFFFFFFFFFFFFFFFFFFFFFFFFFFFFFF46
:101AB000FFFFFFFFFFFFFFFFFFFFFFFFFFFFFFFF36
:101AC000FFFFFFFFFFFFFFFFFFFFFFFFFFFFFFFF26
:101AD000FFFFFFFFFFFFFFFFFFFFFFFFFFFFFFFF16
:101AE000FFFFFFFFFFFFFFFFFFFFFFFFFFFFFFFF06
:101AF000FFFFFFFFFFFFFFFFFFFFFFFFFFFFFFFFF6
:101B0000FFFFFFFFFFFFFFFFFFFFFFFFFFFFFFFFE5
:101B1000FFFFFFFFFFFFFFFFFFFFFFFFFFFFFFFFD5
:101B2000FFFFFFFFFFFFFFFFFFFFFFFFFFFFFFFFC5
:101B3000FFFFFFFFFFFFFFFFFFFFFFFFFFFFFFFFB5
:101B4000FFFF1151115111501150115111511151EB
:101B50001151115111511151115111511151115175
:101B600011502A128CF9EF9FFFFFFFFFFFFFFFFFCD
:101B7000FFFFFFFFFFFFFFFFFFFFFFFFFFFFFFFF75
:101B8000FFFFFFFFFFFFFFFFBE5C429311501151AB
:101B90001151115111511151115111501151115136
:101BA000FFFFFFFFFFFFFFFFFFFFFFFFFFFFFFFF45
:101BB000FFFFFFFFFFFFFFFFFFFFFFFFFFFFFFFF35
:101BC000FFFFFFFFFFFFFFFFFFFFFFFFFFFFFFFF25
:101BD000FFFFFFFFFFFFFFFFFFFFFFFFFFFFFFFF15
:101BE000FFFFFFFFFFFFFFFFFFFFFFFFFFFFFFFF05
:101BF000FFFFFFFFFFFFFFFFFFFFFFFFFFFFFFFFF5
:101C0000FFFFFFFFFFFFFFFFFFFFFFFFFFFFFFFFE4
:101C1000FFFFFFFFFFFFFFFFFFFFFFFFFFFFFFFFD4
:101C2000FFFFFFFFFFFFFFFFFFFFFFFFFFFFFFFFC4
:101C3000FFFFFFFFFFFFFFFFFFFFFFFFFFFFFFFFB4
:101C4000FFFFFFFFFFFFFFFFFFFFFFFFFFFFFFFFA4
:101C5000FFFFFFFFFFFFFFFFFFFFFFFFFFFFFFFF94
:101C6000FFFFFFFFFFFFFFFFFFFFFFFFFFFFFFFF84
:101C7000FFFFFFFFFFFFFFFFFFFFFFFFFFFFFFFF74
:101C8000FFFFFFFFFFFFFFFFFFFFFFFFFFFFFFFF64
:101C9000FFFFFFFFFFFFFFFFFFFFFFFFFFFFFFFF54
:101CA000FFFFFFFFFFFFFFFFFFFFFFFFFFFFFFFF44
:101CB000FFFFFFFFFFFFFFFFFFFFFFFFFFFFFFFF34
:101CC000FFFFFFFFFFFFFFFFFFFFFFFFFFFFFFFF24
:101CD000FFFFFFFFFFFFFFFFFFFFFFFFFFFFFFFF14
:101CE000FFFFFFFFFFFFFFFFFFFFFFFFFFFFFFFF04
:101CF000FFFFFFFFFFFFFFFFFFFFFFFFFFFFFFFFF4
:101D0000FFFFFFFFFFFFFFFFFFFFFFFFFFFFFFFFE3
:101D1000FFFFFFFFFFFFFFFFFFFFFFFFFFFFFFFFD3
:101D2000FFFFFFFF53141150117011501151115149
:101D30001151115111511151115111511151115193
:101D4000115111501150115011511170117021D0B9
:101D500042D374158CB88CD88CB88CD86BD53A52C9
:101D60001970117011511150097011501151115108
:101D70001151115111511151115111512190FFFF68
:101D8000FFFFFFFFFFFFFFFFFFFFFFFFFFFFFFFF63
:101D9000FFFFFFFFFFFFFFFFFFFFFFFFFFFFFFFF53
:101DA000FFFFFFFFFFFFFFFFFFFFFFFFFFFFFFFF43
:101DB000FFFFFFFFFFFFFFFFFFFFFFFFFFFFFFFF33
:101DC000FFFFFFFFFFFFFFFFFFFFFFFFFFFFFFFF23
:101DD000FFFFFFFFFFFFFFFFFFFFFFFFFFFFFFFF13
:101DE000FFFFFFFFFFFFFFFFFFFFFFFFFFFFFFFF03
:101DF000FFFFFFFFFFFFFFFFFFFFFFFFFFFFFFFFF3
:101E0000FFFFFFFFFFFFFFFFFFFFFFFFFFFFFFFFE2
:101E1000FFFFFFFFFFFFFFFFFFFFFFFFFFFFFFFFD2
:101E2000FFFFFFFFFFFFFFFFFFFFFFFFFFFFFFFFC2
:101E3000FFFFFFFFFFFFFFFFFFFFFFFFFFFFFFFFB2
:101E4000FFFFFFFFFFFFFFFFFFFFFFFFFFFFFFFFA2
:101E5000FFFFFFFFFFFFFFFFFFFFFFFFFFFFFFFF92
:101E6000FFFFFFFFFFFFFFFFFFFFFFFFFFFFFFFF82
:101E7000FFFFFFFFFFFFFFFFFFFFFFFFFFFFFFFF72
:101E8000FFFFFFFFFFFFFFFFFFFFFFFFFFFFFFFF62
:101E9000FFFFFFFFFFFFFFFFFFFFFFFFFFFFFFFF52
:101EA000FFFFFFFFFFFFFFFFFFFFFFFFFFFFFFFF42
:101EB000FFFFFFFFFFFFFFFFFFFFFFFFFFFFFFFF32
:101EC000FFFFFFFFFFFFFFFFFFFFFFFFFFFFFFFF22
:101ED000FFFFFFFFFFFFFFFFFFFFFFFFFFFFFFFF12
:101EE000FFFFFFFFFFFFFFFFFFFFFFFFFFFFFFFF02
:101EF000FFFFFFFFFFFFFFFFFFFFFFFFFFFFFFFFF2
:101F0000FFFFFFFFFFFFF7DF197011511151115152
:101F100011511151115111511151115111511151B1
:101F200011511151115011511151115111511150A3
:101F30001151115111511151115111511151115191
:101F4000115111511150115009711151115111516B
:101F500011511151115111511150EFBFFFFFFFFFEE
:101F6000FFFFFFFFFFFFFFFFFFFFFFFFFFFFFFFF81
:101F7000FFFFFFFFFFFFFFFFFFFFFFFFFFFFFFFF71
:101F8000FFFFFFFFFFFFFFFFFFFFFFFFFFFFFFFF61
:101F9000FFFFFFFFFFFFFFFFFFFFFFFFFFFFFFFF51
:101FA000FFFFFFFFFFFFFFFFFFFFFFFFFFFFFFFF41
:101FB000FFFFFFFFFFFFFFFFFFFFFFFFFFFFFFFF31
:101FC000FFFFFFFFFFFFFFFFFFFFFFFFFFFFFFFF21
:101FD000FFFFFFFFFFFFFFFFFFFFFFFFFFFFFFFF11
:101FE000FFFFFFFFFFFFFFFFFFFFFFFFFFFFFFFF01
:101FF000FFFFFFFFFFFFFFFFFFFFFFFFFFFFFFFFF1
:10200000FFFFFFFFFFFFFFFFFFFFFFFFFFFFFFFFE0
:10201000FFFFFFFFFFFFFFFFFFFFFFFFFFFFFFFFD0
